:100000000C94D74B0C94F84B0C94C0D30C94F84B35
:100010000C94F84B0C94F84B0C94F84B0C94F84B54
:100020000C94F84B0C94F84B0C94F84B0C94EBD5C7
:100030000C94F84B0C94F84B0C9408B80C94F84BB7
:100040000C94F84B0C94F84B0C94F84B0C94F84B24
:100050000C94F84B0C94F84B0C94F84B0C94F84B14
:100060000C94F84B0C94DAD30C9469D30C94F84BA1
:100070000C9433CD0C94D5CC0C9411CD0C94F84B3E
:100080000C948BD40C94F84B0C94F84B0C94F84BC8
:100090000C94F84B0C94F84B0C94F84B0C94F84BD4
:1000A0000C94F84B0C94F84B0C94F84B0C9406BF42
:1000B0000C94AABF0C94F84B0C94F84B0C94F9B91F
:1000C0000C94F84B0C94F84B0C94F84B0C94F84BA4
:1000D0000C94F84B0C94F84B0C94F84B0C94F84B94
:1000E0000C94FCA90C94F84B0C94F84B0C94F84B22
:1000F0000C94F84B0C94F84B0C94F84B0C94F84B74
:100100000C94DDBE0C9481BF0C94B4BE0C9458BF0B
:100110000C94F84B0C94F84B0C94F84B0C94F84B53
:100120000C94F84B0C94F84B0C94F84B0C94F84B43
:100130000C94F84B0C945DB90C94F84B0C94F84B60
:100140000C94F84B0C94F84B0C94F84B0C94F84B23
:100150000C94F84B0C94F84B0C94F2A90C94F84BBB
:100160000C94F84B0C94F84B0C94F84B0C94F84B03
:100170000C94F84B0C94F84B0C94F84B0C94F84BF3
:100180000C94F84B0C94F84B0C94F84B0C94F84BE3
:100190000C94F84B0C94F84B0C94F84B0C94F84BD3
:1001A0000C942FBF0C94D3BF0C94F84B0C94F84BC9
:1001B0000C94ABB90C94F84B0C94F84B0C94F84B92
:1001C0000C94F84B0C94F84B0C94F84B0C94F84BA3
:1001D0000C94F84B0C94F84B0C94F84B0C94F84B93
:1001E0000C94F84B0C94F84BE675F075FA750476A0
:1001F0000F76AD7BAD7BAD7BAD7BAD7B1576AD7BFF
:10020000AD7BAD7BAD7BAD7BAD7B177621762B7661
:1002100035763F76AD7BAD7BAD7BAD7BAD7BAD7B8E
:100220004976AD7B9F76AD7BAD7BAD7BAD7BAD7B0A
:10023000AD7BAD7BDE76AD7B9479AD7BAD7BAD7B6D
:10024000AD7BAD7BAD7BAD7BAD7B9479AD7BAD7B89
:10025000AD7B0B7710771A772477267730773B774B
:10026000AD7B4677AD7BAD7B8377AD7BAD7BAD7BE7
:10027000AD7BAD7BAD7BAD7BAD7BAD7BAD7BAD7B3E
:10028000AD7BAD7BAD7BAD7B8D77AD7BAD7BAD7B52
:10029000AD7BAD7BAD7BAD7BAD7BAD7B9777A17748
:1002A000AB77F477FE771778177821782B78357845
:1002B0003F7849784E7858786278AB7BAB7BAB7BE4
:1002C000AB7BAB7BAB7BAB7BAB7BAB7BAB7BAB7BFE
:1002D000AB7BAB7BAB7BAB7BAB7BAB7BAB7BAB7BEE
:1002E000AB7B2178AB7BAB7BAB7BAB7BAB7BAB7B6B
:1002F000AB7BAB7BAB7BAB7BAB7BAB7BAB7BAB7BCE
:10030000AB7BAB7BAB7B6C78767880788A78AB7B89
:10031000AB7BAB7BAB7BAB7BAB7BAB7BAB7B177844
:10032000387BF97AFD7A057BE17AE57AED7AF17A24
:10033000117B247B2C7B307B347B907B097B057984
:1003400016792779AD7BAD7B9F78D775AD7B3879F2
:1003500049795A79947908787C79AD7BB078AD7B0E
:100360006B79C1789478AD7BAD7BAD7BD278E37847
:10037000F4784DBE55BE5DBE65BE6DBE75BE7DBE1C
:1003800085BE78C1D5C0DDC0E5C0EDC0F5C0FDC0FB
:1003900005C10DC115C11DC125C12DC135C13DC14D
:1003A0005DC15DC15DC15DC15DC15DC15DC15DC15D
:1003B0005DC15DC15DC15DC15DC15DC15DC15DC14D
:1003C0005DC15DC15DC15DC15DC15DC15DC15DC13D
:1003D0005DC15DC15DC15DC15DC15DC15DC15DC12D
:1003E0005DC15DC15DC145C14DC15DC15DC15DC145
:1003F0005DC15DC15DC15DC15DC15DC15DC15DC10D
:100400005DC15DC15DC15DC15DC15DC15DC15DC1FC
:100410005DC15DC15DC15DC15DC15DC15DC15DC1EC
:100420005DC15DC15DC15DC15DC15DC15DC15DC1DC
:100430005DC15DC15DC15DC15DC15DC15DC15DC1CC
:100440005DC15DC15DC15DC155C1084AD73B3BCEB1
:10045000016E84BCBFFDC12F3D6C74319ABD5683C3
:100460003DDA3D00C77F11BED9E4BB4C3E916BAA7B
:10047000AABE000000803F05A84CCDB2D44EB938CA
:1004800036A9020C50B9918688083CA6AAAA2ABEB1
:10049000000000803F07634236B79BD8A71A39682F
:1004A0005618AEBAAB558C1D3CB7CC5763BD6DED3D
:1004B000FD753EF6177231BF000000803F08000056
:1004C00000BE922449123EABAAAA2ABECDCCCC4C87
:1004D0003E00000080BEABAAAAAA3E00000000BFFA
:1004E000000000803F0000000000084178D3BB43BB
:1004F00087D1133D190E3CC3BD4282AD2B3E68EC43
:100500008276BED98FE1A93E4C80EFFFBE01C4FFC9
:100510007F3F0000000000000C94E6B00C94545B98
:100520000C94F0CB0C9476CE0C946D5B0C94F47719
:100530000C944D680C9437C50C944DAB0C9465BE6F
:100540000C9438790C945AD10C94325F0C943B770C
:100550000C94DFD00C94AB630C942C600C94E06B87
:100560000C94C6680C940A5F0C94735B0C940E5F39
:100570000C9435760C94FE6F0C9497650C94BED158
:100580000C94B75F0C94D86C0C9446620C9424774E
:100590000C94386D0C9414680C940E4C0C9483CB12
:1005A0000C945DC10C942DC10C949EBC0C949FC006
:1005B0000C94044C0C947F5B0C942CC60C94055E3C
:1005C0000C9482630C943E5F0C9421780C94FA5B3B
:1005D0000C94BFC00C94FA4B0C9483770C948073EA
:1005E0000C94097B0C9459AB0C941DC10C94E2B093
:1005F0000C94D2630C9478C10C940F760C94505EDA
:100600000C94EEB00C94225F0C9467680C946B7998
:100610000C942E5F0C9418680C9418600C946278FB
:100620000C94FD7A0C94615B0C949E5B0C9495B0D9
:100630000C94387B0C9427BE0C94127E0C94C3C08F
:100640000C94755F0C94A8D00C9414600C94525FB9
:100650000C94315E0C9418CB0C94BF5B0C942A5F05
:100660000C94805C0C94365E0C94F5C00C943A5F4C
:100670000C9410600C94135D0C94AAB00C948A5BDB
:100680000C94D2780C94FA750C940A630C94675B02
:100690000C94425F0C94AB580C9416790C9455BE94
:1006A0000C94307B0C94D7750C94BB670C942B7610
:1006B0000C9404600C943ABE0C940B640C94C178B6
:1006C0000C949B680C941EBE0C943D7D0C94CA5BEC
:1006D0000C94A44F0C94565F0C94A95B0C943E733D
:1006E0000C944E5F0C944D4C0C94AA5E0C94F478D0
:1006F0000C9458780C9417760C94495C0C9445AB88
:100700000C9435C10C9415760C9480780C94E57A91
:100710000C9455C10C9419B20C9405790C94907BEF
:100720000C94636C0C9436690C94DE760C9442AF96
:100730000C94FDC00C942B780C94EAB00C94FE77CA
:100740000C9440AF0C945E600C9475BE0C944DBE3E
:100750000C9458670C941ABE0C9432840C94E35C8D
:100760000C9422BE0C945DAB0C94F66C0C946D7DD5
:100770000C94A5C00C940AAF0C9453600C94655E65
:100780000C94F66F0C940C680C9446AF0C94E5C076
:100790000C94165F0C94F0750C94236D0C9484BC2F
:1007A0000C9441AB0C94575E0C94F17A0C9494BD6C
:1007B0000C9455AB0C941C600C9479960C94FF7BB4
:1007C0000C94A87D0C94A6670C945DCB0C945E5E93
:1007D0000C944DC10C94057B0C946C780C945E4C7D
:1007E0000C9411CC0C9497770C945FBD0C94A4617D
:1007F0000C94EDC00C943EBE0C942C5D0C9435789A
:100800000C94617D0C9470CC0C94B5720C94FE61C8
:100810000C94BB830C9434600C94CE620C94AB7B30
:100820000C9448D00C94EF7B0C9446630C942C7B76
:100830000C940B770C94D2710C9430600C9422625F
:100840000C943D7E0C943F780C941E5F0C94FE68D3
:100850000C9465AB0C9425C10C94DDC00C944978C4
:100860000C944FC50C94D5C00C94A1770C943077A0
:100870000C9494790C94347B0C94AD7B0C9409D338
:100880000C94387D0C94E3780C9417780C9436C54E
:100890000C94C6B00C946C5E0C94FA610C942176A6
:1008A0000C94A8620C9448CF0C943DC10C944677EC
:1008B0000C9482CC0C9491BC0C946D620C94115CE1
:1008C0000C948B5E0C94F97A0C94CEBD0C94058636
:1008D0000C9494780C94065F0C9438600C94E67534
:1008E0000C943F5D0C94125F0C9406AF0C943C602A
:1008F0000C9485BE0C948A780C9405C10C941C68E9
:100900000C94265F0C9488C50C94F1BD0C94A662DF
:100910000C94B0780C943F760C94465F0C94955BE5
:100920000C945F880C94B45B0C94D0720C9442B21B
:100930000C94E17A0C948D770C9420600C941068E0
:100940000C9445C10C94E57C0C94657D0C9449791C
:100950000C94795B0C94ED7A0C94E77D0C942779D8
:100960000C94365F0C9415C10C9436BE0C942A84FA
:100970000C944E780C94247B0C9451AB0C947DBE5B
:100980000C9449760C94697D0C9408780C94A96DAC
:100990000C949F760C9404760C9481680C940DC191
:1009A0000C946BC50C9428600C9400600C94985FB8
:1009B0000C941A5F0C9413530C94AD5D0C944A5F25
:1009C0000C9408600C94AB770C945A790C941A77B9
:1009D0000C9424600C94117B0C94945F0C947C799F
:1009E0000C94E35B0C946DBE0C945DBE0C9449AB0F
:1009F0000C94A96C0C940C600C94FC5F0C942E84E9
:100A00000C945D7D0C9408AF0C9448600C94AA5C27
:100A10000C949F780C94DCCF0C9410770C94267770
:100A20000C9461AB0C9476780C9418AC4D6F746F89
:100A30007220256320706F7765722073746174650E
:100A40003A25322E30660A005B257325735D20251A
:100A50007320257320706F736974696F6E25313848
:100A60002E336625730A005B257325735D2025737D
:100A7000202573206F66667365742532302E3366C9
:100A800025730A005B257325735D202573207A6525
:100A9000726F206261636B6F66662531392E336633
:100AA00025730A005B257325735D202573206C6117
:100AB000746368206261636B6F66662531382E331C
:100AC0006625730A005B257325735D202573206CF2
:100AD000617463682076656C6F636974792531335E
:100AE0002E306625732F6D696E0A005B25732573A2
:100AF0005D202573207365617263682076656C6F75
:100B0000636974792531322E306625732F6D696ED5
:100B10000A005B257325735D202573207377697444
:100B20006368206D617825313764205B303D6F66E6
:100B3000662C313D686F6D696E672C323D6C696D56
:100B400069742C333D6C696D69742B686F6D696EC7
:100B5000675D0A005B257325735D2025732073771D
:100B600069746368206D696E25313764205B303DA0
:100B70006F66662C313D686F6D696E672C323D6C17
:100B8000696D69742C333D6C696D69742B686F6D88
:100B9000696E675D0A005B257325735D20257320F0
:100BA0007261646975732076616C75652532302ECB
:100BB000346625730A005B257325735D2025732039
:100BC0006A756E6374696F6E2064657669617469B5
:100BD0006F6E2531342E3466257320286C61726760
:100BE000657220697320666173746572290A005BFF
:100BF000257325735D202573206A65726B20686FED
:100C00006D696E672531362E306625732F6D696EDE
:100C10005E33202A2031206D696C6C696F6E0A008A
:100C20005B257325735D202573206A65726B206DCB
:100C30006178696D756D2531352E306625732F6DA0
:100C4000696E5E33202A2031206D696C6C696F6E8D
:100C50000A005B257325735D20257320747261760D
:100C6000656C206D696E696D756D2531372E336643
:100C700025730A005B257325735D2025732074722C
:100C80006176656C206D6178696D756D2531372EE3
:100C9000336625730A005B257325735D2025732059
:100CA00076656C6F63697479206D6178696D756DB7
:100CB0002531312E306625732F6D696E0A005B2554
:100CC0007325735D202573206665656472617465A4
:100CD000206D6178696D756D2531312E3066257313
:100CE0002F6D696E0A005B257325735D20257320C7
:100CF00061786973206D6F646525313864202573D0
:100D00000A005B6D615D20206D696E206172632059
:100D10007365676D656E742531382E336625730AE9
:100D2000005B736C5D2020736F6674206C696D6965
:100D30007420656E61626C65253132640A005B6304
:100D4000745D202063686F7264616C20746F6C65E1
:100D500072616E63652531372E346625730A005B38
:100D60006A615D20206A756E6374696F6E206163CD
:100D700063656C65726174696F6E25382E30662507
:100D8000730A005B6764695D2064656661756C74F5
:100D90002067636F64652064697374616E636520A6
:100DA0006D6F6465253264205B303D4739302C31EE
:100DB0003D4739315D0A005B6770615D206465669F
:100DC00061756C742067636F64652070617468205E
:100DD000636F6E74726F6C253364205B303D4736F1
:100DE000312C313D4736312E312C323D4736345D82
:100DF0000A005B67636F5D2064656661756C7420D3
:100E000067636F646520636F6F72642073797374B6
:100E1000656D253364205B312D3620284735342D10
:100E2000473539295D0A005B67756E5D206465662C
:100E300061756C742067636F646520756E69747387
:100E4000206D6F6465253564205B303D4732302C62
:100E5000313D4732315D0A005B67706C5D2064652F
:100E60006661756C742067636F646520706C616E79
:100E70006525313064205B303D4731372C313D47AB
:100E800031382C323D4731395D0A00256320776FB8
:100E9000726B206F66667365743A2531322E336645
:100EA00025730A002563206D616368696E65207093
:100EB0006F736E3A2531312E336625730A00256330
:100EC00020706F736974696F6E3A2531352E336601
:100ED00025730A00546F6F6C206E756D6265722009
:100EE00020202020202020202025640A004665653F
:100EF000642072617465206D6F64653A2020202043
:100F0000202025730A0044697374616E6365206D47
:100F10006F64653A2020202020202025730A00508D
:100F2000617468204D6F64653A20202020202020C5
:100F30002020202025730A00506C616E653A202025
:100F40002020202020202020202020202025730A5F
:100F5000004D6F74696F6E206D6F64653A202020BC
:100F600020202020202025730A00436F6F726469BF
:100F70006E6174652073797374656D3A2020202545
:100F8000730A00556E6974733A20202020202020B7
:100F9000202020202020202025730A00486F6D6922
:100FA0006E672073746174653A2020202020202011
:100FB0002025730A0046656564686F6C642073744D
:100FC0006174653A20202020202025730A004D6F8F
:100FD00074696F6E2073746174653A20202020203C
:100FE00020202025730A004379636C6520737461A7
:100FF00074653A20202020202020202025730A001C
:10100000526177206D616368696E652073746174E5
:10101000653A20202025730A004D616368696E657A
:101020002073746174653A202020202020202573CD
:101030000A004C696E65206E756D6265723A2531E5
:10104000302E30660A004665656420726174653A28
:101050002531362E336625732F6D696E0A0056656D
:101060006C6F636974793A2531372E336625732F97
:101070006D696E0A00CC109B107B10473935202D0E
:1010800020756E6974732D7065722D7265766F6C44
:101090007574696F6E206D6F646500473934202D5B
:1010A00020756E6974732D7065722D6D696E75741F
:1010B00065206D6F64652028692E652E2066656544
:1010C0006472617465206D6F64652900473933204F
:1010D0002D20696E76657273652074696D65206D6B
:1010E0006F6465000811E810473931202D20696EC2
:1010F0006372656D656E74616C2064697374616E92
:101100006365206D6F646500473930202D20616272
:10111000736F6C7574652064697374616E636520A8
:101120006D6F646500591141112B11473634202D24
:1011300020636F6E74696E756F7573206D6F646573
:10114000004736312E31202D20657861637420737D
:10115000746F70206D6F646500473631202D2065F7
:10116000786163742070617468206D6F64650093AA
:101170001184117511473139202D20595A20706C76
:10118000616E6500473138202D20585A20706C61FF
:101190006E6500473137202D20585920706C616EE4
:1011A00065001F120D12F411D311AC114738302015
:1011B0002D2063616E63656C206D6F74696F6E20A6
:1011C0006D6F646520286E6F6E652061637469764B
:1011D000652900473320202D20636F756E7465727A
:1011E00020636C6F636B776973652061726320663F
:1011F00065656400473220202D20636C6F636B7738
:1012000069736520617263206665656400473120FB
:10121000202D206C696E65617220666565640047EB
:101220003020202D206C696E6561722074726176A9
:101230006572736520287365656B2900E612CC1210
:10124000B21298127E1264124A12473539202D20AC
:10125000636F6F7264696E6174652073797374650E
:101260006D203600473538202D20636F6F7264691A
:101270006E6174652073797374656D203500473530
:1012800037202D20636F6F7264696E6174652073FF
:10129000797374656D203400473536202D20636FD7
:1012A0006F7264696E6174652073797374656D2003
:1012B0003300473535202D20636F6F7264696E618E
:1012C00074652073797374656D203200473534205E
:1012D0002D20636F6F7264696E617465207379731A
:1012E00074656D203100473533202D206D616368B2
:1012F000696E6520636F6F7264696E6174652073D7
:10130000797374656D00191313130C13486F6D69AD
:101310006E6700486F6D6564004E6F7420486F6D96
:101320006564004D13481343133D1338132F1345C1
:101330006E6420486F6C6400486F6C6400446563A1
:10134000656C00506C616E0053796E63004F666689
:101350000060135C135713486F6C640052756E0085
:1013600053746F70008A1380137A1373136F134AC8
:101370006F6700486F6D696E670050726F6265003D
:101380004D616368696E696E67004F666600C013E1
:10139000BA13B413AF13AB13A5139C13536875742E
:1013A000646F776E004379636C6500456E6400532B
:1013B000746F7000416C61726D00526561647900F8
:1013C000496E697469616C697A696E670023141DDE
:1013D00014171412140E140A140514FF13F913F23F
:1013E00013EE13E51353687574646F776E004A6FDC
:1013F0006700486F6D696E67004379636C650050E4
:10140000726F626500486F6C640052756E00456EC5
:10141000640053746F7000416C61726D00526561BD
:10142000647900496E697469616C697A696E6700F4
:101430004A143414473231202D206D696C6C696D6B
:1014400065746572206D6F646500473230202D2011
:10145000696E63686573206D6F6465008414791428
:101460006D1464145B7261646975735D005B696E11
:10147000686962697465645D005B7374616E646160
:1014800072645D005B64697361626C65645D009E9B
:10149000149A1495142064656700206D6D0020690E
:1014A0006E002A2A2A204E4F54494345202A2A2AD0
:1014B00020526573657474696E672062617564207B
:1014C0007261746520746F202573005B6E65745DB6
:1014D000206E6574776F726B206D6F646525313790
:1014E00064205B303D6D61737465725D0A005B6200
:1014F0006175645D2055534220626175642072619C
:10150000746525313564205B313D393630302C32FD
:101510003D31393230302C333D33383430302C3497
:101520003D35373630302C353D3131353230302C89
:10153000363D3233303430305D0A005B65785D20F3
:1015400020656E61626C6520666C6F7720636F6EDC
:1015500074726F6C25313064205B303D6F66662C91
:10156000313D584F4E2F584F46462C20323D525455
:10157000532F4354535D0A005B65655D2020656E03
:1015800061626C65206563686F25313864205B306B
:101590003D6F66662C313D6F6E5D0A005B65635D75
:1015A0002020657870616E64204C4620746F204363
:1015B000524C46206F6E205458253664205B303DD7
:1015C0006F66662C313D6F6E5D0A00FE15F915F3EE
:1015D00015ED15E715E015D91532333034303000EC
:1015E0003131353230300035373630300033383431
:1015F0003030003139323030003936303000300090
:101600007379730066620000000007025D7D6D6201
:10161000A6622D34850BDC43737973006676000077
:1016200000000703617D6D62A6623134EC51783FA2
:10163000737973006870000000000700657D6D62BB
:10164000D26335340000803F737973006876000000
:1016500000000700697D6D623D7D39340000004166
:101660007379730069640000000004006D7DE57CFF
:10167000A662293400000000000000006E00000097
:1016800000000100065FE35B8263192C000000008C
:10169000000000006C696E6500000100065FFA5BE7
:1016A0008263192C000000000000000076656C00C9
:1016B000000000026C5E115CA6622934000000008C
:1016C0000000000066656564000000028B5E495CF6
:1016D000A6622934000000000000000073746174E9
:1016E000000000000A5F545BA6622934000000007D
:1016F000000000006D616373000000000E5F615B1D
:10170000A6622934000000000000000063796373C2
:1017100000000000125F675BA66229340000000031
:10172000000000006D6F747300000000165F6D5BB9
:10173000A66229340000000000000000686F6C649D
:10174000000000001A5F735BA662293400000000ED
:1017500000000000756E697400000000225F7F5B6E
:10176000A66229340000000000000000636F6F7261
:1017700000000000265F8A5BA6622934000000009A
:10178000000000006D6F6D6F000000002A5F955B28
:10179000A66229340000000000000000706C616E39
:1017A000000000002E5F9E5BA6622934000000004E
:1017B000000000007061746800000000325FA95BE7
:1017C000A662293400000000000000006469737400
:1017D00000000000365FB45BA66229340000000000
:1017E0000000000066726D6F000000003A5FBF5B92
:1017F000A66229340000000000000000746F6F6CC6
:10180000000000003E5FCA5BA662293400000000B1
:101810006D706F006D706F78000000034860AA5C07
:10182000A6622934000000006D706F006D706F7942
:10183000000000034860AA5CA66229340000000092
:101840006D706F006D706F7A000000034860AA5CD5
:10185000A6622934000000006D706F006D706F612A
:10186000000000034860AA5CA66229340000000062
:101870006D706F006D706F62000000034860AA5CBD
:10188000A6622934000000006D706F006D706F63F8
:10189000000000034860AA5CA66229340000000032
:1018A000706F7300706F7378000000033C60805CA1
:1018B000A662293400000000706F7300706F7379A6
:1018C000000000033C60805CA66229340000000038
:1018D000706F7300706F737A000000033C60805C6F
:1018E000A662293400000000706F7300706F73618E
:1018F000000000033C60805CA66229340000000008
:10190000706F7300706F7362000000033C60805C56
:10191000A662293400000000706F7300706F73635B
:10192000000000033C60805CA662293400000000D7
:101930006F6673006F667378000000035360E35CAA
:10194000A6622934000000006F6673006F66737929
:10195000000000035360E35CA6622934000000002D
:101960006F6673006F66737A000000035360E35C78
:10197000A6622934000000006F6673006F66736111
:10198000000000035360E35CA662293400000000FD
:101990006F6673006F667362000000035360E35C60
:1019A000A6622934000000006F6673006F667363DF
:1019B000000000035360E35CA662293400000000CD
:1019C000686F6D00686F6D65000000001E5F795BD9
:1019D000365E293400000000686F6D00686F6D7816
:1019E000000000003C60FE61A662EE2B00000000DB
:1019F000686F6D00686F6D79000000003C60FE61EB
:101A0000A662EF2B00000000686F6D00686F6D7AB2
:101A1000000000003C60FE61A662F02B00000000A8
:101A2000686F6D00686F6D61000000003C60FE61D2
:101A3000A662F12B00000000686F6D00686F6D6298
:101A4000000000003C60FE61A662F22B0000000076
:101A5000686F6D00686F6D63000000003C60FE61A0
:101A6000A662F32B00000000707262007072626563
:101A70000000000036C5FE61A662F42B00000000E5
:101A800070726200707262780000000336C56D6289
:101A9000A662F52B0000000070726200707262791D
:101AA0000000000336C56D62A662F92B000000003D
:101AB000707262007072627A0000000336C56D6257
:101AC000A662FD2B000000007072620070726261FD
:101AD0000000000336C56D62A662012C0000000004
:101AE00070726200707262620000000336C56D623F
:101AF000A662052C000000007072620070726263C2
:101B00000000000336C56D62A662092C00000000CB
:101B10006A6F67006A6F67780000000036C5FA6177
:101B2000505E132C000000006A6F67006A6F6779CF
:101B30000000000036C5FA61575E132C000000005B
:101B40006A6F67006A6F677A0000000036C5FA6145
:101B50005E5E132C000000006A6F67006A6F6761A9
:101B60000000000036C5FA61655E132C000000001D
:101B70007077720070777231000000005E60135D54
:101B8000A66229340000000070777200707772320C
:101B9000000000005E60135DA662293400000000B2
:101BA0007077720070777233000000005E60135D22
:101BB000A6622934000000007077720070777234DA
:101BC000000000005E60135DA66229340000000082
:101BD00000000000737200000000000040AF06AF7C
:101BE00008AF2934000000000000000071720000FE
:101BF00000000000E2B095B0A662293400000000A9
:101C0000000000007169000000000000E6B0AAB00A
:101C1000A66229340000000000000000716F00007F
:101C200000000000EAB0C6B0A6622934000000003F
:101C300000000000657200000000000036C518AC0E
:101C4000A662293400000000000000007166000058
:101C50000000000036C5FA61315E29340000000042
:101C60000000000072780000000000006BC5A6674D
:101C7000A662293400000000000000006D736700B8
:101C80000000000037C5FA61A66229340000000098
:101C900000000000636C65617200000036C51353DC
:101CA00013532934000000000000000074657374B1
:101CB0000000000036C5E77DC3C0293400000000E5
:101CC00000000000646566610000000036C5127EF9
:101CD000A46129340000000000000000626F6F74EE
:101CE0000000000036C53D7E387D2934000000002C
:101CF0000000000068656C700000000036C5A87D1B
:101D0000A662293400000000000000006800000006
:101D10000000000036C5A87DA6622934000000003E
:101D200031000000316D6100000003001EBEFE6145
:101D3000A8625C53000000003100000031736100B4
:101D40000000030322BE6D6284BC64536666E63FF6
:101D5000310000003174720000000B0427BE6D6278
:101D600091BC68530000204231000000316D6900D1
:101D70000000030036BEFE619EBC5D5300000041C2
:101D80003100000031706F00000003003ABEFE61B8
:101D9000CE625E53000000003100000031706D0023
:101DA000000003003EBEFE615FBD5F5300000040C7
:101DB00032000000326D6100000003001EBEFE61B3
:101DC000A86278530000803F320000003273610047
:101DD0000000030322BE6D6284BC80536666E63F4A
:101DE000320000003274720000000B0427BE6D62E6
:101DF00091BC84530000204232000000326D690023
:101E00000000030036BEFE619EBC79530000004115
:101E10003200000032706F00000003003ABEFE6125
:101E2000CE627A53000000003200000032706D0074
:101E3000000003003EBEFE615FBD7B53000000401A
:101E400033000000336D6100000003001EBEFE6120
:101E5000A86294530000803F330000003373610098
:101E60000000030322BE6D6284BC9C536666E63F9D
:101E7000330000003374720000000B0427BE6D6253
:101E800091BCA0530000204233000000336D690074
:101E90000000030036BEFE619EBC95530000004169
:101EA0003300000033706F00000003003ABEFE6193
:101EB000CE6296530000803F3300000033706D0007
:101EC000000003003EBEFE615FBD9753000000406E
:101ED00034000000346D6100000003001EBEFE618E
:101EE000A862B05300000040340000003473610069
:101EF0000000030322BE6D6284BCB8536666E63FF1
:101F0000340000003474720000000B0427BE6D62C0
:101F100091BCBC536076074034000000346D69000A
:101F20000000030036BEFE619EBCB153000080403D
:101F30003400000034706F00000003003ABEFE6100
:101F4000CE62B253000000003400000034706D0017
:101F5000000003003EBEFE615FBDB35300000040C1
:101F60007800000078616D0000000300B75F2C5D11
:101F70003F5DAA2A0000803F7800000078766D005F
:101F800000000B0000606D62BB67AF2A0050434742
:101F9000780000007866720000000B00FC5F6D6244
:101FA000BB67AB2A005043477800000078746E008E
:101FB00000000B0308606D62BB67B72A00000000D9
:101FC0007800000078746D0000000B0304606D62FF
:101FD000BB67B32A0000D24378000000786A6D0026
:101FE00000000B000C606D62AD5DBB2A00409C459B
:101FF00078000000786A680000000B0010606D62D5
:10200000055EBF2A00401C4678000000786A640024
:1020100000000B0414606D62BB67C72A0AD7233C1B
:102020007800000078736E00000003001C60FE6101
:10203000A5C0CE290000803F7800000078737800AA
:10204000000003002060FE61A5C0CF290000000051
:10205000780000007873760000000B0024606D6249
:10206000BB67CF2A00803B4578000000786C760083
:1020700000000B0028606D62BB67D32A0000C842D5
:1020800078000000786C620000000B032C606D6229
:10209000BB67D72A0000A04178000000787A620070
:1020A00000000B0330606D62BB67DB2A000040401C
:1020B0007900000079616D0000000300B75F2C5DBE
:1020C0003F5DDF2A0000803F7900000079766D00D7
:1020D00000000B0000606D62BB67E42A00504347BC
:1020E000790000007966720000000B00FC5F6D62F1
:1020F000BB67E02A005043477900000079746E0006
:1021000000000B0308606D62BB67EC2A0000000052
:102110007900000079746D0000000B0304606D62AB
:10212000BB67E82A0000D24379000000796A6D009D
:1021300000000B000C606D62AD5DF02A00409C4514
:1021400079000000796A680000000B0010606D6281
:10215000055EF42A00401C4679000000796A64009C
:1021600000000B0414606D62BB67FC2A0AD7233C95
:102170007900000079736E00000003001C60FE61AE
:10218000A5C0D0290000803F790000007973780055
:10219000000003002060FE61A5C0D12900000000FE
:1021A000790000007973760000000B0024606D62F6
:1021B000BB67042B00803B4579000000796C7600FA
:1021C00000000B0028606D62BB67082B0000C8424E
:1021D00079000000796C620000000B032C606D62D6
:1021E000BB670C2B0000A04179000000797A6200E7
:1021F00000000B0330606D62BB67102B0000404095
:102200007A0000007A616D0000000300B75F2C5D6A
:102210003F5D142B0000803F7A0000007A766D004D
:1022200000000B0000606D62BB67192B0000964434
:102230007A0000007A66720000000B00FC5F6D629D
:10224000BB67152B000096447A0000007A746E007C
:1022500000000B0308606D62BB67212B00000000CB
:102260007A0000007A746D0000000B0304606D6258
:10227000BB671D2B0000C8427A0000007A6A6D001F
:1022800000000B000C606D62AD5D252B0000C842A4
:102290007A0000007A6A680000000B0010606D622E
:1022A000055E292B00007A447A0000007A6A6400F7
:1022B00000000B0414606D62BB67312B0AD7233C0E
:1022C0007A0000007A736E00000003001C60FE615B
:1022D000A5C0D229000000007A0000007A737800BF
:1022E000000003002060FE61A5C0D3290000803FEC
:1022F0007A0000007A73760000000B0024606D62A3
:10230000BB67392B000096447A0000007A6C760097
:1023100000000B0028606D62BB673D2B0000C842C7
:102320007A0000007A6C620000000B032C606D6282
:10233000BB67412B0000A0417A0000007A7A62005E
:1023400000000B0330606D62BB67452B000020412D
:102350006100000061616D0000000300B75F2C5D4B
:102360003F5D492B0000803F6100000061766D00F9
:102370000000030000606D62D2634E2B00606A476C
:10238000610000006166720000000300FC5F6D6286
:10239000D2634A2B00803B476100000061746E00ED
:1023A0000000030308606D62BB67562B0000C84342
:1023B0006100000061746D000000030304606D6241
:1023C000D263522B000080BF61000000616A6D0083
:1023D000000003000C606D62AD5D5A2B0080BB46AF
:1023E00061000000616A68000000030010606D6217
:1023F000055E5E2B0080BB4661000000616A6400E0
:102400000000030414606D62D263662BCDCCCC3D1A
:10241000610000006172610000000B0318606D62D2
:10242000D2636A2B0000803F6100000061736E0080
:10243000000003001C60FE61A5C0D4290000803F9D
:102440006100000061737800000003002060FE61FD
:10245000A5C0D5290000000061000000617376006E
:102460000000030024606D62D2636E2B0080BB45C8
:1024700061000000616C76000000030028606D625E
:10248000D263722B00007A4461000000616C62002C
:10249000000003032C606D62D263762B0000A04025
:1024A00061000000617A62000000030330606D6229
:1024B000D2637A2B000000406200000062616D0070
:1024C00000000300B75F2C5D3F5D7E2B0000000025
:1024D0006200000062766D000000030000606D6223
:1024E000D263832B000061456200000062667200C7
:1024F00000000300FC5F6D62D2637F2B000061452A
:102500006200000062746E000000030308606D62E8
:10251000BB678B2B000080BF6200000062746D00FF
:102520000000030304606D62D263872B000080BF4C
:1025300062000000626A6D00000003000C606D62C2
:10254000AD5D8F2B0000A04162000000626A640054
:102550000000030014606D62D2639B2B0AD7233CFA
:10256000620000006272610000000B0318606D627F
:10257000D2639F2B0000803F6300000063616D0009
:1025800000000300B75F2C5D3F5DB32B000000002F
:102590006300000063766D000000030000606D6260
:1025A000D263B82B000061456300000063667200CF
:1025B00000000300FC5F6D62D263B42B0000614534
:1025C0006300000063746E000000030308606D6226
:1025D000BB67C02B000080BF6300000063746D0008
:1025E0000000030304606D62D263BC2B000080BF57
:1025F00063000000636A6D00000003000C606D6200
:10260000AD5DC42B0000A04163000000636A64005C
:102610000000030014606D62D263D02B0AD7233C04
:10262000630000006372610000000B0318606D62BC
:10263000D263D42B0000803F70310000703166728D
:102640007100030041AB6D62D26338520000C84292
:1026500070310000703163736C00030045AB6D6234
:10266000D2633C5200007A447031000070316373D1
:102670006800030049AB6D62D26340520000FA4427
:1026800070310000703163706C0003034DAB6D62FC
:10269000D26344520000003E70310000703163701C
:1026A0006800030351AB6D62D2634852CDCC4C3EFF
:1026B00070310000703177736C00030055AB6D62B0
:1026C000D2634C5200007A4470310000703177734D
:1026D0006800030059AB6D62D26350520000FA44A7
:1026E00070310000703177706C0003035DAB6D6278
:1026F000D26354520000003E703100007031777098
:102700006800030361AB6D62D2635852CDCC4C3E7E
:10271000703100007031706F6600030365AB6D624D
:10272000D2635C52CDCCCC3D67353400673534780C
:1027300000000B0334606D62BB671A2A00000000C2
:10274000673534006735347900000B0334606D62FF
:10275000BB671E2A00000000673534006735347AF5
:1027600000000B0334606D62BB67222A000000008A
:10277000673534006735346100000B0334606D62E7
:10278000BB67262A000000006735340067353462D5
:1027900000000B0334606D62BB672A2A0000000052
:1027A000673534006735346300000B0334606D62B5
:1027B000BB672E2A00000000673535006735357885
:1027C00000000B0334606D62BB67322A0000524385
:1027D000673535006735357900000B0334606D626D
:1027E000BB67362A00005243673535006735357AB6
:1027F00000000B0334606D62BB673A2A00000000E2
:10280000673535006735356100000B0334606D6254
:10281000BB673E2A0000000067353500673535622A
:1028200000000B0334606D62BB67422A00000000A9
:10283000673535006735356300000B0334606D6222
:10284000BB67462A000000006735360067353678DA
:1028500000000B0334606D62BB674A2A00005243DC
:10286000673536006735367900000B0334606D62DA
:10287000BB674E2A0000A041673536006735367ABF
:1028800000000B0334606D62BB67522A000020C158
:10289000673536006735366100000B0334606D62C2
:1028A000BB67562A00000000673536006735366280
:1028B00000000B0334606D62BB675A2A0000000001
:1028C000673536006735366300000B0334606D6290
:1028D000BB675E2A00000000673537006735377830
:1028E00000000B0334606D62BB67622A00000000C9
:1028F000673537006735377900000B0334606D6248
:10290000BB67662A00000000673537006735377AF5
:1029100000000B0334606D62BB676A2A0000000090
:10292000673537006735376100000B0334606D622F
:10293000BB676E2A000000006735370067353762D5
:1029400000000B0334606D62BB67722A0000000058
:10295000673537006735376300000B0334606D62FD
:10296000BB67762A00000000673538006735387885
:1029700000000B0334606D62BB677A2A0000000020
:10298000673538006735387900000B0334606D62B5
:10299000BB677E2A00000000673538006735387A4B
:1029A00000000B0334606D62BB67822A00000000E8
:1029B000673538006735386100000B0334606D629D
:1029C000BB67862A0000000067353800673538622B
:1029D00000000B0334606D62BB678A2A00000000B0
:1029E000673538006735386300000B0334606D626B
:1029F000BB678E2A000000006735390067353978DB
:102A000000000B0334606D62BB67922A0000000077
:102A1000673539006735397900000B0334606D6222
:102A2000BB67962A00000000673539006735397AA0
:102A300000000B0334606D62BB679A2A000000003F
:102A4000673539006735396100000B0334606D620A
:102A5000BB679E2A00000000673539006735396280
:102A600000000B0334606D62BB67A22A0000000007
:102A7000673539006735396300000B0334606D62D8
:102A8000BB67A62A00000000673932006739327838
:102A90000000010334606D62A6628A2C0000000011
:102AA00067393200673932790000010334606D62A2
:102AB000A6628E2C00000000673932006739327A36
:102AC0000000010334606D62A662922C00000000D9
:102AD00067393200673932610000010334606D628A
:102AE000A662962C00000000673932006739326216
:102AF0000000010334606D62A6629A2C00000000A1
:102B000067393200673932630000010334606D6257
:102B1000A6629E2C000000006732380067323878C9
:102B20000000010338606D62A662A22C0000000064
:102B300067323800673238790000010338606D620F
:102B4000A662A62C00000000673238006732387A8F
:102B50000000010338606D62A662AA2C000000002C
:102B600067323800673238610000010338606D62F7
:102B7000A662AE2C0000000067323800673238626F
:102B80000000010338606D62A662B22C00000000F4
:102B900067323800673238630000010338606D62C5
:102BA000A662B62C0000000067333000673330782F
:102BB0000000010338606D62A662BA2C00000000BC
:102BC00067333000673330790000010338606D628D
:102BD000A662BE2C00000000673330006733307AF5
:102BE0000000010338606D62A662C22C0000000084
:102BF00067333000673330610000010338606D6275
:102C0000A662C62C000000006733300067333062D4
:102C10000000010338606D62A662CA2C000000004B
:102C200067333000673330630000010338606D6242
:102C3000A662CE2C000000006A6964006A696461C3
:102C40000000000036C54662AB635134000000004E
:102C50006A6964006A6964620000000036C5466201
:102C6000AB635534000000006A6964006A696463FC
:102C70000000000036C54662AB6359340000000016
:102C80006A6964006A6964640000000036C54662CF
:102C9000AB635D3400000000737973006A6100006B
:102CA00000000F00565F6D62BB67E8290024F449FD
:102CB000737973006374000000000F04755F6D6228
:102CC000BB67EC290AD7233C73797300736C00004F
:102CD00000000700945FFE61A862F0290000000078
:102CE000737973007374000000000700BFC0FE61B9
:102CF0009FC0C3290000803F737973006D7400008A
:102D0000000007021ABE6D6294BD585300000040D7
:102D1000000000006D6500000000000037C5F1BD37
:102D2000F1BD293400000000000000006D640000C7
:102D30000000000037C5CEBDCEBD29340000000024
:102D400073797300656A0000000007002A84FE6141
:102D5000CE62DE330000803F737973006A76000034
:102D6000000007002E84FE61BB83F8370000A040FE
:102D7000737973006A730000000007003284FE61FB
:102D8000CE62FA370000803F7379730074760000DA
:102D9000000007002CC6FE61CE62BF540000803FD9
:102DA000737973007176000000000700EEB0FE61D9
:102DB000466391520000000073797300737600003F
:102DC0000000070046AFFE610A639E520000803F8C
:102DD00073797300736900000000070042AF22623C
:102DE0000AAF9F5200007A43737973006563000055
:102DF000000007000C68FE61C668DF3300000000B9
:102E00007379730065650000000007001068FE61BB
:102E10003669E033000000007379730065780000C4
:102E2000000007001468FE61FE68E1330000803F87
:102E30007379730062617564000004001868FE61B4
:102E40005867E2330000A040737973006E65740028
:102E5000000007001C68FE61A8624034000000000A
:102E60007379730067706C0000000700425FFE61B9
:102E70000A63FE29000000007379730067756E0015
:102E800000000700465FFE61CE62FF290000803F20
:102E90007379730067636F00000007004A5FFE618B
:102EA000A862FD290000803F73797300677061009C
:102EB000000007004E5FFE610A63002A0000004028
:102EC000737973006764690000000700525FFE6158
:102ED000CE62012A000000000000000067630000CD
:102EE0000000000036C5EF7BFF7B293400000000A6
:102EF000000000006D61000000000B04985F6D622F
:102F0000BB67F529CDCCCC3D000000006664000015
:102F1000000003004FC5FE61CE62F93700000000DB
:102F20007564610075646130000003006BC5466222
:102F3000AB63E433000000007564610075646131C7
:102F4000000003006BC54662AB63E833000000007D
:102F50007564610075646132000003006BC54662F0
:102F6000AB63EC330000000075646100756461338D
:102F7000000003006BC54662AB63F0330000000045
:102F80007564620075646230000003006BC54662C0
:102F9000AB63F43300000000756462007564623155
:102FA000000003006BC54662AB63F833000000000D
:102FB0007564620075646232000003006BC546628E
:102FC000AB63FC330000000075646200756462331B
:102FD000000003006BC54662AB63003400000000D4
:102FE0007564630075646330000003006BC546625E
:102FF000AB630434000000007564630075646331E2
:10300000000003006BC54662AB630834000000009B
:103010007564630075646332000003006BC546622B
:10302000AB630C34000000007564630075646333A7
:10303000000003006BC54662AB6310340000000063
:103040007564640075646430000003006BC54662FB
:10305000AB6314340000000075646400756464316F
:10306000000003006BC54662AB631834000000002B
:103070007564640075646432000003006BC54662C9
:10308000AB631C3400000000756464007564643335
:10309000000003006BC54662AB63203400000000F3
:1030A0005F7465005F7465780000000288C56D621A
:1030B000A6620750000000005F7465005F746579C8
:1030C0000000000288C56D62A6620B50000000007F
:1030D0005F7465005F74657A0000000288C56D62E8
:1030E000A6620F50000000005F7465005F746561A8
:1030F0000000000288C56D62A66213500000000047
:103100005F7465005F7465620000000288C56D62CF
:10311000A6621750000000005F7465005F7465636D
:103120000000000288C56D62A6621B50000000000E
:103130005F7472005F7472780000000288C56D626F
:10314000A6622C51000000005F7472005F747279F7
:103150000000000288C56D62A662305100000000C8
:103160005F7472005F74727A0000000288C56D623D
:10317000A6623451000000005F7472005F747261D7
:103180000000000288C56D62A66238510000000090
:103190005F7472005F7472620000000288C56D6225
:1031A000A6623C51000000005F7472005F7472639D
:1031B0000000000288C56D62A66240510000000058
:1031C0005F7473005F7473310000000288C56D6224
:1031D000A6629750000000005F7073005F7073314B
:1031E0000000000288C56D62A662A75000000000C2
:1031F0005F6373005F6373310000000288C56D6216
:10320000A662B750000000005F6573005F65733110
:103210000000000288C56D62A662C7500000000071
:103220005F7873005F7873310000000288C56D62BB
:10323000A662E753000000005F6665005F666531C7
:103240000000000288C56D62A662D7500000000031
:103250005F7473005F7473320000000288C56D6292
:10326000A6629B50000000005F7073005F707332B5
:103270000000000288C56D62A662AB50000000002D
:103280005F6373005F6373320000000288C56D6284
:10329000A662BB50000000005F6573005F6573327B
:1032A0000000000288C56D62A662CB5000000000DD
:1032B0005F7873005F7873320000000288C56D622A
:1032C000A662FF53000000005F6665005F6665321E
:1032D0000000000288C56D62A662DB50000000009D
:1032E0005F7473005F7473330000000288C56D6201
:1032F000A6629F50000000005F7073005F70733320
:103300000000000288C56D62A662AF500000000098
:103310005F6373005F6373330000000288C56D62F2
:10332000A662BF50000000005F6573005F657333E5
:103330000000000288C56D62A662CF500000000048
:103340005F7873005F7873330000000288C56D6298
:10335000A6621754000000005F6665005F66653373
:103360000000000288C56D62A662DF500000000008
:103370005F7473005F7473340000000288C56D626F
:10338000A662A350000000005F7073005F7073348A
:103390000000000288C56D62A662B3500000000004
:1033A0005F6373005F6373340000000288C56D6261
:1033B000A662C350000000005F6573005F65733450
:1033C0000000000288C56D62A662D35000000000B4
:1033D0005F7873005F7873340000000288C56D6207
:1033E000A6622F54000000005F6665005F666534CA
:1033F0000000000288C56D62A662E3500000000074
:10340000000000005F64616D0000000036C5AA5E28
:10341000AA5E29340000000000000000736530300F
:103420000000020036C522628263AA52000000003A
:1034300000000000736530310000020036C52262D2
:103440008263AC520000000000000000736530325F
:103450000000020036C522628263AE520000000006
:1034600000000000736530330000020036C52262A0
:103470008263B05200000000000000007365303429
:103480000000020036C522628263B25200000000D2
:1034900000000000736530350000020036C522626E
:1034A0008263B452000000000000000073653036F3
:1034B0000000020036C522628263B652000000009E
:1034C00000000000736530370000020036C522623C
:1034D0008263B852000000000000000073653038BD
:1034E0000000020036C522628263BA52000000006A
:1034F00000000000736530390000020036C522620A
:103500008263BC520000000000000000736531308F
:103510000000020036C522628263BE520000000035
:1035200000000000736531310000020036C52262E0
:103530008263C05200000000000000007365313259
:103540000000020036C522628263C2520000000001
:1035500000000000736531330000020036C52262AE
:103560008263C45200000000000000007365313423
:103570000000020036C522628263C65200000000CD
:1035800000000000736531350000020036C522627C
:103590008263C852000000000000000073653136ED
:1035A0000000020036C522628263CA520000000099
:1035B00000000000736531370000020036C522624A
:1035C0008263CC52000000000000000073653138B7
:1035D0000000020036C522628263CE520000000065
:1035E00000000000736531390000020036C5226218
:1035F0008263D0520000000000000000736532308A
:103600000000020036C522628263D2520000000030
:1036100000000000736532310000020036C52262EE
:103620008263D45200000000000000007365323253
:103630000000020036C522628263D65200000000FC
:1036400000000000736532330000020036C52262BC
:103650008263D8520000000000000000736532341D
:103660000000020036C522628263DA5200000000C8
:1036700000000000736532350000020036C522628A
:103680008263DC52000000000000000073653236E7
:103690000000020036C522628263DE520000000094
:1036A00000000000736532370000020036C5226258
:1036B0008263E052000000000000000073653238B1
:1036C0000000020036C522628263E2520000000060
:1036D00000000000736532390000020036C5226226
:1036E0008263E45200000000000000007379730060
:1036F0000000000036C597650B6429340000000007
:1037000000000000703100000000000036C5976521
:103710000B642934000000000000000031000000AC
:103720000000000036C597650B64293400000000D6
:1037300000000000320000000000000036C5976560
:103740000B6429340000000000000000330000007A
:103750000000000036C597650B64293400000000A6
:1037600000000000340000000000000036C597652E
:103770000B64293400000000000000007800000005
:103780000000000036C597650B6429340000000076
:1037900000000000790000000000000036C59765B9
:1037A0000B64293400000000000000007A000000D3
:1037B0000000000036C597650B6429340000000046
:1037C00000000000610000000000000036C59765A1
:1037D0000B642934000000000000000062000000BB
:1037E0000000000036C597650B6429340000000016
:1037F00000000000630000000000000036C597656F
:103800000B6429340000000000000000673534001C
:103810000000000036C597650B64293400000000E5
:1038200000000000673535000000000036C59765D0
:103830000B642934000000000000000067353600EA
:103840000000000036C597650B64293400000000B5
:1038500000000000673537000000000036C597659E
:103860000B642934000000000000000067353800B8
:103870000000000036C597650B6429340000000085
:1038800000000000673539000000000036C597656C
:103890000B6429340000000000000000673932008A
:1038A0000000000036C597650B6429340000000055
:1038B00000000000673238000000000036C5976540
:1038C0000B64293400000000000000006733300062
:1038D0000000000036C597650B6429340000000025
:1038E000000000006D706F000000000036C5976595
:1038F0000B6429340000000000000000706F7300AA
:103900000000000036C597650B64293400000000F4
:10391000000000006F6673000000000036C5976568
:103920000B6429340000000000000000686F6D0087
:103930000000000036C597650B64293400000000C4
:1039400000000000707262000000000036C597653C
:103950000B64293400000000000000007077720042
:103960000000000036C597650B6429340000000094
:10397000000000006A6F67000000000036C5976510
:103980000B64293400000000000000006A69640034
:103990000000000036C597650B6429340000000064
:1039A00000000000756461000000000036C59765E6
:1039B0000B64293400000000000000007564620000
:1039C0000000000036C597650B6429340000000034
:1039D00000000000756463000000000036C59765B4
:1039E0000B642934000000000000000075646400CE
:1039F0000000000036C597650B6429340000000004
:103A0000000000005F7465000000000036C5976587
:103A10000B64293400000000000000005F74720095
:103A20000000000036C597650B64293400000000D3
:103A3000000000005F7473000000000036C5976549
:103A40000B64293400000000000000005F70730068
:103A50000000000036C597650B64293400000000A3
:103A6000000000005F6373000000000036C597652A
:103A70000B64293400000000000000005F65730043
:103A80000000000036C597650B6429340000000073
:103A9000000000005F7873000000000036C59765E5
:103AA0000B64293400000000000000005F66650020
:103AB0000000000036C597650B6429340000000043
:103AC000000000006D0000000000000036C58168A5
:103AD000A662293400000000000000007100000010
:103AE0000000000036C56768A662293400000000A7
:103AF000000000006F0000000000000036C54D68A7
:103B0000A66229340000000000000000240000002C
:103B10000000000036C59B68A66229340000000042
:103B2000456E64206F6620636F6D6D616E64206604
:103B3000696C650A00486F6D696E67206572726F07
:103B400072202D2025632061786973207365747459
:103B5000696E6773206D6973636F6E6669677572EE
:103B600065640050726F62696E67206572726F7271
:103B7000202D20256320617869732063616E6E6F4C
:103B800074206D6F766520647572696E672070723F
:103B90006F62696E67005B69645D202054696E79AD
:103BA00047204944253330730A005B68765D202046
:103BB00068617264776172652076657273696F6E91
:103BC0002531362E32660A005B68705D2020686100
:103BD00072647761726520706C6174666F726D25B6
:103BE00031352E32660A005B66765D20206669728A
:103BF0006D776172652076657273696F6E253136F7
:103C00002E32660A005B66625D20206669726D77FF
:103C1000617265206275696C642531382E32660ADE
:103C200000456E7465722024626F6F743D3120749C
:103C30006F20656E7465722074686520626F6F74A2
:103C4000206C6F616465722E0A000A0A0A2323231E
:103C50002054696E794720424F4F54204C4F4144C5
:103C600045522048656C70202323230A00456E745A
:103C700065722024646566613D3120746F20726531
:103C8000736574207468652073797374656D20742E
:103C90006F2074686520666163746F727920646553
:103CA0006661756C742076616C7565732E0A546854
:103CB00069732077696C6C206F76657277726974AE
:103CC0006520616E79206368616E67657320796F26
:103CD000752068617665206D6164652E0A000A0AA8
:103CE0000A2323232054696E794720524553544FA9
:103CF00052452044454641554C54532048656C700C
:103D0000202323230A00496E766F6B652073656C50
:103D100066207465737420627920656E74657269BB
:103D20006E672024746573743D4E207768657265F4
:103D3000204E206973206F6E65206F663A0A20203E
:103D400024746573743D312020736D6F6B6520742E
:103D50006573740A202024746573743D32202068D2
:103D60006F6D696E67207465737420202028796FE9
:103D700075206D757374207472697020686F6D6939
:103D80006E67207377697463686573290A2020243D
:103D9000746573743D33202073717561726520748E
:103DA0006573742020202861207365726965732013
:103DB0006F662073717561726573290A20202474FF
:103DC0006573743D342020617263207465737420C0
:103DD000202020202028736F6D65206C617267653C
:103DE00020636972636C6573290A202024746573EB
:103DF000743D3520206477656C6C20746573742085
:103E0000202020286D6F7665732073706163656470
:103E10002062792031207365636F6E64206477655A
:103E20006C6C73290A202024746573743D3620203D
:103E300066656564686F6C642074657374202865BA
:103E40006E746572202120616E64207E20746F2064
:103E5000686F6C6420616E64207265737461727443
:103E60002C20726573706563746976656C79290AB4
:103E7000202024746573743D3720204D20636F64C7
:103E8000657320746573742020284D20636F64650A
:103E90007320696E7465726D696E676C65642077F6
:103EA000697468206D6F766573290A202024746513
:103EB00073743D3820204A534F4E2074657374202C
:103EC00020202020286D6F74696F6E2074657374D4
:103ED0002072756E207573696E67204A534F4E20AD
:103EE000636F6D6D616E6473290A2020247465739D
:103EF000743D392020696E76657273652074696D32
:103F00006520746573740A202024746573743D31D0
:103F10003020726F74617279206D6F74696F6E20DA
:103F2000746573740A202024746573743D313120E4
:103F3000736D616C6C206D6F76657320746573743E
:103F40000A202024746573743D313220736C6F77BE
:103F5000206D6F76657320746573740A2020247455
:103F60006573743D313320636F6F7264696E617481
:103F7000652073797374656D206F66667365742050
:103F80007465737420284739322C204735342D4707
:103F90003539290A0A546573747320617373756D1A
:103FA0006520612063656E746572656420585920D0
:103FB0006F726967696E20616E64206174206C6540
:103FC0006173742038306D6D20636C656172616E51
:103FD000636520696E20616C6C206469726563742E
:103FE000696F6E730A546573747320617373756DB2
:103FF00065205A20686173206174206C6561737458
:104000002034306D6D20706F736969746976652036
:10401000636C656172616E63650A546573747320C5
:10402000737461727420776974682061204730204E
:104030005830205930205A30206D6F76650A486F0D
:104040006D696E67206973207468652065786365A3
:104050007074696F6E2E204E6F20696E697469618D
:104060006C20706F736974696F6E206F7220636C5F
:10407000656172616E636520697320617373756D2C
:1040800065640A000A0A0A2323232054696E7947CB
:104090002053454C4620544553542048656C7020AD
:1040A0002323230A0045616368202420636F6D6D1C
:1040B000616E642061626F766520616C736F20644D
:1040C0006973706C6179732074686520746F6B65B7
:1040D0006E20666F72206561636820736574746911
:1040E0006E6720696E205B205D20627261636B6584
:1040F00074730A546F2076696577207365747469E8
:104100006E677320656E746572206120746F6B65D5
:104110006E3A0A0A2020243C746F6B656E3E0A0AD0
:10412000466F72206578616D706C652024796672C7
:1041300020746F20646973706C61792074686520E5
:1041400059206D6178206665656420726174650A26
:104150000A546F20757064617465207365747469A6
:104160006E677320656E74657220746F6B656E2068
:10417000657175616C732076616C75653A0A0A2009
:1041800020243C746F6B656E3E3D3C76616C7565BA
:104190003E0A0A466F72206578616D706C65202456
:1041A0007966723D38303020746F207365742074E6
:1041B00068652059206D61782066656564207261AC
:1041C000746520746F20383030206D6D2F6D696EEE
:1041D0007574650A466F7220636F6E6669677572E3
:1041E0006174696F6E2064657461696C73207365B6
:1041F000653A2068747470733A2F2F676974687514
:10420000622E636F6D2F73796E746865746F732F90
:1042100054696E79472F77696B692F54696E7947B6
:104220002D436F6E66696775726174696F6E0A00FF
:10423000546865736520636F6D6D616E6473206192
:1042400072652061637469766520666F7220636FA2
:104250006E66696775726174696F6E3A0A20202410
:104260007379732053686F772073797374656D2049
:104270002867656E6572616C292073657474696E58
:1042800067730A2020243120202053686F77206D27
:104290006F746F7220312073657474696E67732058
:1042A000286F72207768617465766572206D6F740F
:1042B0006F7220796F752077616E7420312C322CEB
:1042C000332C34290A2020247820202053686F774B
:1042D000205820617869732073657474696E677300
:1042E00020286F7220776861746576657220617826
:1042F000697320796F752077616E7420782C792C22
:104300007A2C612C622C63290A2020246D20202025
:1043100053686F7720616C6C206D6F746F722073BF
:10432000657474696E67730A2020247120202053FD
:10433000686F7720616C6C20617869732073657495
:1043400074696E67730A2020246F20202053686FE1
:104350007720616C6C206F6666736574207365747A
:1043600074696E67730A2020242420202053686F0C
:104370007720616C6C2073657474696E67730A20B2
:1043800020246820202053686F7720746869732088
:1043900068656C702073637265656E0A0A000A0AAC
:1043A0000A2323232054696E794720434F4E464900
:1043B0004755524154494F4E2048656C7020232385
:1043C000230A000A466F722064657461696C656433
:1043D0002054696E794720696E666F207365653A6F
:1043E0002068747470733A2F2F6769746875622E31
:1043F000636F6D2F73796E746865746F732F546972
:104400006E79472F77696B692F0A466F722074683F
:1044100065206C6174657374206669726D77617272
:1044200065207365653A2068747470733A2F2F673E
:1044300069746875622E636F6D2F73796E74686529
:10444000746F732F54696E79470A506C6561736598
:10445000206C6F6720616E792069737375657320B6
:10446000617420687474703A2F2F7777772E737980
:104470006E746865746F732E636F6D2F666F7275DF
:104480006D730A486176652066756E0A000A4E6F84
:1044900074653A2054696E79472067656E6572616C
:1044A000746573206175746F6D61746963207374D2
:1044B00061747573207265706F72747320627920F5
:1044C00064656661756C740A546869732063616E13
:1044D0002062652064697361626C65642062792082
:1044E000656E746572696E67202473763D300A5379
:1044F0006565207468652077696B692062656C6FFB
:104500007720666F72206D6F7265206465746169D3
:104510006C732E0A00546865736520636F6D6D615E
:104520006E647320617265206163746976652066CC
:10453000726F6D2074686520636F6D6D616E6420AD
:104540006C696E653A0A205E7820202020202020A9
:1045500020202020202052657365742028636F6E10
:1045600074726F6C207829202D20736F66747761C8
:1045700072652072657365740A20203F2020202018
:104580002020202020202020204D616368696E6556
:1045900020706F736974696F6E20616E6420676349
:1045A0006F6465206D6F64656C2073746174650A57
:1045B00020202420202020202020202020202020F7
:1045C00053686F7720616E642073657420636F6E2B
:1045D00066696775726174696F6E2073657474695A
:1045E0006E67730A202021202020202020202020F8
:1045F0002020202046656564686F6C64202D207340
:10460000746F70206D6F74696F6E20776974686F56
:104610007574206C6F73696E6720706F736974694D
:104620006F6E0A20207E20202020202020202020A5
:104630002020204379636C65205374617274202DAF
:1046400020726573746172742066726F6D20666586
:104650006564686F6C640A20206820202020202078
:104660002020202020202053686F772074686973F1
:104670002068656C702073637265656E0A20202463
:104680006820202020202020202020202053686F18
:104690007720636F6E66696775726174696F6E20EB
:1046A00068656C702073637265656E0A20202474DF
:1046B0006573742020202020202020204C697374F2
:1046C0002073656C662D74657374730A20202474DE
:1046D0006573743D4E2020202020202052756E20CE
:1046E00073656C662D74657374204E0A20202468EF
:1046F0006F6D653D312020202020202052756E20D6
:104700006120686F6D696E67206379636C650A204C
:104710002024646566613D31202020202020205225
:104720006573746F726520616C6C20736574746955
:104730006E677320746F2022666163746F727922D2
:104740002064656661756C74730A000A0A0A232383
:10475000232054696E79472048656C7020232323F9
:104760000A005B6A735D20206A736F6E2073657246
:1047700069616C697A65207374796C652539642088
:104780005B303D72656C617865642C313D73747289
:104790006963745D0A005B6A765D20206A736F6EE0
:1047A00020766572626F7369747925313564205B98
:1047B000303D73696C656E742C313D666F6F746546
:1047C000722C323D6D657373616765732C333D6385
:1047D0006F6E666967732C343D6C696E656E756DBE
:1047E0002C353D766572626F73655D0A005B656AA4
:1047F0005D2020656E61626C65206A736F6E206D4E
:104800006F646525313364205B303D746578742CAA
:10481000313D4A534F4E5D0A00FA58F458ED58E8BE
:1048200058DF58D458C958BD58B158A3588C587D32
:104830005870586458505843582E581A58175814DE
:10484000580558F057DB57CC57BC57AA57935776A3
:1048500057595740572A5719570757FA56E856CE0F
:1048600056CB56C856C556C256BF56BC56B956B694
:1048700056B356B056AD56AA56A756A456A1569E44
:10488000569B569856955692568F568C56895686F4
:1048900056835680567D567A567756745671566EA4
:1048A000566B566856655662565F565C5659565654
:1048B00056535650564D564A564756445641563E04
:1048C000563B563856355632562F562C560856E813
:1048D00055CE55B4559A557655595541552B5511C8
:1048E00055ED54DB54C954B0549A5484546C545408
:1048F00054425424540F54F153CC53C853C453C09E
:1049000053BC53B853B453B053AC53A853A453A09F
:10491000539C539853945390538C5388536E5354D1
:1049200053415325531353FC52DB52CA52AA528AA5
:1049300052705256523F520C52DF51BF519D517727
:1049400051505134511551FB50E150BC5093507BA4
:104950005050502450EE4FB94FA74F954F864F738C
:104960004F5A4F384F264F144F024FF04EDE4ECC69
:104970004EBA4EA84E964E844E724E604E4E4E3CEF
:104980004E384E344E304E2C4E284E244E204E1C67
:104990004E184E144E104E0C4E084E044E004EFC57
:1049A0004DF84DF44DF04DEC4DD84DBA4D9E4D7334
:1049B0004D4E4D294D254D214D1D4D194D154D1176
:1049C0004D0D4D094D054D014DFD4CF94CF54CF18A
:1049D0004CDD4CC14CA54C894C6D4C514C354C199F
:1049E0004CFD4BE14BC54BA94B8D4B894B854B8106
:1049F0004B7D4B794B754B714B5D4B354B0E4BE8FB
:104A00004ABB4A954A684A644A604A5C4A494A280D
:104A10004A134A4A6F6767696E67206379636C65FA
:104A2000206661696C65640050726F626520656E16
:104A300064706F696E742069732073746172746935
:104A40006E6720706F696E740050726F62652063CC
:104A500079636C65206661696C6564003234390085
:104A60003234380032343700486F6D696E67204544
:104A700072726F72202D20486F6D696E6720737798
:104A8000697463686573206D6973636F6E666967C7
:104A90007572656400486F6D696E67204572726F4C
:104AA00072202D204E65676174697665206C617493
:104AB0006368206261636B6F666600486F6D696E44
:104AC00067204572726F72202D2054726176656C7A
:104AD000206D696E2026206D6178206172652074DA
:104AE00068652073616D6500486F6D696E6720456C
:104AF00072726F72202D204C617463682076656C31
:104B00006F63697479206973207A65726F00486FEA
:104B10006D696E67204572726F72202D205365613A
:104B20007263682076656C6F63697479206973209D
:104B30007A65726F00486F6D696E67204572726F9B
:104B400072202D20426164206F72206E6F20617888
:104B500069732073706563696669656400486F6D89
:104B6000696E67206379636C65206661696C656452
:104B700000323339003233380032333700323336C3
:104B800000323335003233340032333300536F6632
:104B900074206C696D69742065786365656465640B
:104BA000202D2043206D617800536F6674206C695E
:104BB0006D6974206578636565646564202D2043A4
:104BC000206D696E00536F6674206C696D69742086
:104BD0006578636565646564202D2042206D617889
:104BE00000536F6674206C696D6974206578636525
:104BF00065646564202D2042206D696E00536F66E8
:104C000074206C696D69742065786365656465649A
:104C1000202D2041206D617800536F6674206C69EF
:104C20006D6974206578636565646564202D204135
:104C3000206D696E00536F6674206C696D69742015
:104C40006578636565646564202D205A206D617800
:104C500000536F6674206C696D69742065786365B4
:104C600065646564202D205A206D696E00536F665F
:104C700074206C696D69742065786365656465642A
:104C8000202D2059206D617800536F6674206C6967
:104C90006D6974206578636565646564202D2059AD
:104CA000206D696E00536F6674206C696D697420A5
:104CB0006578636565646564202D2058206D617892
:104CC00000536F6674206C696D6974206578636544
:104CD00065646564202D2058206D696E00536F66F1
:104CE00074206C696D6974206578636565646564BA
:104CF000003231390032313800323137003231364A
:104D00000032313500323134003231330032313249
:104D10000032313100323130003230390032303837
:104D200000323037003230360054726170657A6F6D
:104D3000696420706C616E6E6572206661696C6575
:104D40006420746F20636F6E7665726765004C69CE
:104D50006D69742073776974636820686974202DA5
:104D60002053687574646F776E206F636375727219
:104D70006564004D616368696E6520697320616CCC
:104D800061726D6564202D20436F6D6D616E6420CE
:104D90006E6F742070726F636573736564004D6F1E
:104DA0007665206C657373207468616E206D696E22
:104DB000696D756D2074696D65004D6F7665206C49
:104DC000657373207468616E206D696E696D756DB1
:104DD000206C656E6774680047656E657269632054
:104DE00054696E7947206572726F720031393900EB
:104DF0003139380031393700313936003139350031
:104E00003139340031393300313932003139310030
:104E10003139300031383900313838003138370015
:104E2000313836003138350031383400313833000C
:104E30003138320031383100313830005420776F4A
:104E4000726420697320696E76616C696400542015
:104E5000776F7264206973206D697373696E670080
:104E60005220776F726420697320696E76616C6975
:104E700064005220776F7264206973206D697373C8
:104E8000696E67005120776F726420697320696EC4
:104E900076616C6964005120776F726420697320B9
:104EA0006D697373696E67004C20776F7264206957
:104EB0007320696E76616C6964004C20776F726450
:104EC000206973206D697373696E67004820776F7E
:104ED000726420697320696E76616C696400482091
:104EE000776F7264206973206D697373696E6700F0
:104EF0004520776F726420697320696E76616C69F2
:104F000064004520776F7264206973206D69737344
:104F1000696E67004420776F726420697320696E40
:104F200076616C6964004420776F72642069732035
:104F30006D697373696E67005020776F72642069C2
:104F400073206E6F7420612076616C696420746FC9
:104F50006F6C206E756D626572005020776F7264A1
:104F6000206973206E6F7420616E20696E746567AE
:104F70006572005020776F7264206973206E6567D8
:104F80006174697665005020776F726420697320C0
:104F90007A65726F005020776F72642069732069A0
:104FA0006E76616C6964005020776F72642069735B
:104FB000206D697373696E67004172632073706559
:104FC00063696669636174696F6E206572726F727E
:104FD000202D20656E64706F696E74206973207374
:104FE00074617274696E6720706F696E74004172CB
:104FF000632073706563696669636174696F6E20AD
:105000006572726F72202D20726164697573206100
:105010007263206F7574206F6620746F6C657261A7
:105020006E636500417263207370656369666963CE
:105030006174696F6E206572726F72202D206D69C8
:105040007373696E67206F666673657428732900D1
:105050004172632073706563696669636174696F27
:105060006E206572726F72202D206D697373696E88
:105070006720617869732865732900417263207322
:10508000706563696669636174696F6E20657272C9
:105090006F72005370696E646C65206D7573742057
:1050A0006265207475726E696E6720666F72207417
:1050B00068697320636F6D6D616E64005370696E13
:1050C000646C65206D757374206265206F66662060
:1050D000666F72207468697320636F6D6D616E64B2
:1050E000005370696E646C65205320776F72642082
:1050F000697320696E76616C6964005370696E64CF
:105100006C65205320776F7264206973206D69731A
:1051100073696E67005370696E646C6520737065A7
:105120006564206578636565646564206D61786990
:105130006D756D005370696E646C65207370656584
:10514000642062656C6F77206D696E696D756D00A6
:1051500050726F6772616D6D656420706F696E74F7
:105160002073616D652061732063757272656E7462
:1051700020706F696E740043757474657220636F7C
:105180006D70656E736174696F6E2063616E6E6FB2
:105190007420626520656E61626C656400526571A1
:1051A0007565737465642076656C6F6369747920C6
:1051B00065786365656473206C696D697473004715
:1051C00030206F72204731206D7573742062652026
:1051D00061637469766520666F72204735330052CB
:1051E0006F7461727920617865732063616E6E6F90
:1051F0007420626520757365642077697468207413
:1052000068697320636F6D6D616E6400496E7665C9
:105210007273652074696D65206D6F6465206361CC
:105220006E6E6F7420626520757365642077697493
:1052300068207468697320636F6D6D616E640046E9
:1052400065656472617465206E6F74207370656348
:1052500069666965640053656C6563746564207094
:105260006C616E6520697320696E76616C6964009B
:1052700053656C656374656420706C616E6520694C
:1052800073206D697373696E670041786973207468
:10529000617267657420706F736974696F6E2069DD
:1052A0007320696E76616C6964004178697320745B
:1052B000617267657420706F736974696F6E2069BD
:1052C00073206D697373696E670041786973206933
:1052D000732064697361626C65640041786973204E
:1052E000697320696E76616C696420666F722074E0
:1052F00068697320636F6D6D616E640041786973D6
:105300002063616E6E6F74206265207072657365D4
:105310006E74004178697320776F7264206D6973D1
:1053200073696E670047636F6465206D6F64616CBD
:105330002067726F75702076696F6C6174696F6E2B
:10534000004D20636F646520756E737570706F72A9
:105350007465640047636F646520636F6D6D616E93
:105360006420756E737570706F7274656400476544
:105370006E657269632047636F646520696E70753E
:1053800074206572726F7200313239003132380028
:1053900031323700313236003132350031323400AB
:1053A00031323300313232003132310031323000AB
:1053B0003131390031313800313137003131360087
:1053C000313135003131340031313300436F6D6D8F
:1053D000616E642063616E6E6F742062652074611B
:1053E0006B656E20617420746869732074696D65E3
:1053F00000436F6E666967206E6F742074616B6521
:105400006E20647572696E67206379636C65004A0B
:10541000534F4E206F757470757420746F6F206CCD
:105420006F6E67004A534F4E20696E707574206826
:10543000617320746F6F206D616E79207061697285
:1054400073004A534F4E2073796E746178206572F1
:10545000726F7200496E7075742076616C7565208C
:10546000756E737570706F7274656400496E7075D7
:10547000742076616C75652072616E676520657257
:10548000726F7200496E7075742076616C7565205C
:10549000746F6F206C6172676500496E707574205F
:1054A00076616C756520746F6F20736D616C6C0034
:1054B000496E7075742065786365656473206D61ED
:1054C00078206C656E67746800426164206E756D4B
:1054D00062657220666F726D6174004D616C666FFB
:1054E000726D656420636F6D6D616E6400556E72E0
:1054F00065636F676E697A656420636F6D6D616E59
:1055000064206F7220636F6E666967206E616D65DF
:105510000047656E657269632061737365727469B3
:105520006F6E206661696C757265004D656D6F7296
:1055300079206661756C7420646574656374656454
:1055400000537461636B206F766572666C6F7720B1
:10555000646574656374656400436F6E74726F6C28
:105560006C657220617373657274696F6E20666119
:10557000696C7572650043616E6F6E6963616C2062
:105580006D616368696E6520617373657274696FBC
:105590006E206661696C75726500506C616E6E6537
:1055A0007220617373657274696F6E206661696CD5
:1055B00075726500537465707065722061737365F0
:1055C0007274696F6E206661696C75726500456EF4
:1055D000636F64657220617373657274696F6E20A6
:1055E0006661696C75726500494F207375622D7331
:1055F000797374656D20617373657274696F6E2061
:105600006661696C75726500436F6E6669672073C9
:1056100075622D73797374656D206173736572742F
:10562000696F6E206661696C757265003839003883
:105630003800383700383600383500383400383311
:105640000038320038310038300037390037380040
:1056500037370037360037350037340037330037F7
:1056600032003731003730003639003638003637EF
:105670000036360036350036340036330036320018
:1056800036310036300035390035380035370035D1
:1056900036003535003534003533003532003531CC
:1056A00000353000343900343800343700343600E7
:1056B00034350034340034330034320034310034B3
:1056C000300033390033380033370033360042615D
:1056D0006420737461747573207265706F727420C6
:1056E00073657474696E670050657273697374656D
:1056F0006E6365206572726F7200466C6F61742014
:105700006973204E414E00466C6F617420697320AE
:10571000696E66696E697465004D6F76652074699F
:105720006D65206973204E414E004D6F7665207483
:10573000696D6520697320696E66696E69746500BC
:1057400047656E6572696320657863657074696F1B
:105750006E207265706F7274004661696C656420BA
:10576000746F2067657420706C616E6E6572206264
:1057700075666665720053797374656D20616C613E
:10578000726D202D207368757474696E6720646F64
:10579000776E00496E697469616C697A6174696FCA
:1057A0006E206661696C75726500526561642D6F6B
:1057B0006E6C79206164647265737300496E766102
:1057C0006C6964204164647265737300446976692E
:1057D0006465206279207A65726F00466C6F61742F
:1057E000696E6720706F696E74206572726F7200E7
:1057F000496E7465726E616C2072616E67652065BA
:1058000072726F7200496E7465726E616C2065729F
:10581000726F720031390031380046756E637469F9
:105820006F6E206973207374756262656400456EE3
:10583000746572696E6720626F6F74206C6F61644B
:10584000657200496E697469616C697A696E670096
:105850004275666665722066756C6C202D206661E7
:1058600074616C004275666665722066756C6C00CA
:1058700042756666657220656D707479004E6F20A2
:105880007375636820646576696365004D6178208F
:1058900066696C652073697A6520657863656564FF
:1058A00065640046696C65206E6F74206F70656E6C
:1058B00000456E64206F662066696C6500456E6405
:1058C000206F66206C696E650048617264207265A5
:1058D000736574005465726D696E6174656400432C
:1058E0006F6D706C657465004E6F6F700045616719
:1058F00061696E004572726F72004F4B005B7031D0
:10590000706F665D2070776D207068617365206FC1
:1059100066662020202531352E3366205B302E2E02
:10592000315D0A005B70317770685D2070776D20A3
:105930006363772070686173652068692531352E4F
:105940003366205B302E2E315D0A005B703177703C
:105950006C5D2070776D206363772070686173657C
:10596000206C6F2531352E3366205B302E2E315D55
:105970000A005B70317773685D2070776D20636318
:10598000772073706565642068692531352E30662F
:105990002052504D0A005B703177736C5D20707738
:1059A0006D20636377207370656564206C6F2531AB
:1059B000352E30662052504D0A005B70316370689E
:1059C0005D2070776D206377207068617365206853
:1059D00069202531352E3366205B302E2E315D0A4D
:1059E000005B703163706C5D2070776D2063772091
:1059F0007068617365206C6F202531352E33662009
:105A00005B302E2E315D0A005B70316373685D2060
:105A100070776D20637720737065656420686920F6
:105A20002531352E30662052504D0A005B703163AF
:105A3000736C5D2070776D2063772073706565648B
:105A4000206C6F202531352E30662052504D0A00D3
:105A50005B70316672715D2070776D206672657162
:105A600075656E63792020202531352E30662048FB
:105A70007A0A0053595354454D2052454144590028
:105A80004C6F6164696E6720636F6E66696773202F
:105A900066726F6D20454550524F4D00496E6974D6
:105AA00069616C697A696E6720636F6E6669677396
:105AB00020746F2053686170656F6B6F32203530D2
:105AC000306D6D2070726F66696C65007B22657247
:105AD000223A7B226662223A25302E32662C2273CD
:105AE00074223A25642C226D7367223A2225732290
:105AF0007D7D0A007B65723A7B66623A25302E32E4
:105B0000662C73743A25642C6D73673A22257322D0
:105B10007D7D0A005B71765D20207175657565205D
:105B20007265706F727420766572626F73697479D2
:105B3000253764205B303D6F66662C313D73696E9E
:105B4000676C652C323D747269706C655D0A00711A
:105B50006F3A25640A0071693A25640A0071723A45
:105B600025640A005B73765D20207374617475731D
:105B7000207265706F727420766572626F736974DB
:105B800079253664205B303D6F66662C313D666951
:105B90006C74657265642C323D766572626F7365F4
:105BA0005D0A005B73695D202073746174757320F6
:105BB000696E74657276616C2531342E3066206DA5
:105BC000730A005B257325735D206D257320706F4C
:105BD000776572206D616E6167656D656E742531E4
:105BE0003064205B303D64697361626C65642C31A4
:105BF0003D616C77617973206F6E2C323D696E2048
:105C00006379636C652C333D7768656E206D6F76C4
:105C1000696E675D0A005B257325735D206D2573D2
:105C200020706F6C617269747925313864205B3043
:105C30003D6E6F726D616C2C313D7265766572736D
:105C4000655D0A005B257325735D206D2573206DEE
:105C50006963726F737465707325313664205B31CC
:105C60002C322C342C385D0A005B257325735D20A3
:105C70006D25732074726176656C20706572207278
:105C800065766F6C7574696F6E2531302E346625BC
:105C9000730A005B257325735D206D257320737473
:105CA000657020616E676C652532302E3366257312
:105CB0000A005B257325735D206D2573206D61706F
:105CC00020746F206178697325313564205B303D25
:105CD000582C313D592C323D5A2E2E2E5D0A005B38
:105CE0006D745D20206D6F746F722069646C652027
:105CF00074696D656F75742531342E326620536575
:105D0000630A00125D0E5D095D2064656700206D09
:105D10006D0020696E005B73745D20207377697479
:105D20006368207479706525313864205B303D4E9E
:105D30004F2C313D4E435D0A00546573742023257A
:105D400064206E6F7420666F756E640A004E362094
:105D500047393220583735205930205A300A4E37CB
:105D600020463530302E300A4E3820473159302EFB
:105D70003239315A2D322E3139380A4E39205837BE
:105D8000342E37363759302E3035385A2D322E339F
:105D900035350A4E3130205837342E373039592DA9
:105DA000302E3030305A2D322E3337310A4E3131C9
:105DB000205837342E3532395A2D322E3236340AA5
:105DC0004E3132205837342E36333459302E31305C
:105DD000355A2D322E3331390A4E3133205837346B
:105DE0002E38343359302E3331345A2D322E313847
:105DF000330A4E3134205837352E30303059302E5A
:105E00003437315A2D322E3132360A4E313520593F
:105E1000302E3635305A2D322E3130300A4E313652
:105E2000205837342E37383359302E3433345A2DE6
:105E3000322E3133310A4E3137205837342E353631
:105E40003659302E3231375A2D322E3234340A4EF2
:105E50003138205837342E333530592D302E3030EC
:105E6000305A2D322E3138320A4E313920583734DB
:105E70002E3137305A2D322E3134340A4E32302002
:105E80005837342E34323959302E3235395A2D3272
:105E90002E3136350A4E3231205837342E353333D1
:105EA00059302E3336335A2D322E3139310A4E3293
:105EB00032205837342E36383959302E3531395A48
:105EC0002D322E3131340A4E3233205837342E38A9
:105ED000343459302E3637345A2D322E3039360A72
:105EE0004E3234205837352E30303059302E38333A
:105EF000305A2D322E3131340A4E32352059312E5E
:105F00003031305A2D322E3134340A4E3236205848
:105F100037342E37383759302E3739375A2D322EFD
:105F20003039380A4E3237205837342E3632385905
:105F3000302E3633385A2D322E3130380A4E323820
:105F4000205837342E34363959302E3437385A2DBC
:105F5000322E3135370A4E3239205837342E33300D
:105F60003959302E3331395A2D322E3131300A4ED3
:105F70003330205837342E30343459302E303533C6
:105F80005A2D322E3130380A4E3331205837332EC5
:105F900039393059302E3030305A2D322E30373793
:105FA0000A4E3332205837332E3831315A2D312EA4
:105FB0003934370A4E3333205837332E3937335973
:105FC000302E3136325A2D322E3037390A4E333494
:105FD000205837342E32343359302E3433325A2D40
:105FE000322E3038340A4E3335205837342E34357B
:105FF0003959302E3634395A2D322E3135370A4E32
:106000003336205837342E36373659302E38363519
:106010005A2D322E3130390A4E3337205837342E2C
:1060200038333859312E3032375A2D322E31313102
:106030000A4E3338205837352E30303059312E3112
:1060400038395A2D322E3136300A4E3339205931F3
:106050002E3336395A2D322E3139340A4E3430200F
:106060005837342E38343259312E3231315A2D329C
:106070002E3133340A4E3431205837342E363834EA
:1060800059312E3035335A2D322E3132300A4E34BA
:1060900032205837342E34323159302E3739305A75
:1060A0002D322E3137360A4E3433205837342E33C2
:1060B000313659302E3638345A2D322E3133370A94
:1060C0004E3434205837342E31353859302E35324D
:1060D000365A2D322E3037370A4E34352058373362
:1060E0002E39343759302E3331365A2D322E303640
:1060F000370A4E3436205837332E38393459302E3B
:106100003236335A2D322E3034360A4E3437205838
:1061100037332E37333759302E3130355A2D312E13
:106120003931380A4E3438205837332E3633315906
:10613000302E3030305A2D312E3837320A4E343925
:10614000205837332E3435325A2D312E3831350A16
:106150004E3530205837332E36363559302E3231C1
:10616000345A2D312E3931340A4E353120583733D7
:106170002E38323559302E3337345A2D322E3032B4
:10618000380A4E3532205837332E38373959302EA9
:106190003432375A2D322E3037360A4E35332058A6
:1061A00037342E30393259302E3634315A2D322E82
:1061B0003039340A4E3534205837342E333036597E
:1061C000302E3835345A2D322E3139320A4E35358B
:1061D000205837342E35313959312E3036385A2D32
:1061E000322E3134310A4E3536205837342E37337B
:1061F0003359312E3238315A2D322E3134330A4E42
:106200003537205837342E38343059312E3338381A
:106210005A2D322E3137340A4E3538205837342E25
:1062200038393359312E3434325A2D322E313639F1
:106230000A4E3539205837352E30303059312E3509
:1062400034385A2D322E3132310A4E3630205931FF
:106250002E3732385A2D322E3037360A4E3631200C
:106260005837342E38343359312E3537315A2D3290
:106270002E3133300A4E3632205837342E373338E9
:1062800059312E3436365A2D322E3139350A4E36A2
:1062900033205837342E34373659312E3230345A71
:1062A0002D322E3134370A4E3634205837342E32C0
:1062B000313559302E3934335A2D322E3230320A9C
:1062C0004E3635205837332E39303059302E36324D
:1062D000385A2D322E3130310A4E36362058373367
:1062E0002E38343859302E3537365A2D322E303933
:1062F000360A4E3637205837332E35383659302E39
:106300003331345A2D312E3931330A4E3638205834
:1063100037332E33373759302E3130355A2D312E11
:106320003830380A4E3639205837332E3237325902
:10633000302E3030305A2D312E3738370A4E373024
:10634000205837332E3138325A2D312E3738370A0C
:106350004E3731205837332E3039325A2D312E37BF
:1063600035300A4E3732205837332E3431305930D9
:106370002E3331385A2D312E3836380A4E373320E5
:106380005837332E37383159302E3638395A2D3266
:106390002E3038360A4E3734205837342E303939BB
:1063A00059312E3030375A2D322E3232340A4E3790
:1063B00035205837342E32303559312E3131335A59
:1063C0002D322E3231310A4E3736205837342E33A3
:1063D000363459312E3237325A2D322E3137360A71
:1063E0004E3737205837342E36323959312E35331F
:1063F000375A2D322E3139310A4E3738205837343A
:106400002E36383259312E3539305A2D322E313719
:10641000370A4E3739205837342E38393459312E0F
:106420003830325A2D322E3036360A4E3830205817
:1064300037352E30303059312E3930385A2D322EF2
:106440003034360A4E38312059322E3038375A2DF2
:10645000322E3035310A4E3832205837342E383308
:106460003959312E3932375A2D322E3036320A4EC2
:106470003833205837342E36373959312E3736369F
:106480005A2D322E3133360A4E3834205837342EB6
:1064900036323559312E3731335A2D322E3137308D
:1064A0000A4E3835205837342E35373259312E368A
:1064B00035395A2D322E3138300A4E383620583779
:1064C000342E33353859312E3434355A2D322E315D
:1064D00035370A4E3837205837342E31393759314D
:1064E0002E3238345A2D322E3139350A4E38382072
:1064F0005837342E30393059312E3137375A2D3202
:106500002E3234350A4E3839205837332E39383345
:1065100059312E3037305A2D322E3232350A4E391B
:1065200030205837332E38323359302E3931305AE3
:106530002D322E3133380A4E3931205837332E332D
:10654000393459302E3438325A2D312E3931370AF8
:106550004E3932205837332E31383059302E3236BA
:10656000385A2D312E3832350A4E393320583732C9
:106570002E39363659302E3035345A2D312E3731AA
:10658000310A4E3934205837322E393133592D30B3
:106590002E3030305A2D312E3639330A4E393520CF
:1065A0005837322E3733335A2D312E3634360A4E81
:1065B0003936205837322E39393759302E32363461
:1065C0005A2D312E3735330A4E3937205837332E6E
:1065D00032363059302E3532375A2D312E3930324D
:1065E0000A4E3938205837332E36323959302E3842
:1065F00039365A2D322E3037370A4E39392058372E
:10660000332E38343059312E3130375A2D322E3224
:1066100032340A4E313030205837332E383933591E
:10662000312E3136305A2D322E3234350A4E313039
:10663000312058373559305A300A004E3120543104
:106640004D360A4E32204731370A4E332047323119
:106650000A4E382046313830300A4E392047310A48
:106660004E3130302047393220582D32352E3137D7
:1066700037592D33342E303732205A2D312E3030C9
:1066800030202854454D502C2052454D4F56452022
:106690004C41544552290A4E33343320582D32355B
:1066A0002E353935592D33342E3334390A4E33349F
:1066B0003420582D32352E373031592D33342E3485
:1066C00033360A4E33343520582D32352E37393192
:1066D000592D33342E3532300A4E33343620582D6E
:1066E00032352E383634592D33342E3630310A4E69
:1066F00033343720582D32352E393230592D33343A
:106700002E3637390A4E33343820582D32352E394B
:106710003630592D33342E3735340A4E3334392040
:10672000582D32352E393832592D33342E383236F1
:106730000A4E33353020582D32352E393837592D01
:1067400033342E3839350A4E33353120582D323511
:106750002E393736592D33342E3936310A4E3335EA
:106760003220582D32352E393438592D33352E30CC
:1067700032330A4E33353320582D32352E393033EB
:10678000592D33352E3038320A4E33353420582DBA
:1067900032352E383431592D33352E3133380A4EB7
:1067A00033353520582D32352E373633592D333584
:1067B0002E3139300A4E33353620582D32352E36AB
:1067C0003639592D33352E3233390A4E3335372089
:1067D000582D32352E353539592D33352E32383442
:1067E0000A4E33353820582D32352E343333592D57
:1067F00033352E3332350A4E33353920582D323564
:106800002E323931592D33352E3336330A4E333645
:106810003020582D32352E313334592D33352E3327
:1068200039370A4E33363120582D32342E3936332B
:10683000592D33352E3432380A4E33363220582D06
:1068400032342E373737592D33352E3435350A4EFD
:1068500033363320582D32342E353737592D3335D2
:106860002E3437370A4E33363420582D32342E33F7
:106870003637592D33352E3439360A4E33363520D6
:10688000582D32342E313434592D33352E353131A3
:106890000A4E33363620582D32332E393039592DA1
:1068A00033352E3532320A4E33363720582D3233B7
:1068B0002E363631592D33352E3532390A4E333690
:1068C0003820582D32332E343033592D33352E3570
:1068D00033320A4E33363920582D32332E3133338A
:1068E000592D33352E3533320A4E33373020582D5B
:1068F00032322E383533592D33352E3532370A2F73
:106900004E3235313820473058302E333237592DFA
:1069100033332E3532315A2D312E3030300A4E324B
:10692000353139204D3330004E31204732300A4E58
:106930003520473430204731370A4E31302054312A
:10694000204D30360A284E31352047393020473027
:10695000205830205930205A30290A4E32302053E6
:1069600035303030204D3033200A4E32352058300B
:106970002E3036342059302E333236205A300A4EDB
:10698000343020473031204631362E300A4E3530F3
:106990002058302E3036342059302E3332360A4EBD
:1069A00035352058302E3036302059302E3239339C
:1069B0000A4E36302058302E3037372059302E329C
:1069C00036370A4E36352058302E31313120593085
:1069D0002E3235370A4E37302058302E3134392098
:1069E00059302E3235320A4E37352058302E313854
:1069F000382059302E3235350A4E38302058302E56
:106A00003232372059302E3236380A4E3835205837
:106A1000302E3235372059302E3237310A4E393048
:106A20002058302E3333352059302E3236350A4E29
:106A300039352058302E3431322059302E3237310A
:106A40000A4E3130302058302E3437342059302E11
:106A50003238370A4E3130352058302E3439312013
:106A600059302E3238390A4E3131302058302E35D7
:106A700031372059302E3237330A4E3131352058D4
:106A8000302E3534342059302E3236330A4E3132DE
:106A9000302058302E3538302059302E3236310AD9
:106AA0004E3132352058302E3539352059302E327E
:106AB00036330A4E3133302058302E363231205999
:106AC000302E3237340A4E3133352058302E363599
:106AD000392059302E3330360A4E31343020583078
:106AE0002E3637332059302E3333350A4E31343574
:106AF0002058302E3637392059302E3336310A4E51
:106B00003135302058302E3637382059302E333832
:106B1000390A4E3135352058302E3637302059302D
:106B20002E3432300A4E3136302058302E3637303F
:106B30002059302E3434360A4E3136352058302E16
:106B40003638302059302E3437340A4E3137302021
:106B500058302E3730342059302E3439370A4E31E0
:106B600037352058302E3733322059302E353135D5
:106B70000A4E3138302058302E3739342059302ED3
:106B80003533350A4E3138352058302E38373220DB
:106B900059302E3536370A4E3139302058302E399B
:106BA00035302059302E3630340A4E3139352058A0
:106BB000312E3033312059302E3634370A4E3230B0
:106BC000302058312E3134392059302E3732320AA4
:106BD0004E3230352058312E3330382059302E384F
:106BE00035340A4E3231302058312E34333020596A
:106BF000302E3938340A4E3231352058312E343463
:106C0000372059302E3938360A4E3232302058313A
:106C10002E3632382059302E3832320A4E32323542
:106C20002058312E3733322059302E3731340A4E26
:106C30003233302058322E3030392059302E33380C
:106C4000310A4E3233352058322E31313620593008
:106C50002E3236360A4E3234302058322E32323806
:106C60002059302E3135370A4E3234352058322EE5
:106C70003238302059302E3132330A4E32353020FE
:106C800058322E3333322059302E3039340A4E32B6
:106C900035352058322E3432332059302E303730AB
:106CA0000A4E3236302058322E3438392059302EA0
:106CB0003036350A4E3236352058322E35353720AB
:106CC00059302E3036360A4E3237302058322E3672
:106CD00032372059302E3038340A4E32373520586A
:106CE000322E3639332059302E3130390A4E32386F
:106CF000302058322E3733302059302E3133330A7A
:106D00004E3238352058322E3830352059302E3119
:106D100039300A4E3239302058322E383239205923
:106D2000302E3231360A4E3239352058322E38382C
:106D3000302059302E3239310A4E3330302058321B
:106D40002E3838342059302E3330300A4E33303517
:106D50002058322E3839382059302E3333320A4EEB
:106D60003331302058322E3930352059302E3336D9
:106D7000370A4E3331352058322E393130205930D0
:106D80002E3430370A4E3332302058322E393038D4
:106D90002059302E3434360A4E3332352058322EB4
:106DA0003930312059302E3439350A4E33333020C2
:106DB00058322E3839372059302E3439350A4E336F
:106DC00033352058322E3839302059302E35323470
:106DD0000A4E3334302058322E3834322059302E77
:106DE0003630340A4E3334352058322E3831342080
:106DF00059302E3636350A4E3335302058322E373C
:106E000039342059302E3735300A4E333535205835
:106E1000322E3739312059302E3833380A4E333636
:106E2000302058322E3831392059302E3937360A31
:106E30004E3336352058322E3833372059312E30E4
:106E400034340A4E3337302058322E3836322059F7
:106E5000312E3131320A4E3337352058322E383701
:106E6000372059312E3134350A4E333830205832DC
:106E70002E3931322059312E3231370A4E333835DE
:106E80002058322E3931372059312E3232360A4EBF
:106E90003339302058322E3935312059312E32389D
:106EA000310A4E3339352058322E39373020593196
:106EB0002E3239350A4E3430302058322E39393698
:106EC0002059312E3239350A4E3430352058332E80
:106ED0003031332059312E3237350A4E343130209B
:106EE00058332E3032342059312E3235340A4E3454
:106EF00031352058332E3037302059312E3135314D
:106F00000A4E3432302058332E3037372059312E44
:106F10003133340A4E3432352058332E3132352055
:106F200059312E3033390A4E3433302058332E3114
:106F300033382059312E3031390A4E343335205808
:106F4000332E3230352059302E3930380A4E343411
:106F5000302058332E3238322059302E3739370A04
:106F60004E3434352058332E3336312059302E36B6
:106F700039310A4E3435302058332E3432362059C8
:106F8000302E3539320A4E3435352058332E3435CB
:106F9000362059302E3534330A4E343630205833AB
:106FA0002E3437392059302E3439330A4E343635A1
:106FB0002058332E3439342059302E3437320A4E8B
:106FC0003437302058332E3530352059302E343474
:106FD000360A4E3437352058332E35313820593063
:106FE0002E3431370A4E3438302058332E35333072
:106FF0002059302E3339310A4E3438352058332E4B
:107000003536342059302E3330300A4E3439302062
:1070100058332E3537372059302E3235330A4E3417
:1070200039352058332E3536382059302E3231320A
:107030000A4E3530302058332E3534342059302E16
:107040003137360A4E3530352058332E353431201D
:1070500059302E3134360A4E3531302058332E35E2
:1070600035332059302E3131390A4E3531352058DB
:10707000332E3537362059302E3130360A4E3532E0
:10708000302058332E3539372059302E3130320ADE
:107090004E3532352058332E3631382059302E3186
:1070A00030390A4E3533302058332E363339205993
:1070B000302E3132390A4E3533352058332E36359D
:1070C000302059302E3135390A4E3534302058337E
:1070D0002E3636332059302E3137380A4E35343576
:1070E0002058332E3637382059302E3139320A4E57
:1070F0003535302058332E3639392059302E313934
:10710000370A4E3535352058332E37323320593033
:107110002E3139360A4E3536302058332E37363434
:107120002059302E3137390A4E3536352058332E16
:107130003830352059302E3136350A4E353730202B
:1071400058332E3838342059302E3135390A4E35DF
:1071500037352058332E3934392059302E313635D1
:107160000A4E3538302058332E3936362059302ED5
:107170003137350A4E3538352058332E39373820D7
:1071800059302E3139340A4E3539302058332E39A2
:1071900037382059302E3232330A4E35393520589F
:1071A000332E3936302059302E3234350A4E3630AF
:1071B000302058332E3833342059302E3331310AB1
:1071C0004E3630352058332E3736322059302E3354
:1071D00034350A4E3631302058332E373236205966
:1071E000302E3338390A4E3631352058332E373069
:1071F000332059302E3435380A4E36323020583349
:107200002E3638322059302E3533300A4E3632354C
:107210002058332E3637392059302E3533340A4E24
:107220003633302058332E3632362059302E363809
:10723000310A4E3633352058332E35363820593002
:107240002E3832380A4E3634302058332E34343407
:107250002059312E3038300A4E3634352058332EEE
:107260003430352059312E3136370A4E36353020FC
:1072700058332E3430342059312E3136370A4E36B9
:1072800035352058332E3338372059312E323038A7
:107290000A4E3636302058332E3338342059312EAA
:1072A0003230380A4E3636352058332E33363520B4
:1072B00059312E3236350A4E3637302058332E3378
:1072C00035352059312E3238350A4E36373520586B
:1072D000332E3334382059312E3330380A4E363875
:1072E000302058332E3333332059312E3335300A82
:1072F0004E3638352058332E3332312059312E3323
:1073000039310A4E3639302058332E333131205935
:10731000312E3432380A4E3639352058332E333335
:10732000392059312E3432330A4E37303020583319
:107330002E3434302059312E3430360A4E37303521
:107340002058332E3531302059312E3430380A4E02
:107350003731302058332E3538352059312E3432DC
:10736000310A4E3731352058332E363131205931DC
:107370002E3433390A4E3732302058332E363131DD
:107380002059312E3434310A4E3732352058332EBD
:107390003631352059312E3434310A4E37333020CE
:1073A00058332E3633362059312E3438380A4E377A
:1073B00033352058332E3633342059312E3531377A
:1073C0000A4E3734302058332E3632322059312E7F
:1073D0003534330A4E3734352058332E3630352085
:1073E00059312E3536330A4E3735302058332E3545
:1073F00037362059312E3537350A4E373535205836
:10740000332E3534342059312E3538310A4E373643
:10741000302058332E3437392059312E3539320A3D
:107420004E3736352058332E3435312059312E35EC
:1074300039380A4E3737302058332E3338372059F1
:10744000312E3632360A4E3737352058332E3339FF
:10745000302059312E3633360A4E373830205833E3
:107460002E3533322059312E3630320A4E373835E8
:107470002058332E3630312059312E3539370A4EC7
:107480003739302058332E3636382059312E353999
:10749000380A4E3739352058332E37383220593193
:1074A0002E3631320A4E3830302058332E373934A8
:1074B0002059312E3631380A4E3830352058332E87
:1074C0003836382059312E3633360A4E383130208E
:1074D00058332E3931382059312E3635350A4E3849
:1074E00031352058332E3934352059312E36363740
:1074F0000A4E3832302058332E3936342059312E46
:107500003638350A4E3832352058332E3936372042
:1075100059312E3638350A4E3833302058332E390B
:1075200037342059312E3639390A4E383335205800
:10753000332E3938342059312E3732350A4E38340B
:10754000302058332E3938342059312E3735380A07
:107550004E3834352058332E3937302059312E37B4
:1075600039300A4E3835302058332E3934352059C9
:10757000312E3831370A4E3835352058332E3931CF
:10758000382059312E3832360A4E383630205833AA
:107590002E3839312059312E3832370A4E383635A7
:1075A0002058332E3834322059312E3830390A4E93
:1075B0003837302058332E3739382059312E373864
:1075C000340A4E3837352058332E37343620593167
:1075D0002E3737320A4E3838302058332E36393865
:1075E0002059312E3736340A4E3838352058332E4C
:1075F0003633352059312E3736360A4E3839302059
:1076000058332E3535332059312E3738350A4E3818
:1076100039352058332E3437382059312E3832300E
:107620000A4E3930302058332E3430392059312E1B
:107630003836340A4E3930352058332E333435201D
:1076400059312E3931380A4E3931302058332E32E3
:1076500036342059322E3032330A4E3931352058E3
:10766000332E3234382059322E3035310A4E3932E9
:10767000302058332E3234302059322E3038310AEF
:107680004E3932352058332E3331362059322E3090
:1076900038360A4E3933302058332E33393020599A
:1076A000322E3130340A4E3933352058332E3431AE
:1076B000342059322E3132310A4E39343020583389
:1076C0002E3433312059322E3135330A4E39343588
:1076D0002058332E3433332059322E3138300A4E6D
:1076E0003935302058332E3432372059322E32304B
:1076F000350A4E3935352058332E3431332059323E
:107700002E3232340A4E3936302058332E33393245
:107710002059322E3234320A4E3936352058332E23
:107720003333352059322E3234340A4E3937302033
:1077300058332E3237382059322E3233360A4E39EA
:1077400037352058332E3235362059322E323432E6
:107750000A4E3938302058332E3233392059322EE0
:107760003235310A4E3938352058332E32313120F6
:1077700059322E3238300A4E3939302058332E31B2
:1077800037342059322E3335360A4E3939352058A0
:10779000332E3135392059322E3339370A4E3130B4
:1077A00030302058332E3135302059322E34333892
:1077B0000A4E313030352058332E31343020593292
:1077C0002E3438310A4E313031302058332E313397
:1077D000322059322E3531300A4E31303135205871
:1077E000332E3131382059322E3534330A4E313070
:1077F00032302058332E3039392059322E35373631
:107800000A4E313032352058332E3035312059323E
:107810002E3633310A4E313033302058332E30304B
:10782000332059322E3636360A4E31303335205811
:10783000322E3935372059322E3638350A4E31300E
:1078400034302058322E3930372059322E363939DB
:107850000A4E313034352058322E383630205932E5
:107860002E3731310A4E313035302058322E3831F2
:10787000392059322E3732370A4E313035352058BB
:10788000322E3736382059322E3734350A4E3130C1
:1078900036302058322E3731362059322E37353790
:1078A0000A4E313036352058322E3637352059328F
:1078B0002E3735370A4E313037302058322E353793
:1078C000392059322E3733310A4E3130373520586E
:1078D000322E3537302059322E3732330A4E31307E
:1078E00038302058322E3535392059322E37323043
:1078F0000A4E313038352058322E35333020593247
:107900002E3730310A4E313039302058322E353052
:10791000312059322E3639330A4E3130393520581C
:10792000322E3437312059322E3638330A4E313127
:1079300030302058322E3434332059322E363638F7
:107940000A4E313130352058322E333936205932F3
:107950002E3633340A4E313131302058322E333501
:10796000342059322E3539310A4E313131352058D3
:10797000322E3335322059322E3539310A4E3131DB
:1079800032302058322E3332352059322E353433AE
:107990000A4E313132352058322E333135205932AA
:1079A0002E3532310A4E313133302058322E3330B9
:1079B000372059322E3439380A4E31313335205878
:1079C000322E3239362059322E3436340A4E313185
:1079D00034302058322E3239332059322E34323757
:1079E0000A4E313134352058322E32393520593251
:1079F0002E3336360A4E313135302058322E33325E
:107A0000312059322E3330330A4E3131353520583A
:107A1000322E3335382059322E3234370A4E313136
:107A200036302058322E3431392059322E3230330C
:107A30000A4E313136352058322E34313920593200
:107A40002E3137390A4E313137302058322E34300A
:107A5000352059322E3135380A4E313137352058DC
:107A6000322E3336322059322E3132330A4E3131F2
:107A700038302058322E3335342059322E313034BC
:107A80000A4E313138352058322E333534205932B0
:107A90002E3039310A4E313139302058322E3338B8
:107AA000302059322E3036350A4E31313935205892
:107AB000322E3431302059322E3035310A4E3132A7
:107AC00030302058322E3431302059322E30343775
:107AD0000A4E313230352058322E3430352059326A
:107AE0002E3032380A4E313231302058322E343076
:107AF000382059322E3031300A4E3132313520584B
:107B0000322E3431362059312E3939350A4E313240
:107B100032302058322E3433332059312E39383216
:107B20000A4E313232352058322E34333820593112
:107B30002E3936330A4E313233302058322E343417
:107B4000372059312E3934380A4E313233352058E6
:107B5000322E3436312059312E3933380A4E3132F3
:107B600034302058322E3438302059312E393331C8
:107B70000A4E313234352058322E343738205931BC
:107B80002E3839390A4E313235302058322E3438B9
:107B9000372059312E3837350A4E31323535205895
:107BA000322E3530342059312E3835340A4E3132A8
:107BB00036302058322E3532372059312E3834386D
:107BC0000A4E313236352058322E3534392059316B
:107BD0002E3834390A4E313237302058322E35376C
:107BE000372059312E3836310A4E31323735205848
:107BF000322E3630342059312E3836360A4E313254
:107C000038302058322E3633312059312E38353421
:107C10000A4E313238352058322E36343020593120
:107C20002E3832370A4E313239302058322E36341F
:107C3000302059312E3739320A4E313239352058F9
:107C4000322E3632392059312E3735390A4E3133FA
:107C500030302058322E3631322059312E373237DB
:107C60000A4E313330352058322E353736205931CF
:107C70002E3639340A4E313331302058322E3533D6
:107C8000362059312E3636320A4E313331352058AE
:107C9000322E3437302059312E3631360A4E3133B8
:107CA00032302058322E3334352059312E3535318B
:107CB0000A4E313332352058322E33303720593185
:107CC0002E3532310A4E313333302058322E32368F
:107CD000302059312E3438320A4E31333335205862
:107CE000322E3234332059312E3437370A4E313365
:107CF00034302058322E3232382059312E34363931
:107D00000A4E313334352058322E32323220593136
:107D10002E3434380A4E313335302058322E323238
:107D2000382059312E3432350A4E3133353520580A
:107D3000322E3235342059312E3430350A4E31331B
:107D400036302058322E3236382059312E333733E0
:107D50000A4E313336352058322E323739205931D8
:107D60002E3334320A4E313337302058322E3330EE
:107D7000382059312E3238370A4E313337352058B2
:107D8000322E3334302059312E3235340A4E3133CD
:107D900038302058322E3430372059312E3230319D
:107DA0000A4E313338352058322E3434312059318F
:107DB0002E3135360A4E313339302058322E343593
:107DC000342059312E3133310A4E31333935205870
:107DD000322E3436302059312E3130360A4E31347D
:107DE00030302058322E3436342059312E31303252
:107DF0000A4E313430352058322E34373120593143
:107E00002E3033360A4E313431302058322E34364B
:107E1000362059302E3937310A4E31343135205819
:107E2000322E3435312059302E3839370A4E31341C
:107E300032302058322E3431352059302E373931F6
:107E40000A4E313432352058322E343033205930F6
:107E50002E3736370A4E313433302058322E3338ED
:107E6000382059302E3736350A4E313433352058C4
:107E7000322E3330362059302E3834310A4E3134D8
:107E800034302058322E3232322059302E393131AE
:107E90000A4E313434352058322E313134205930A5
:107EA0002E3939350A4E313435302058322E3030A3
:107EB000322059312E3037360A4E3134353520587C
:107EC000312E3930352059312E3133390A4E313483
:107ED00036302058312E3735342059312E32323356
:107EE0000A4E313436352058312E36333720593149
:107EF0002E3237380A4E313437302058312E35384B
:107F0000322059312E3330310A4E31343735205832
:107F1000312E3535382059312E3331350A4E313432
:107F200038302058312E3436302059312E33353206
:107F30000A4E313438352058312E333939205931F1
:107F40002E3336300A4E313439302058312E333307
:107F5000382059312E3335340A4E313439352058D2
:107F6000312E3238372059312E3332390A4E3135DD
:107F700030302058312E3234382059312E323934B5
:107F80000A4E313530352058312E323137205931B3
:107F90002E3235340A4E313531302058312E3231BF
:107FA000342059312E3235320A4E31353135205890
:107FB000312E3137322059312E3139350A4E313593
:107FC00032302058312E3132382059312E31333968
:107FD0000A4E313532352058312E31313020593169
:107FE0002E3131370A4E313533302058302E393565
:107FF000382059302E3934310A4E31353335205836
:10800000302E3839312059302E3837330A4E313539
:1080100034302058302E3832352059302E38303810
:108020000A4E313534352058302E37353520593009
:108030002E3734370A4E313535302058302E363110
:10804000392059302E3633330A4E313535352058E4
:10805000302E3437372059302E3532360A4E3135EE
:1080600036302058302E3437372059302E353234C0
:108070000A4E313536352058302E343131205930C2
:108080002E3437360A4E313537302058302E3333C0
:10809000312059302E3435340A4E31353735205899
:1080A000302E3237382059302E3432370A4E31359F
:1080B00038302058302E3233312059302E33393772
:1080C0000A4E313538352058302E3138332059306A
:1080D0002E3337390A4E313539302058302E31336E
:1080E000352059302E3336350A4E31353935205842
:1080F000302E3037362059302E3334310A4E313657
:10810000303520473030204633302E300A4E31365D
:108110003130204D3035200A4E3136313520473947
:1081200030205830205930205A300A4E31363135FF
:10813000204D33300A28456E64206F6620434E433D
:108140002050726F6772616D2900284D53472A2AAB
:108150002A2A204D6963726F7374657020546573A9
:1081600074205B76315D202A2A2A2A290A4730307A
:1081700020473137204732312047343020473439C7
:1081800020473830204739300A6730783079307AE4
:10819000300A7B22316D69223A317D0A7B22326DB1
:1081A00069223A317D0A7B22336D69223A317D0A98
:1081B0007B22346D69223A317D0A67302078313074
:1081C0000A7B22316D69223A327D0A78300A7B229D
:1081D000316D69223A347D0A7831300A7B22316D63
:1081E00069223A387D0A78300A6730207931300ABE
:1081F0007B22326D69223A327D0A79300A7B223243
:108200006D69223A347D0A7931300A7B22326D69F8
:10821000223A387D0A79300A6730207A31300A7B79
:1082200022336D69223A327D0A7A300A7B22336D1D
:1082300069223A347D0A7A31300A7B22336D692211
:108240003A387D0A7A300A6730206131300A7B2261
:10825000346D69223A327D0A61300A7B22346D69BD
:10826000223A347D0A6131300A7B22346D69223A28
:10827000387D0A61300A6D3200284D53472A2A2A78
:108280002A20436F6F7264696E617465206F666641
:10829000736574732074657374205B76315D202A76
:1082A0002A2A2A290A673030673137673231673422
:1082B000306734396738306739300A6735340A67D0
:1082C0003932783079307A300A663630300A284DC3
:1082D00053472A2A2A2A207465737420473932208A
:1082E0006F6666736574732A2A2A2A290A286D73B1
:1082F000675374657020313A204D6F766520667241
:108300006F6D20302C3020746F2033302C30206D76
:108310006D20696E20706F736974697665205820CE
:10832000646972656374696F6E290A286D73675397
:1083300074657020323A205265736574206F7269DB
:1083400067696E20746F20302E30207573696E67F8
:1083500020473932290A286D7367537465702033BA
:108360003A204D6F766520746F2032302C302E20ED
:1083700053686F756C64206D6F7665203230206DA8
:108380006D20696E20706F7369746976652058205E
:10839000646972656374696F6E20616E64207374C2
:1083A00061747573207265706F72742073686F7575
:1083B0006C642073746172742066726F6D20302C4F
:1083C00030290A286D73675374657020343A204D44
:1083D0006F766520746F20302E3020202053686F18
:1083E000756C64206D6F7665203230206D6D20696C
:1083F0006E206E65676174697665205820646972C5
:10840000656374696F6E20616E6420737461747546
:1084100073207265706F72742073686F756C64205E
:1084200073746172742066726F6D2032302C302943
:108430000A67317833300A67393278300A67317821
:1084400032300A6731783079300A2473720A67391A
:108450003278300A673470302E350A284D53472A57
:108460002A2A2A207465737420473535206F666682
:10847000736574732A2A2A2A290A286D736753742C
:10848000657020313A2053657420436F6F726469C0
:108490006E6174652073797374656D2032205B673B
:1084A00035355D20746F206F6666736574206F6666
:1084B0002035302C3530290A286D73675374657068
:1084C00020323A2053656C6563742047353520634C
:1084D0006F6F7264696E6174652073797374656D12
:1084E000290A286D73675374657020333A204D6FE5
:1084F000766520746F20302C302E20486561642012
:1085000073686F756C64206D6F7665206469616750
:108510006F6E616C6C7920696E202B5820616E64DF
:10852000202B5920616E64207374617475732072FE
:1085300065706F72742073686F756C6420737461FA
:1085400072742066726F6D20302C30290A673130CA
:108550004C3270327835307935300A6735350A67F4
:1085600030783079300A673470302E350A284D5310
:10857000472A2A2A2A2074657374204735332061DC
:1085800062736F6C757465206F766572726964656D
:1085900073202A2A2A2A290A286D73675374657062
:1085A00020313A2052756E206120737175617265B9
:1085B00020696E204735352073797374656D290AFB
:1085C000286D73675374657020323A2052756E209F
:1085D000612073717561726520772F473533206F85
:1085E00076657272696465290A6730783079300A75
:1085F000673078323079300A67307832307932300B
:108600000A673078307932300A6730783079300A4A
:10861000673470302E350A673533673078307930FB
:108620000A673533673078323079300A6735336717
:10863000307832307932300A6735336730783079C4
:1086400032300A6735336730783079300A673078EE
:108650003079300A673470302E350A284D53472A56
:108660002A2A2A20746573742052657475726E20EC
:10867000746F20686F6D65202A2A2A2A290A286DBE
:1086800073675374657020313A2052657475726E49
:1086900020746F20686F6D65207573696E67204761
:1086A0003238290A286D73675374657020323A2076
:1086B000526573657420746F2047353420636F6F83
:1086C00072642073797374656D290A6732380A679A
:1086D00035340A6D333000284D53472A2A2A2A2080
:1086E00054657374206163637572616379206F668A
:1086F00020736C6F77206D6F766573205B76315DCC
:10870000202A2A2A2A290A6735350A6730783079DB
:10871000300A673470302E350A673470302E350ACF
:1087200067317831306632320A6735340A6730781B
:108730003079300A6D333000284D53472A2A2A2ACF
:10874000205465737420766572792073686F727433
:10875000206D6F766573205B76315D202A2A2A2A88
:10876000290A6730783079300A673470302E350A3C
:10877000673178302E3166313030300A78300A78FF
:10878000302E310A78300A78302E310A78300A7863
:10879000302E310A78300A78302E310A78300A7853
:1087A000302E310A78300A78302E310A78300A7843
:1087B000302E310A78300A78302E310A78300A7833
:1087C000302E310A78300A78302E310A78300A7823
:1087D000302E310A78300A78302E310A78300A7813
:1087E000302E310A78300A78302E310A67347030F2
:1087F0002E350A78300A78302E30310A78300A78EF
:10880000302E30310A78300A78302E30310A783004
:108810000A78302E30310A78300A78302E30310A1A
:1088200078300A78302E30310A78300A78302E309D
:10883000310A78300A78302E30310A78300A7830B0
:108840002E30310A78300A78302E30310A78300AEA
:1088500078302E30310A78300A78302E30310A786C
:10886000300A78302E30310A78300A78302E3031A4
:108870000A6730783079300A6D3200284D53472A24
:108880002A2A2A20526F74617279204178697320F4
:108890004D6F74696F6E2054657374205B76315D23
:1088A000202A2A2A2A290A6730306731376732316D
:1088B0006734306734396738306739300A67307861
:1088C0003079307A306130623063300A6735350A8A
:1088D0006730783079300A6633363030300A6730A6
:1088E000613336300A623336300A633336300A6118
:1088F000300A62300A63300A673161313434300A39
:1089000062313434300A63313434300A61300A62FF
:10891000300A63300A6731613134343062373230C3
:10892000633336300A783079307A306130623063C0
:10893000300A673178363061313434306237323062
:10894000633336300A783079307A306130623063A0
:10895000300A6731783630793530613134343062FD
:10896000373230633336300A783079307A306130DC
:10897000623063300A673178363079353078323595
:10898000613134343062373230633336300A783014
:1089900079307A306130623063300A6735340A6783
:1089A00030783079300A6D333000284D53472A2A09
:1089B0002A2A20496E76657273652054696D652098
:1089C0004D6F74696F6E2054657374205B76315DF2
:1089D000202A2A2A2A290A6730306731376732313C
:1089E0006734306734396738306739300A6735356E
:1089F0000A6730783079300A6739330A66302E30AA
:108A0000310A67317831300A7931300A7A31300AE7
:108A10006131300A78300A79300A7A300A61300AD6
:108A200067317831307931307A2D31306131300A27
:108A30006730783079307A3061300A66302E310A0A
:108A40006732783130792D31307A2D3230693130DA
:108A50000A6730783079307A300A67337831307984
:108A60002D31307A2D32306931300A6730783079E3
:108A7000307A300A673278323079307A2D32306984
:108A800031300A6730783079307A300A673378329B
:108A90003079306931300A6730783079307A300A8D
:108AA0006732783079307A2D33306931300A673364
:108AB000783079307A306931300A673078307930FF
:108AC0007A300A673278307930693230202843575B
:108AD000203336302064656772656573290A673311
:108AE000783079306932302028434357203336308C
:108AF0002064656772656573290A6739340A6735CA
:108B0000340A6730783079300A6D3330007B226761
:108B100063223A2267303067313767323167343049
:108B2000673439673830673930227D0A7B226763C2
:108B3000223A22673535227D0A7B226763223A2258
:108B4000673078307930227D0A7B226763223A22AF
:108B500066353030227D0A7B226763223A22284D17
:108B600053477371756172657329227D0A7B226791
:108B700063223A226730783230227D0A7B22676393
:108B8000223A22793230227D0A7B226763223A22FE
:108B90007830227D0A7B226763223A227930227D57
:108BA0000A7B226763223A226731783130227D0ABC
:108BB0007B226763223A22793130227D0A7B226749
:108BC00063223A227830227D0A7B226763223A228E
:108BD0007930227D0A7B226763223A22284D53474F
:108BE000636972636C657329227D0A7B2267632245
:108BF0003A226732783130792D3130693130227D37
:108C00000A7B226763223A22673078307930227DEE
:108C10000A7B226763223A226733783130792D311B
:108C200030693130227D0A7B226763223A22673025
:108C300078307930227D0A7B226763223A226732BC
:108C40007832307930693130227D0A7B22676322A5
:108C50003A22673078307930227D0A7B226763229E
:108C60003A2267337832307930693130227D0A7B9D
:108C7000226763223A22673078307930227D0A7B7E
:108C8000226763223A2267327830793069313022A4
:108C90007D0A7B226763223A226733783079306914
:108CA0003130227D0A7B226763223A2267353422E3
:108CB0007D0A7B226763223A22673078307930223E
:108CC0007D0A7B226763223A226D3330227D0028A1
:108CD0004D53472A2A2A2A204D636F6465732074F6
:108CE000657374205B76315D202A2A2A2A290A6757
:108CF00035350A6730783079300A6D330A67347059
:108D0000310A6D350A673470310A6D340A67347080
:108D1000310A6D350A673470310A6D370A6734706D
:108D2000310A6D390A673470310A6D380A67347058
:108D3000310A6D390A663530300A67307832300AC8
:108D40007932300A6D330A78300A6D340A79300A84
:108D50006D350A67317831300A6D370A7931300A5A
:108D60006D380A78300A6D390A79300A67327831FD
:108D700030792D31306931300A6D330A67307830FF
:108D800079300A6D340A6733783130792D313069A2
:108D900031300A6D350A6730783079300A6D370A1C
:108DA000673278323079306931300A6D380A67308D
:108DB000783079300A6D390A673378323079306922
:108DC00031300A6730783079300A6732783079305C
:108DD0006931300A6733783079306931300A673564
:108DE000340A6730783079300A6D333000284D53BB
:108DF000472A2A2A2A2046656564686F6C642054D5
:108E0000657374205B76315D202A2A2A2A290A2874
:108E10004D53472A2A2A2A204D616E75616C6C7960
:108E200020656E746572202120616E64207E20644E
:108E30007572696E67206D6F76656D656E742074EE
:108E40006F2074657374202A2A2A2A290A67353507
:108E50000A6730783079300A673470330A67303007
:108E60006731376732316734306734396738306794
:108E700039300A663630300A67307831303076372C
:108E8000362E3736350A783079300A6735340A6736
:108E900030783079300A6D333000284D53472A2A14
:108EA0002A2A204477656C6C2054657374205B76A5
:108EB000315D202A2A2A2A290A673030673137672C
:108EC00032316739300A6735350A673078307930A2
:108ED0000A663530300A67307831300A67347031CD
:108EE0000A67307832300A673470310A6730783177
:108EF000300A673470310A67307830300A6734706E
:108F0000310A79350A6735340A6730783079300AA2
:108F10006D330A673470310A673078313079313017
:108F20000A6D350A673470310A6730783230793229
:108F3000300A6D340A673470310A6730783330791B
:108F400033300A6D380A673470310A67307834304C
:108F50007934300A6D390A673470310A67307835F0
:108F6000307935300A6730783079300A6D33300027
:108F70002F286D73672A2A2A2A204172632054659C
:108F80007374205B76315D202A2A2A2A290A4E3101
:108F900020673030673137673231673430673439B2
:108FA0006738306739300A4E313020673078307991
:108FB000300A4E323020663530300A4E333020676A
:108FC00032783130792D31306931302028435720C3
:108FD0003237302064656772656573290A4E343014
:108FE000206730783079300A4E3530206733783159
:108FF00030792D31306931302028434357203930C2
:109000002064656772656573290A4E3630206730C3
:10901000783079300A4E3830206732783230793003
:109020006931302028435720313830206465677219
:10903000656573290A4E3730206730783079300AF9
:109040004E3830206733783230793069313020281B
:109050004343572031383020646567726565732952
:109060000A4E3930206730783079300A4E3939204D
:1090700046313230300A4E31303020673278307924
:1090800030693230202843572033363020646567FA
:1090900072656573290A4E31313020673278307934
:1090A00030693230202843572033363020616761E1
:1090B000696E290A4E31323020663730302028431D
:1090C00068616E67652066656564207261746520FD
:1090D0007768696C6520696E204732206D6F74690E
:1090E0006F6E206D6F6465290A4E31333020673210
:1090F0007830793069323020284357203336302099
:109100003372642074696D65290A4E3134302067EA
:109110003278307930693230202843572033363066
:10912000203474682074696D65290A4E3135302009
:10913000663530300A4E313630206733783079303A
:109140007A34306932302028434357203336302078
:10915000646567726565732077697468206C696EF1
:109160006561722074726176656C290A4E31373000
:10917000206733783079307A3069323020284343A1
:10918000572033363020616761696E290A4E3138C5
:1091900030206637303020286D73672A2A2A2A4308
:1091A00068616E676520666565642072617465201C
:1091B0007768696C6520696E204733206D6F74692C
:1091C0006F6E206D6F64652A2A2A2A290A4E31396A
:1091D0003020673378307930693230202843435764
:1091E00020333630203372642074696D65290A4E4D
:1091F000323030206733783079306932302028437C
:10920000435720333630203474682074696D6529E3
:109210000A4E32313020286D73672A2A2A2A4731B4
:1092200038204576616C20746573742A2A2A2A29AD
:109230000A4E323230204731205833302E37303703
:10924000205A35302E37323720463530300A4E32EC
:1092500033302047313820473032205836372E37C8
:109260003338205A32332E363137205232352046A9
:109270003235300A4E323430206738300A4E3235BB
:1092800030206730783079307A300A4E32363020EC
:109290006D333000284D53472A2A2A2A20537175EE
:1092A00061726573204D6F74696F6E2054657374BD
:1092B000205B76315D202A2A2A2A290A6730306706
:1092C000313767323167343067343967383067395E
:1092D000300A6730783079300A67307832302028A9
:1092E000747261766572736520612032306D6D2015
:1092F00073717561726520696E205820616E6420FB
:1093000059290A7932300A78300A79300A67317877
:109310003130663530302028647261772061203129
:10932000306D6D2073717561726520696E205820F3
:10933000616E6420592061742046353030290A79E5
:1093400031300A78300A79300A67307A3230202892
:10935000747261766572736520612032306D6D20A4
:1093600073717561726520696E205820616E64208A
:109370005A290A7832300A7A300A78300A67317806
:1093800032307932307A32306635303020286665B6
:10939000656420612032306D6D20646961676F6E95
:1093A000616C20696E20582C205920616E64205A0F
:1093B000290A783079307A300A7834307934307A42
:1093C00034302028747261766572736520612034B0
:1093D000306D6D206375626520696E20582C2059B0
:1093E00020616E64205A290A78343079307A300A44
:1093F00078307934307A34300A7834307934307ACD
:10940000300A783079307A34300A78307934307AEA
:10941000300A78343079307A34300A783079307ADA
:10942000300A6738300A6730783079300A67307828
:10943000310A673078300A6D333000284D53472A9F
:109440002A2A2A20486F6D696E672054657374203C
:109450005B76315D202A2A2A2A290A6732382E3281
:10946000783079307A300A6D333000284D53472AEE
:109470002A2A2A20536D6F6B652054657374205B14
:1094800076315D202A2A2A2A290A4730302047319E
:10949000372047323120473430204734392047388D
:1094A00030204739300A6D33673470310A6D3567C3
:1094B0003470310A6D34673470310A6D336734703B
:1094C000310A6D35673470310A6D37673470310A8F
:1094D0006D39673470310A6D38673470310A6D390F
:1094E0000A6730783079307A300A67303020783245
:1094F000300A78300A7932300A79300A7A32300A02
:109500007A300A6132300A61300A473030207832CE
:109510003020793230207A3230206132300A4730C0
:1095200030207830207930207A302061300A47307E
:109530003120663330207832207932207A3220612F
:10954000320A7830207930207A302061300A673052
:1095500078310A673078300A6D32002C000A002515
:109560007300256C750025312E3066002573002CA4
:10957000000A0025733A25730025733A256C75009F
:1095800025733A25312E30660025733A2573005B2A
:1095900074765D20207465787420766572626F73CE
:1095A00069747925313564205B303D73696C656E73
:1095B000742C313D766572626F73655D0A002566B5
:1095C0000A00256C750A0025640A0025730A0074D8
:1095D000696E7967205B25735D206572723A20257C
:1095E000733A202573200074696E7967205B2573B8
:1095F0005D206F6B3E200083CB18CBF0CB11CC707D
:10960000CC5DCB48CF18CBDCCF48D076CE5DCB003D
:1096100000400640061040B800B848CF18CBDCCF59
:1096200048D076CE5DCB0000400620060840B8004A
:10963000B8BED118CBDFD05AD109D3A8D0A00840EA
:10964000060506090108BED118CBDFD05AD182CC5D
:109650005DCBB00840060540B0308000000000003F
:10966000F0E0D0C0100100CF673322211F1B13018F
:10967000016E616E00696E66004E414E494E49545E
:1096800059494E46CDCCCC3D0AD7233C17B7D138EB
:1096900077CC2B329595E6241FB14F0A000020416C
:1096A0000000C84200401C4620BCBE4CCA1B0E5ADB
:1096B000AEC59D7400407A10F35A00A0724E18098E
:1096C0000010A5D4E80000E87648170000E40B5429
:1096D000020000CA9A3B000000E1F50500008096F8
:1096E0009800000040420F000000A086010000002A
:1096F000102700000000E8030000000064000000E4
:1097000000000A00000000000100000000002C76AC
:10971000D888DC674F0823DFC1DFAE59E1B1B796C7
:10972000E5E3E453C63AE651997696E8E6C2842624
:10973000EB898C9B62ED407C6FFCEFBC9C9F40F200
:10974000BAA56FA5F490055A2AF75C936B6CF9677C
:109750006DC11BFCE0E40D47FEF520E6B500D0ED41
:10976000902E0300943577050080841E08000020A9
:109770004E0A000000C80C333333330F986E128347
:109780001141EF8D2114893BE65516CFFEE6DB181B
:10979000D1844B381BF77C1D901DA4BBE4242032E0
:1097A00084725E228100C9F124ECA1E53D271124D9
:1097B0001FBECFEFCDBFDFE5DEBF00E00CBF13E281
:1097C000A0E0B0E2ECE9FCEC01E00BBF02C00790C6
:1097D0000D92AC38B107D9F724E5ACE8B3E201C08B
:1097E0001D92A43DB207E1F70E94D4840C944CE68C
:1097F0000C940000FC0160817181828193810E9440
:109800001DD860936A2C0895FC016081718182816A
:1098100093810E941DD86093692C0895AF92BF92E6
:10982000CF92DF92EF92FF920F931F93CF93DF932C
:109830007B018C018EEEC82E8BE2D82EE601AA2485
:10984000A394BC2EBC18F701619171918191919103
:109850007F012CEA35EC47E257E30E94ACD9181699
:109860004CF4F80140815181628173818B2D0E94FB
:109870004286A8820C5F1F4F2196FBE2C43FDF07A0
:1098800001F7DF91CF911F910F91FF90EF90DF9043
:10989000CF90BF90AF900C944D86FC016081718198
:1098A000828193810E941DD860936B2C613019F4E2
:1098B00081E00E94047C81E00C94257CCF93DF93AF
:1098C000CDB7DEB76897CDBFDEBFFC016081718187
:1098D000828193810E941DD860936C2C81E061305D
:1098E00019F40E94047C0CC00E94257CCE010196D4
:1098F00028E1FC0111922A95E9F7BC010E944D4C28
:109900006896CDBFDEBFDF91CF9108950F931F936F
:10991000CF93DF93CDB7DEB72D97CDBFDEBF27E066
:10992000E2EDF0E28E010F5F1F4FD80101900D9222
:109930002A95E1F7BC01660F771F680F791F660F44
:10994000771F660F771F660F771F6C5F794E45E0B4
:1099500050E0CE0108960E94A2E3688570E0C8013D
:109960000E94D0E3009739F46B8570E0C8010E9433
:10997000D0E3009711F0801B01C08FEF2D96CDBF73
:10998000DEBFDF91CF911F910F9108950F931F9329
:10999000CF93DF93CDB7DEB72D97CDBFDEBF27E0E6
:1099A000E9EDF0E28E010F5F1F4FD80101900D929B
:1099B0002A95E1F7BC01660F771F680F791F660FC4
:1099C000771F660F771F660F771F6C5F794E45E034
:1099D00050E0CE0108960E94A2E36B8570E0C801BA
:1099E0000E94D0E3009711F0801B01C08FEF2D96ED
:1099F000CDBFDEBFDF91CF911F910F910895EF9200
:109A0000FF920F931F93CF93DF938C01F62EE72ED7
:109A1000EC012D96FC0161857285838594850E94F9
:109A20001DD81F926F93DF93CF930F5E1F4F1F932D
:109A30000F93DF93CF93EF92FF92E0EDF4E58181F6
:109A40008F9380818F930E9469E4EDB7FEB73C96B7
:109A5000EDBFFEBFDF91CF911F910F91FF90EF906F
:109A600008950F931F93CF93DF93EC01162F072FC9
:109A70008C819D810E94864C83305CF58F3FA1F5DF
:109A800028C09E01235F3F4F9F938F938C858F93B8
:109A90008B858F938A858F9389858F933F932F939F
:109AA0006196DF93CF933F932F930F931F938091F2
:109AB000D1548F938091D0548F930E9469E48DB7D5
:109AC0009EB740968DBF9EBFDF91CF911F910F91A2
:109AD0000895E3E9F4E1659174914FE450E080E08A
:109AE00098E30E94A2E3CDCFE091642CF0E0EE0F6A
:109AF000FF1FE157FB4E659174914FE450E080E009
:109B000098E30E94A2E3BDCF0F931F93CF93DF93FF
:109B1000EC01162F072F8C819D810E94864C83308B
:109B20007CF58F3FC1F52CC0AE014F5E5F4F9E01AB
:109B3000235F3F4F9F938F938C858F938B858F935C
:109B40008A858F9389858F935F934F933F932F934C
:109B50005F934F933F932F930F931F938091D15413
:109B60008F938091D0548F930E9469E48DB79EB7F4
:109B700042968DBF9EBFDF91CF911F910F910895A7
:109B8000E3E9F4E1659174914FE450E080E098E3FB
:109B90000E94A2E3C9CFE091642CF0E0EE0FFF1F1A
:109BA000E157FB4E659174914FE450E080E098E3FB
:109BB0000E94A2E3B9CFDF92EF92FF920F931F931F
:109BC000CF93DF93CDB7DEB72897CDBFDEBF8B0134
:109BD000E42ED52E37E0E0EEF0E2DE0111960190A2
:109BE0000D923A95E1F728870E94864CF82E288539
:109BF00082E08F1518F0E22FF0E002C0E2E0F0E022
:109C0000EE0FFF1FE157FB4E659174914FE450E05A
:109C100080E098E30E94A2E39F938F93F8018381F1
:109C20008F9382818F9381818F9380818F93E1E0E5
:109C3000F0E0EC0FFD1FEF0DF11D80811F928F935F
:109C4000DF92EF928091D1548F938091D0548F9373
:109C50000E9469E4CDBFDEBF2896CDBFDEBFDF9195
:109C6000CF911F910F91FF90EF90DF9008954F9249
:109C70005F926F927F92AF92BF92CF92DF92EF92FC
:109C8000FF920F931F93CF93DF93CEEEDBE203EBB4
:109C90001AE25C018991813009F042C0F801C48068
:109CA000D580E680F7804080518062807380A30178
:109CB0009201C701B6010E943AD69F772CEA35EC93
:109CC00047E257E30E94A9D787FD2AC020E034E28B
:109CD00044E759ECC701B6010E94ACD918165CF4F0
:109CE000F5012081318142815381C701B6010E9473
:109CF000ACD9181604F120E034E244E759ECC30172
:109D0000B2010E94ACD918165CF4F50120813181B2
:109D100042815381C301B2010E94A9D787FD0BC0C4
:109D20000B5C1F4FF4E0AF0EB11C8BE2C43FD807B1
:109D300009F0B0CF02C08CED01C080E0DF91CF917F
:109D40001F910F91FF90EF90DF90CF90BF90AF9059
:109D50007F906F905F904F9008958091EA2B8111D2
:109D600005C08091E92B8093E82B29C0823031F423
:109D700087E08093E82B8091E92B21C0833031F478
:109D800089E08093E82B8091E92B19C0843031F46D
:109D90008AE08093E82B8091E92B11C08091EB2B16
:109DA000813031F485E08093E82B8091E92B07C066
:109DB000823019F486E08093E82B8091E92B86307D
:109DC00019F08091E82B08958BE08093E82B08959B
:109DD0008091E92B08958093EB2B813059F018F096
:109DE000823041F0089589E19CE28093172C909392
:109DF000182C089587E291E58093172C9093182CE6
:109E00000895FC0184810895845B9F4FFC0180814B
:109E10000895855B9F4FFC0180810895825B9F4F71
:109E2000FC0180810895815B9F4FFC018081089532
:109E3000875B9F4FFC01808108950C94289BCD96F1
:109E4000FC0160817181828193810895FC016483AA
:109E500008958C5A9F4FFC01608308958F5B9F4F3C
:109E6000FC01408351836283738308956093192CAE
:109E700070931A2C80931B2C90931C2C89EE91E2EA
:109E80000C94E366BF92CF92DF92EF92FF920F9312
:109E90001F93CF93DF93D090662C7C010AE81CE2DD
:109EA0008091652C90E0EC01CC0FDD1FC80FD91F0D
:109EB000CC0FDD1FCC0FDD1FCC0FDD1FCE5FD54DCE
:109EC00081E0D816A9F0B881A981CA80BB804091F1
:109ED000DD2C413091F4F8012081318142815381A0
:109EE0006B2F7A2F8C2D9B2D0E943BD69B0109C096
:109EF00020E030E080E090E004C02B2F3A2F8C2D42
:109F00009B2DA901BC01F701458F568F678F70A368
:109F1000F4E0EF0EF11C0C5F1F4F24968CE2023A26
:109F2000180771F6DF91CF911F910F91FF90EF907D
:109F3000DF90CF90BF900895835B9F4FFC016083BB
:109F400089E19CE20C94424F4F925F926F927F9214
:109F50008F929F92AF92BF92CF92DF92EF92FF9239
:109F60000F931F93CF93DF93CDB7DEB76897CDBF25
:109F7000DEBF8C016091DD2C70E080E090E00E94FB
:109F80004BD82B013C01F801608171818281938162
:109F90000E941DD870E05B01AA0CBB1CA60EB71E68
:109FA000AA0CBB1CAA0CBB1CAA0CBB1CC5018E5F57
:109FB000954D5C010AE81CE2FE0131964F01F50166
:109FC000C190D190E190F1905F01F80161917191A0
:109FD000819191918F01A30192010E944EDA9B0120
:109FE000AC01C701B6010E943BD6F40161937193A5
:109FF000819391934F01FCE2023A1F0701F7CE01D2
:10A0000001960E940B9B89E19CE20E94424F689658
:10A01000CDBFDEBFDF91CF911F910F91FF90EF90E9
:10A02000DF90CF90BF90AF909F908F907F906F9078
:10A030005F904F90089589519C4269F4E62FF0E0BB
:10A04000EE0FFF1FEE0FFF1FEE58F34D6081718181
:10A05000828193810895862F0C94009BCF92DF928A
:10A06000EF92FF920F931F93CF93DF93EC018CE25B
:10A07000C931D80709F04AC070E0FB01EE0FFF1F9D
:10A08000EE0FFF1FEE58F34DC080D180E280F380C9
:10A090008091662C813059F18091652C90E0FC0113
:10A0A000EE0FFF1FE80FF91FEE0FFF1FE60FF71F60
:10A0B000EE0FFF1FEE0FFF1FEE5FF54D00811181C8
:10A0C000B281A3812091DD2C2130B1F4FB01EE0F90
:10A0D000FF1FEE0FFF1FE657F34D208131814281B4
:10A0E0005381B8018B2F9A2F0E943BD608C060E0A5
:10A0F00070E080E090E003C0B8018B2F9A2F9B01A5
:10A10000AC01C701B6010E943AD603C0862F0E9457
:10A11000149BC55BDF4F2881211106C023E333E385
:10A120004BEC51E40E94B0D7DF91CF911F910F917A
:10A13000FF90EF90DF90CF90089588E1EEE1FCE290
:10A14000A2E7BCE201900D928A95E1F78091622C22
:10A1500081110CC080911D2C813041F41092562C3D
:10A160001092572C1092582C1092592C08954F92FF
:10A170005F926F927F928F929F92AF92BF92CF9297
:10A18000DF92EF92FF920F931F93CF93DF93CDB7A0
:10A19000DEB76997CDBFDEBF8091EA2B811155C034
:10A1A00080910F2C813009F050C00E94ABCA811100
:10A1B0004CC010920F2C7AE1672E7AE2772EE6E3FC
:10A1C0008E2E912C8E010E5E1F4FF7EEAF2EF0E219
:10A1D000BF2E33C0F70181917F011F928F935F9251
:10A1E0004F92BF92AF921F930F930E9434E5B80134
:10A1F00082E593E20E9449648D839E83F6018191FA
:10A200009191A191B1916F018A879B87AC87BD879E
:10A21000CE0101960E941B61CDBFDEBF98EDE9160D
:10A2200090E2F906B9F6E8E16E0E711CFFEF8F1AA5
:10A230009F0A8CE38816910441F0240163EDE62E19
:10A2400060E2F62E630188E7C8CF80E06996CDBF53
:10A25000DEBFDF91CF911F910F91FF90EF90DF90C4
:10A26000CF90BF90AF909F908F907F906F905F90B6
:10A270004F9008952F923F924F925F926F927F92EC
:10A280008F929F92AF92BF92CF92DF92EF92FF9206
:10A290000F931F93CF93DF93CDB7DEB72997CDBF31
:10A2A000DEBF4C015B014090682C5090662C2090E2
:10A2B000652C6090DD2C7090642C6B018EE19CE22B
:10A2C00088879987BAEAEB2EBAE2FB2E98E1299E9D
:10A2D000100111248401D6016D917D918D919D9184
:10A2E0006D012CEA35EC47E257E30E94A9D787FDC0
:10A2F00080C0F70180818150823008F07AC041101F
:10A300004CC0F1E05F1609F1E885F985E20DF31D17
:10A31000EC51F2408081898391819D83B281A38138
:10A32000E1E06E1217C0E885F985E459FF4F2081FE
:10A33000318142815381BC018B2F9A2F0E943BD6E1
:10A3400069837D838E839F8307C019821D821E824D
:10A350001F8202C0BE83AF8371100CC023E333E3BE
:10A360004BEC51E4D8016D917D918D919C910E94AF
:10A370004EDA05C0F8016081718182819381298163
:10A380003D814E815F810E943BD6A885B9856D9342
:10A390007D938D939C9313972CC0A885B9858D913F
:10A3A0009D910D90BC91A02D89839A83AB83BC8332
:10A3B00071100EC023E333E34BEC51E4F8016081EC
:10A3C0007181828193810E944EDA9B01AC0105C0AC
:10A3D000D8012D913D914D915C9169817A818B815C
:10A3E0009C810E943BD6E885F985608371838283D6
:10A3F00093838885998504968887998795E3E90EE4
:10A40000F11C0C5F1F4FA885B985AA52BC4209F008
:10A4100062CF6090642C7090682CF091662CF98368
:10A42000C090652C2091DD2C2D838CE0A80EB11CF2
:10A43000A9E4BBE2A887B987AAE2EA2EACE2FA2E29
:10A44000B8E1CB9E600111248401F5016191719105
:10A45000819191915F012CEA35EC47E257E30E942C
:10A46000A9D787FD8CC0A885B9858C91882309F46C
:10A4700086C08150823030F4F801248435844684CB
:10A4800057843BC0611016C023E333E34BEC51E427
:10A49000D8011C966D917D918D919C911F970E9482
:10A4A0004EDA20E030E044EB53E40E944EDA1B0128
:10A4B0002C010DC020E030E044EB53E4F80164854A
:10A4C0007585868597850E944EDA1B012C012BED40
:10A4D0003FE049EC50E4A885B98591966D917D9156
:10A4E0008D919C9194970E944EDA9B01AC01C20120
:10A4F000B1010E94B0D71B012C01711031C0B9818C
:10A50000B130E1F0F701EC0DFD1DEC51F240A081FE
:10A51000B18192808380ED81E130A1F4F701E459AB
:10A52000FF4F2081318142815381BD01892D982DBA
:10A530000E943BD6DB01982E892E04C0A0E0B0E03B
:10A54000912C812CA2019101BD01892D982D0E9491
:10A550003BD6D7016D937D938D939C9313970FC03A
:10A56000A2019101F70160817181828193810E9432
:10A570003BD6D7016D937D938D939C931397E8857C
:10A58000F985F596E887F987F4E0EF0EF11C0C5F8A
:10A590001F4F88859985885E9B4209F056CF299682
:10A5A000CDBFDEBFDF91CF911F910F91FF90EF9054
:10A5B000DF90CF90BF90AF909F908F907F906F90E3
:10A5C0005F904F903F902F9008958091E629909151
:10A5D000E7298F3E924111F08FE5089580919A2DE1
:10A5E00090919B2D8F3E9241B9F780916E2C909166
:10A5F0006F2C8F3E924181F78091E42C9091E52C55
:10A600008F3E924149F780917E5190917F518F3ECC
:10A61000924111F780913652909137528F3E92417C
:10A62000D9F680E008958091EA2B811104C083E07F
:10A630008093E92B03C085E08093E92B80E00895A7
:10A64000CF93C82F0E941DB780E00E9454B28C2F78
:10A650000E94D8AB86E08093E92B8C2FCF91089590
:10A660008093632C80E008958093642C80E00895AB
:10A670008093682C80E00895AF92BF92CF92DF92D2
:10A68000EF92FF920F931F93CF93DF939FEF980F5B
:10A69000963008F041C0A090642C7A018B0198E1BB
:10A6A000899F60011124F601EA51F64D6F01C0E067
:10A6B000D0E0BB24B394F7016191719181919191A4
:10A6C0007F012CEA35EC47E257E30E94ACD918161B
:10A6D000E4F4A1100CC023E333E34BEC51E4F801A4
:10A6E00060817181828193810E944EDA05C0F801F8
:10A6F0006081718182819381F601EC0FFD1F648F6F
:10A70000758F868F978FB0920F2C24960C5F1F4FFA
:10A71000C831D10581F602C085E101C080E0DF913A
:10A72000CF911F910F91FF90EF90DF90CF90BF904E
:10A73000AF900895CF93DF93CDB7DEB76897CDBFC5
:10A74000DEBF8093652C682F70E080E090E00E946F
:10A7500049D869837A838B839C831D821E821F82E2
:10A76000188619861A861B861C861D861E861F86DD
:10A77000188A198A1A8A1B8A1C8A1D8A1E8A1F8AAD
:10A78000188EAE014F5F5F4FBA0184EA9FE40E94CA
:10A79000848780E06896CDBFDEBFDF91CF910895BA
:10A7A000CF93DF93E9E1FCE285E5DF011D928A9515
:10A7B000E9F78AE5A6EEBCE2ED01982F19929A9589
:10A7C000E9F7A0E4BDE2ED0119928A95E9F78FEE71
:10A7D00092E18093E6299093E72980939A2D9093B4
:10A7E0009B2D80936E2C90936F2C8093E42C9093F0
:10A7F000E52C80937E5190937F51809336529093B5
:10A800003752E093172CF093182C8091FF298093F6
:10A81000642C8091FD290E949A538091FE29809397
:10A82000632C8091002A8093672C8091012A809369
:10A83000682C81E08093622C8093DE2C94E09093CE
:10A840001D2C1092102C1092112C1092122C80930F
:10A85000E92B8093E82B0E94F2B0DF91CF910C940A
:10A86000C688CF92DF92EF92FF92CF93C82F6A01F2
:10A870007B01E82FF0E0DF01AA0FBB1FAA0FBB1F6F
:10A88000AE58B34D4D935D936D937C931397EE0F3C
:10A89000FF1FEE0FFF1FE25EF34D40835183628383
:10A8A00073838C2F0E943786B701A6018C2F0E94DC
:10A8B0004286CF91FF90EF90DF90CF900C944D8621
:10A8C0003F924F925F926F927F928F929F92AF9240
:10A8D000BF92CF92DF92EF92FF920F931F93CF938D
:10A8E000DF93CDB7DEB76897CDBFDEBF362E872E9C
:10A8F000A62EB72E6C0100E010E0E12CF12C9E2C6E
:10A90000F50161917191819191915F012CEA35EC92
:10A9100047E257E30E94ACD918160CF050C0809162
:10A92000652C90E0FC01EE0FFF1FE80FF91FEE0F02
:10A93000FF1FEE0DFF1DEE0FFF1FEE0FFF1FEE5F5F
:10A94000F54D40805180628073808091642C81112C
:10A950000EC023E333E34BEC51E4F60160817181D7
:10A96000828193810E944EDA9B01AC0105C0F60101
:10A970002081318142815381C301B2010E943BD6C3
:10A98000AB01BC01E1E0F0E0EC0FFD1FE00FF11FB7
:10A99000408351836283738398012A51364DF901B4
:10A9A000E457FD4F4083518362837383E455F1097B
:10A9B0004083518362837383892D0E943786FFEF22
:10A9C000EF1AFF0A0C5F1F4F84E0C80ED11C08313C
:10A9D000110509F094CF432D582DBE016F5F7F4FB5
:10A9E0008EE09CE40E94848780E06896CDBFDEBF45
:10A9F000DF91CF911F910F91FF90EF90DF90CF905B
:10AA0000BF90AF909F908F907F906F905F904F908E
:10AA10003F9008954F925F926F927F928F929F9294
:10AA2000AF92BF92CF92DF92EF92FF920F931F935C
:10AA3000CF93DF93CDB7DEB76897CDBFDEBF21E000
:10AA40002093DD2C8090652C9090642C5B016C0130
:10AA500002E71CE2882D90E07C01EE0CFF1CE80E62
:10AA6000F91EEE0CFF1CEE0CFF1CEE0CFF1CC701C8
:10AA70008E5F954D7C01F50161917191819191916C
:10AA80005F012CEA35EC47E257E30E94ACD9181677
:10AA900064F5F7012081318142815381F8016081A1
:10AAA0007181828193810E943AD62B013C019110E1
:10AAB0000EC023E333E34BEC51E4F6016081718176
:10AAC000828193810E944EDA9B01AC0105C0F601A0
:10AAD0002081318142815381C301B2010E943AD663
:10AAE000F801608F718F828F938FF4E0CF0ED11CAD
:10AAF0000C5F1F4F84E0E80EF11C9CE20A38190736
:10AB000009F0B9CF682D70E080E090E00E9449D84C
:10AB100069837A838B839C831D821E821F821886A1
:10AB200019861A861B861C861D861E861F86188A15
:10AB3000198A1A8A1B8A1C8A1D8A1E8A1F8A188EE5
:10AB4000AE014F5F5F4FBA0184EA9FE40E948487A1
:10AB500080E06896CDBFDEBFDF91CF911F910F914E
:10AB6000FF90EF90DF90CF90BF90AF909F908F902D
:10AB70007F906F905F904F900895CF93DF93CDB704
:10AB8000DEB76897CDBFDEBF1092DD2C10928A2C05
:10AB900010928B2C10928C2C10928D2C10928E2C4B
:10ABA00010928F2C1092902C1092912C1092922C2B
:10ABB0001092932C1092942C1092952C1092962C0B
:10ABC0001092972C1092982C1092992C10929A2CEB
:10ABD00010929B2C10929C2C10929D2C10929E2CCB
:10ABE00010929F2C1092A02C1092A12C6091652C99
:10ABF00070E080E090E00E9449D869837A838B837B
:10AC00009C831D821E821F82188619861A861B86C7
:10AC10001C861D861E861F86188A198A1A8A1B8A18
:10AC20001C8A1D8A1E8A1F8A188EAE014F5F5F4FD5
:10AC3000BA0184EA9FE40E94848780E06896CDBFD1
:10AC4000DEBFDF91CF910895CF93DF93CDB7DEB70D
:10AC50006897CDBFDEBF1092DD2C6091652C70E04F
:10AC600080E090E00E9449D869837A838B839C833B
:10AC70001D821E821F82188619861A861B861C86D4
:10AC80001D861E861F86188A198A1A8A1B8A1C8AA4
:10AC90001D8A1E8A1F8A188EAE014F5F5F4FBA0150
:10ACA00084EA9FE40E94848780E06896CDBFDEBF7F
:10ACB000DF91CF910895CF93DF93CDB7DEB768973B
:10ACC000CDBFDEBF81E08093DD2C6091652C70E00C
:10ACD00080E090E00E9449D869837A838B839C83CB
:10ACE0001D821E821F82188619861A861B861C8664
:10ACF0001D861E861F86188A198A1A8A1B8A1C8A34
:10AD00001D8A1E8A1F8A188EAE014F5F5F4FBA01DF
:10AD100084EA9FE40E94848780E06896CDBFDEBF0E
:10AD2000DF91CF910895CF9310921D2C0E943A513C
:10AD30008091F029813069F48EE19CE20E94374EC7
:10AD4000C82F882331F00E94D8AB82E08093E92B92
:10AD500017C089E19CE20E94424F85E08093E92B75
:10AD60008091EA2B811105C081E08093EA2B0E943B
:10AD70004AAF89E19CE20E94359B0E949D50C0E051
:10AD80008C2FCF91089588E1E2E7FCE2A2EABCE2D1
:10AD900001900D928A95E1F780E008950F931F933B
:10ADA000CF93DF93CDB7DEB76A97CDBFDEBF8C01FF
:10ADB00081E08093662C89E19CE2698F7A8F0E9402
:10ADC000424F698D7A8DC8010E9493560E94BE86BB
:10ADD0008823E1F388E1E0E0F0E2DE0111960190E2
:10ADE0000D928A95E1F7BE016F5F7F4F82EA9CE288
:10ADF0000E9493566A96CDBFDEBFDF91CF911F911F
:10AE00000F91089588E1E2E7FCE2AAEBBCE2019031
:10AE10000D928A95E1F780E008950F931F93CF93E9
:10AE2000DF93CDB7DEB76A97CDBFDEBF8C0181E07F
:10AE30008093662C89E19CE2698F7A8F0E94424F51
:10AE4000698D7A8DC8010E9493560E94BE86882320
:10AE5000E1F388E1E0E0F0E2DE01119601900D926D
:10AE60008A95E1F7BE016F5F7F4F8AEB9CE20E94FB
:10AE700093566A96CDBFDEBFDF91CF911F910F91A0
:10AE80000895FB01DC018091622C811111C09B01AE
:10AE9000AD0160E070E080E89FE30E94B0D760936E
:10AEA000562C7093572C8093582C9093592C18C083
:10AEB0008091642C811109C023E333E34BEC51E40E
:10AEC000CD010E944EDAFB0101C0CD01AF01BC01F2
:10AED0004093562C5093572C6093582C7093592CB8
:10AEE00080E008958093622C80E008958093672C21
:10AEF00080E0089560935E2C70935F2C8093602CAB
:10AF00009093612C0E94DC8780E008950F931F933B
:10AF1000CF93DF93EC018B018091622C882399F011
:10AF20008091562C9091572CA091582CB091592C6F
:10AF3000BC01CD019F772CEA35EC47E257E30E9434
:10AF4000A9D787FD30C081E080931D2CB801CE01C8
:10AF50000E943A518091F029813069F48EE19CE29F
:10AF60000E94374EC82F882331F00E94D8AB82E070
:10AF70008093E92B19C089E19CE20E94424F85E051
:10AF80008093E92B8091EA2B811105C081E08093A9
:10AF9000EA2B0E944AAF89E19CE20E94359BC82FB0
:10AFA0000E949D5001C0CEE88C2FDF91CF911F9160
:10AFB0000F910895CF93DF93CDB7DEB76897CDBFDC
:10AFC000DEBF682F70E080E090E00E9449D869837E
:10AFD0007A838B839C831D821E821F82188619862A
:10AFE0001A861B861C861D861E861F86188A198A4D
:10AFF0001A8A1B8A1C8A1D8A1E8A1F8A188EAE0115
:10B000004F5F5F4FBA018AEF9BE40E94848780E024
:10B010006896CDBFDEBFDF91CF910895CF93DF93C8
:10B02000CDB7DEB76897CDBFDEBF60916A2C70E008
:10B0300080E090E00E9449D869837A838B839C8367
:10B040001D821E821F82188619861A861B861C8600
:10B050001D861E861F86188A198A1A8A1B8A1C8AD0
:10B060001D8A1E8A1F8A188EAE014F5F5F4FBA017C
:10B0700084E09CE40E94848780E06896CDBFDEBFB8
:10B08000DF91CF910895CF93DF93CDB7DEB7689767
:10B09000CDBFDEBF682F70E080E090E00E9449D80D
:10B0A00069837A838B839C831D821E821F8218860C
:10B0B00019861A861B861C861D861E861F86188A80
:10B0C000198A1A8A1B8A1C8A1D8A1E8A1F8A188E50
:10B0D000AE014F5F5F4FBA018DE49CE40E9484870C
:10B0E00080E06896CDBFDEBFDF91CF910895CF930A
:10B0F000DF93CDB7DEB76897CDBFDEBF682F70E0B6
:10B1000080E090E00E9449D869837A838B839C8396
:10B110001D821E821F82188619861A861B861C862F
:10B120001D861E861F86188A198A1A8A1B8A1C8AFF
:10B130001D8A1E8A1F8A188EAE014F5F5F4FBA01AB
:10B140008EE59CE40E94848780E06896CDBFDEBFD8
:10B15000DF91CF910895CF93FC016081718182814D
:10B1600093810E941DD86093E92B1092EB2B89E10B
:10B170009CE28093172C9093182C8091EA2B8130BD
:10B1800011F41092EA2B1092EC2B1092122C0E94C8
:10B19000EE9AC091E92BC430C9F40E94BD5580914C
:10B1A000FD290E949A538091FE298093632C8091FF
:10B1B000012A8093682C80E00E9454B280E00E94B3
:10B1C000775881E08093622CC0931D2C81E0CF9151
:10B1D0000C940EAE8093DA2C8093DB2C8093E32CBE
:10B1E00080E008952CEA35EC47E257E36091862D24
:10B1F0007091872D8091882D9091892D0E94ACD9D6
:10B200001816B4F480912C2D90912D2DA0912E2DF7
:10B21000B0912F2DBC01CD019F772CEA35EC47E290
:10B2200057E30E94A9D787FF03C01092DA2C03C00E
:10B2300081E08093DA2C80E008958093DA2C80916D
:10B240002C2D90912D2DA0912E2DB0912F2D8093EE
:10B25000D22C9093D32CA093D42CB093D52C80E0F7
:10B2600008952CEA35EC47E257E36091862D709102
:10B27000872D8091882D9091892D0E94ACD9181628
:10B28000B4F480912C2D90912D2DA0912E2DB09164
:10B290002F2DBC01CD019F772CEA35EC47E257E317
:10B2A0000E94A9D787FF03C01092DB2C03C081E066
:10B2B0008093DB2C80E008958093DB2C80912C2DF3
:10B2C00090912D2DA0912E2DB0912F2D8093D62CC5
:10B2D0009093D72CA093D82CB093D92C80E00895CC
:10B2E0002CEA35EC47E257E36091862D7091872D6B
:10B2F0008091882D9091892D0E94ACD91816B4F4B4
:10B3000080912C2D90912D2DA0912E2DB0912F2D2F
:10B31000BC01CD019F772CEA35EC47E257E30E9450
:10B32000A9D787FF03C01092E32C03C081E080936C
:10B33000E32C80E008958093E32C80912C2D909154
:10B340002D2DA0912E2DB0912F2D8093DF2C909339
:10B35000E02CA093E12CB093E22C80E00895BC0196
:10B360008EEE90E20C94066781E08093102C089595
:10B3700081E08093112C089581E08093122C089530
:10B380001F93CF93DF93CDB7DEB76897CDBFDEBFF6
:10B390000E94289B8130C9F10E9481D40E9441877C
:10B3A00080E00E945FAF0E9468B010E0812F0E9491
:10B3B000009BAB01BC01812F0E9431541F5F1630EE
:10B3C000A9F780E090E0A0E4B0E489839A83AB839E
:10B3D000BC831D821E821F82188619861A861B86D0
:10B3E0001C861D861E861F86188A198A1A8A1B8A41
:10B3F0001C8A1D8A1E8A1F8A188EBE016F5F7F4FAE
:10B40000CB010E94AB5880E001C080E76896CDBFB9
:10B41000DEBFDF91CF911F9108958091102C813074
:10B42000A9F42091EB2B213079F48091EC2B811140
:10B430000BC082E08093EB2B87E291E58093172C81
:10B440009093182C2093EC2B1092102C8091112C9F
:10B45000813091F48091EB2B882331F0823061F4BC
:10B460009091EC2B943051F40E94289B811104C0E0
:10B470001092112C0E94C0599091EC2B8091122CAB
:10B480008130C1F42091112C211114C091509330BE
:10B4900088F01092122C95E09093EC2B9093E92B6E
:10B4A0009091EA2B911104C08093EA2B0E944AAF3D
:10B4B0000E9479A380E0089585E08093E92B809134
:10B4C000EA2B811105C081E08093EA2B0C944AAFEE
:10B4D0000895CF93DF93CDB7DEB76897CDBFDEBFBA
:10B4E0008091EA2B882311F180E090E0A0E4B0E4A1
:10B4F00089839A83AB83BC831D821E821F82188638
:10B5000019861A861B861C861D861E861F86188A2B
:10B51000198A1A8A1B8A1C8A1D8A1E8A1F8A188EFB
:10B52000BE016F5F7F4FCB010E94AB586896CDBFC5
:10B53000DEBFDF91CF910895CF93DF93CDB7DEB714
:10B540006897CDBFDEBF80E090E0A0E4B0E48983DF
:10B550009A83AB83BC831D821E821F821886198644
:10B560001A861B861C861D861E861F86188A198AC7
:10B570001A8A1B8A1C8A1D8A1E8A1F8A188EAE018F
:10B580004F5F5F4FBA018BEA98E50E948487689607
:10B59000CDBFDEBFDF91CF910895CF93DF93CDB7BD
:10B5A000DEB76897CDBFDEBF80E090E0A0E8B0E4F2
:10B5B00089839A83AB83BC831D821E821F82188677
:10B5C00019861A861B861C861D861E861F86188A6B
:10B5D000198A1A8A1B8A1C8A1D8A1E8A1F8A188E3B
:10B5E000AE014F5F5F4FBA018BEA98E50E948487F6
:10B5F0006896CDBFDEBFDF91CF910895CF93DF93E3
:10B60000CDB7DEB72797CDBFDEBF97E0E0EEF0E223
:10B61000DE01119601900D929A95E1F7873050F472
:10B62000E1E0F0E0EC0FFD1FE80FF11D87FDFA955A
:10B63000808101C080E22796CDBFDEBFDF91CF9130
:10B640000895EF92FF920F931F93CF93DF931F9272
:10B65000CDB7DEB77C018B01642F70E080E090E015
:10B6600049830E9449D8F70161877287838794874D
:10B6700082E087834981E42FF0E0EE0FFF1FE00FA7
:10B68000F11F659174914FE450E080E098E30E94CF
:10B69000A2E3BC01C7010F90DF91CF911F910F91E1
:10B6A000FF90EF900C94A866CF93DF93EC010E947B
:10B6B000AD4E482F6DEC73E1CE01DF91CF910C942C
:10B6C000215B4091E92B6EE873E10C94215B409182
:10B6D000EA2B65E673E10C94215B4091EB2B61E56D
:10B6E00073E10C94215B4091EC2B63E273E10C94C9
:10B6F000215B4091ED2B66E073E10C94215BE091BE
:10B70000172CF091182CE55BFF4F408160E374E14A
:10B710000C94215BE091172CF091182CE45BFF4F07
:10B7200040816CE372E10C94215BE091172CF09165
:10B73000182C448162EA71E10C94215BE091172C92
:10B74000F091182CE65BFF4F40816FE671E10C949D
:10B75000215BE091172CF091182CE25BFF4F4081A8
:10B7600065E271E10C94215BE091172CF091182CAB
:10B77000E15BFF4F408164EE70E10C94215BE0914E
:10B78000172CF091182CE75BFF4F408165E770E1C3
:10B790000C94215BCF93DF93EC01E091172CF09197
:10B7A000182CE05BFF4F608170E080E090E00E9429
:10B7B00049D869877A878B879C8782E08F8380E06E
:10B7C000DF91CF910895CF93DF93EC016091192C15
:10B7D00070911A2C80911B2C90911C2C0E9449D89E
:10B7E00069877A878B879C8782E08F8380E0DF91EF
:10B7F000CF910895CF93DF93EC01E091172CF09156
:10B80000182C60817181828193810E9449D8698757
:10B810007A878B879C8782E08F8380E0DF91CF914E
:10B820000895CF93DF93EC018091EB2B811105C03C
:10B8300019861A861B861C8614C00E94F79A69878F
:10B840007A878B879C872091725121110AC025E845
:10B8500032E441E25DE30E944EDA69877A878B87A2
:10B860009C878C819D81FC01EE0FFF1FE80FF91F63
:10B87000EE0FFF1FEE0FFF1FEE0FFF1FE55FF94EEC
:10B8800085919491888784E08F8380E0DF91CF91C8
:10B890000895CF93DF93EC012091172C3091182C51
:10B8A000F901FD96608171818281938169877A8730
:10B8B0008B879C873E96208121110AC025E832E4BF
:10B8C00041E25DE30E944EDA69877A878B879C8725
:10B8D0008C819D81FC01EE0FFF1FE80FF91FEE0F19
:10B8E000FF1FEE0FFF1FEE0FFF1FE55FF94E859163
:10B8F0009491888784E08F8380E0DF91CF910895D1
:10B90000CF93DF93EC018C819D810E94864C682F40
:10B910008091172C9091182C0E942E5069877A875D
:10B920008B879C878C819D81FC01EE0FFF1FE80FA8
:10B93000F91FEE0FFF1FEE0FFF1FEE0FFF1FE55F5A
:10B94000F94E85919491888784E08F8380E0DF9120
:10B95000CF910895CF93DF93EC018C819D810E945C
:10B96000864C2091172C3091182C29513C4269F4B7
:10B97000E82FF0E0EE0FFF1FEE0FFF1FEE58F34D24
:10B98000608171818281938102C00E94009B6987DE
:10B990007A878B879C878C819D81FC01EE0FFF1F2E
:10B9A000E80FF91FEE0FFF1FEE0FFF1FEE0FFF1F37
:10B9B000E55FF94E85919491888784E08F8380E0DC
:10B9C000DF91CF910895CF93DF93EC018C819D811E
:10B9D0000E94864CE091172CF091182C94E0899FDE
:10B9E000E00DF11D1124458D568D678D70A149879D
:10B9F0005A876B877C878C819D81FC01EE0FFF1F2E
:10BA0000E80FF91FEE0FFF1FEE0FFF1FEE0FFF1FD6
:10BA1000E55FF94E85919491888784E08F8380E07B
:10BA2000DF91CF910895CF93DF93EC018C819D81BD
:10BA30000E94C64C0E9471B7682F70E080E090E0D1
:10BA40000E9449D869877A878B879C8782E08F8399
:10BA500080E0DF91CF910895CF93DF93EC010E94B6
:10BA6000FE6169857A858B859C850E941DD8462F4D
:10BA70006CE574E1CE01DF91CF910C94215BCF9303
:10BA8000DF93EC018C819D810E94864C833054F4BD
:10BA90008F3FA9F407C0CE010E94A86280E01CC0BD
:10BAA0008BE61AC020E030E040E450E469857A85F6
:10BAB0008B859C850E94ACD9181694F3ECCF20E0BE
:10BAC00030E040E050E469857A858B859C850E9452
:10BAD000ACD918162CF3DFCFDF91CF91089595E301
:10BAE000899FF0011124E554F54D608171818281B7
:10BAF00093810895CF92DF92EF92FF92CF93DF93DD
:10BB00006A017B0125E3829FC00111248A51964D71
:10BB1000FC01EB52FF4F4083518362837383EC013E
:10BB2000C352DF4F20E034E244E759E4C701B601D5
:10BB30000E944EDA9B01AC0160E070E080E89FE378
:10BB40000E94B0D7688379838A839B83DF91CF91EA
:10BB5000FF90EF90DF90CF900895CF92DF92EF9219
:10BB6000FF92CF93DF93EC01C984DA84EB84FC84E9
:10BB700020E034E244E759E4C701B6010E94ACD9A1
:10BB8000181664F420E034E244E759E4C701B60132
:10BB90000E94B0D769877A878B879C87CE010E94E5
:10BBA000BB67C984DA84EB84FC848C819D810E940C
:10BBB000864C25E3829FC00111248A51964DFC01D9
:10BBC000EB52FF4FC082D182E282F382EC01C3527A
:10BBD000DF4F20E034E244E759E4C701B6010E9498
:10BBE0004EDA9B01AC0160E070E080E89FE30E94C8
:10BBF000B0D7688379838A839B8380E0DF91CF917C
:10BC0000FF90EF90DF90CF900895CF92DF92EF9268
:10BC1000FF92CF93DF93EC01C984DA84EB84FC8438
:10BC200020E034E244E759E4C701B6010E94ACD9F0
:10BC3000181664F420E034E244E759E4C701B60181
:10BC40000E94B0D769877A878B879C87CE010E9434
:10BC5000BB6780E0DF91CF91FF90EF90DF90CF90B6
:10BC6000089581E08093112C80E008952CEA35EC52
:10BC700047E257E3FC0161857285838594850E94C4
:10BC8000ACD9181614F40E94946F80E00895609166
:10BC9000132C7091142C8091152C9091162C0895D2
:10BCA0000E94D26380E00E94177280E008950E9493
:10BCB000D26381E00E94177280E008950E94D263EF
:10BCC00082E00E94177280E008950E94D26383E0B0
:10BCD0000E94177280E00895CF93DF93EC01E0910A
:10BCE000172CF091182CE55BFF4FE081F0E0EE0F90
:10BCF000FF1FE157FB4E659174914FE450E080E0E7
:10BD000098E30E94A2E3AC016EE570E1CE01DF9101
:10BD1000CF910C9411C6CF93DF93EC01E091172CD7
:10BD2000F091182CE55BFF4FE081F0E0EE0FFF1F74
:10BD3000E157FB4E659174914FE450E080E098E349
:10BD40000E94A2E3AC0166E470E1CE01DF91CF91E5
:10BD50000C9411C6CF93DF93EC0182EF90E20E9426
:10BD600007E5CE010E946C5ECE010E948B5E62E30D
:10BD700070E1CE010E94D8C569E170E1CE010E9458
:10BD8000A3C560E070E1CE010E94A3C567EE7FE02D
:10BD9000CE010E94A3C56EEC7FE0CE010E94A3C538
:10BDA00065EB7FE0CE010E94A3C56CE97FE0CE0188
:10BDB0000E94A3C563E87FE0CE010E94A3C56AE6A6
:10BDC0007FE0CE010E94A3C561E57FE0CE010E9425
:10BDD000A3C568E37FE0CE010E94A3C56FE17FE0C9
:10BDE000CE010E94A3C566E07FE0CE010E94A3C5FC
:10BDF0006DEE7EE0CE010E94A3C564ED7EE0CE0133
:10BE00000E94D8C580E0DF91CF91089562E370E190
:10BE10000C94D8C569E170E10C94A3C560E070E1B1
:10BE20000C94A3C567EE7FE00C94A3C56EEC7FE095
:10BE30000C94A3C565EB7FE00C94A3C56CE97FE08F
:10BE40000C94A3C563E87FE00C94A3C56AE67FE089
:10BE50000C94A3C561E57FE00C94A3C568E37FE083
:10BE60000C94A3C56FE17FE00C94A3C566E07FE06E
:10BE70000C94A3C56DEE7EE00C94A3C564ED7EE04A
:10BE80000C94D8C568E57EE00C94D8C567E27EE0E6
:10BE90000C94D8C562EF7DE00C94D8C567EB7DE0CB
:10BEA0000C94D8C563E87DE00C94D8C5CF93DF939C
:10BEB000EC01E091172CF091182CE55BFF4FE0812D
:10BEC000F0E0EE0FFF1FE157FB4E659174914FE4D8
:10BED00050E080E098E30E94A2E3AC016FE57DE0D2
:10BEE000CE01DF91CF910C9411C6CF93DF93EC017B
:10BEF000E091172CF091182CE55BFF4FE081F0E00A
:10BF0000EE0FFF1FE157FB4E659174914FE450E037
:10BF100080E098E30E94A2E3AC016EE37DE0CE01F5
:10BF2000DF91CF910C9411C661E27DE00C94B9C50C
:10BF3000CF93DF93EC01E091172CF091182CE55B87
:10BF4000FF4FE081F0E0EE0FFF1FE157FB4E6591E0
:10BF500074914FE450E080E098E30E94A2E3AC01CA
:10BF600062E07DE0CE01DF91CF910C9411C60F937A
:10BF70001F93CF93DF938C01FC01618572858385CC
:10BF800094850E941DD8E62FF0E0EE0FFF1FE45AC3
:10BF9000FB4E659174914FE450E080E098E30E947D
:10BFA000A2E3E8012D969F938F93F8016185728536
:10BFB000838594850E941DD81F926F93DF93CF9342
:10BFC0000F5E1F4F1F930F93DF93CF9386EE9CE07E
:10BFD0009F938F93E0EDF4E581818F9380818F9320
:10BFE0000E9469E4EDB7FEB73E96EDBFFEBFDF915C
:10BFF000CF911F910F9108956EEB7CE00C94314D21
:10C0000066E97CE00C94314D64E77CE00C94314DA2
:10C0100062E57CE00C94314D60E27CE00C94314DA3
:10C020006FEE7BE00C94314D66EB7BE00C94314D70
:10C0300066E97BE00C94314D64E57BE00C94FF4CA9
:10C0400062E17BE00C94FF4C6BEE7AE00C94314D96
:10C0500065EC7AE00C94314D64EA7AE00C94314D51
:10C0600064E87AE00C94314D67E67AE00C94844DF4
:10C0700068E47AE00C94844DBC01675F7F4F2091A7
:10C08000642C4EEB5EE0FC01848195810C94DB4DC9
:10C09000BC01675F7F4F21E044EA5EE0FC018481E0
:10C0A00095810C94DB4DBC01675F7F4F21E04BE82D
:10C0B0005EE0FC01848195810C94DB4D0F931F930E
:10C0C000CF93DF93CDB7DEB72797CDBFDEBF8C010F
:10C0D000FC018481958127E0E9EDF0E2DE01119613
:10C0E00001900D922A95E1F70E94C64CF8019485C3
:10C0F0009F9393859F9392859F9391859F93E1E072
:10C10000F0E0EC0FFD1FE80FF11D80811F928F936F
:10C110008CE29AE09F938F93E0EDF4E581818F9319
:10C1200080818F930E9469E4CDBFDEBF2796CDBF8B
:10C13000DEBFDF91CF911F910F9108950F931F9351
:10C14000CF93DF93EC010C811D810E946E6908176B
:10C150001907C0F48C819D81FC01EE0FFF1FE80FD1
:10C16000F91FEE0FFF1FEE0FFF1FEE0FFF1FE05F27
:10C17000F94E25913491CE01F901DF91CF911F91B4
:10C180000F91199485E1DF91CF911F910F9108953F
:10C190000F931F93CF93DF93EC010C811D810E94BD
:10C1A0006E6908171907C0F48C819D81FC01EE0FA0
:10C1B000FF1FE80FF91FEE0FFF1FEE0FFF1FEE0F1F
:10C1C000FF1FE25FF94E25913491CE01F901DF9115
:10C1D000CF911F910F91199485E1DF91CF911F911C
:10C1E0000F9108950F931F93CF93DF93EC010C8170
:10C1F0001D810E946E6908171907C0F48C819D810A
:10C20000FC01EE0FFF1FE80FF91FEE0FFF1FEE0FEF
:10C21000FF1FEE0FFF1FE45FF94E25913491CE0111
:10C22000F901DF91CF911F910F911994DF91CF9177
:10C230001F910F910895CF93DF93EC018C819D8125
:10C240000E9481698823C9F08C819D81FC01EE0FD9
:10C25000FF1FE80FF91FEE0FFF1FEE0FFF1FEE0F7E
:10C26000FF1FE65FF94EE491E1FF05C0CE01DF91CB
:10C27000CF910C945D8580E001C085E1DF91CF9185
:10C2800008950F931F93CF93DF93EC0181E00E94F9
:10C2900034531C821D8280E090E08E010F5E1F4FA0
:10C2A00047C08C819D819C01220F331FF901E80F4B
:10C2B000F91FEE0FFF1FEE0FFF1FEE0FFF1FE65FD0
:10C2C000F94EE491E0FF2EC0280F391F220F331FD3
:10C2D000220F331F220F331F2C5E394EF901459177
:10C2E00055916591749149875A876B877C87BC010A
:10C2F000660F771F680F791F660F771F660F771F0E
:10C30000660F771F6C5F794E45E050E0C8010E94D0
:10C31000A2E3CE010E949E60CE010E941B612C818F
:10C320003D8101C09C012F5F3F4F2C833D83C9019C
:10C330000E9471698111B5CF0E948EACDF91CF91BF
:10C340001F910F910C9446ACCF93DF93EC012CEA34
:10C3500035EC47E257E369857A858B859C850E9499
:10C36000A9D787FF05C0CE01DF91CF910C94127E33
:10C37000CE010E94416182E08F8340E050E060E89E
:10C380007FE349875A876B877C8780E0DF91CF9175
:10C3900008958091DC339091DD338F3E924111F00E
:10C3A0008AE5089580912434909125348F3E9241FE
:10C3B000B9F78091B22E9091B32E8F3E924181F7C2
:10C3C0008091D4319091D5318F3E924149F780913F
:10C3D000D6319091D7318F3E924111F78091DA3367
:10C3E0009091DB338F3E9241D9F680914F38811185
:10C3F000D7CF0895FC01178283E00895CF93DF9390
:10C40000EC018C819D81FC01EE0FFF1FE80FF91FED
:10C41000EE0FFF1FEE0FFF1FEE0FFF1FEE5EF94E38
:10C42000A591B4916C9170E080E090E00E9449D8B1
:10C4300069877A878B879C8782E08F8380E0DF9192
:10C44000CF910895CF93DF93EC018C819D81FC0106
:10C45000EE0FFF1FE80FF91FEE0FFF1FEE0FFF1F7C
:10C46000EE0FFF1FEE5EF94EA591B4916D917D9197
:10C470008D919C910E9449D869877A878B879C8788
:10C4800082E08F8380E0DF91CF910895CF93DF9397
:10C49000DC0114968D919C911597FC01EE0FFF1F06
:10C4A000E80FF91FEE0FFF1FEE0FFF1FEE0FFF1F2C
:10C4B000EE5EF94EC591D491488159816A817B81A4
:10C4C00019964D935D936D937C931C9783E017961B
:10C4D0008C9380E0DF91CF910895CF93DF93DC01BF
:10C4E00014968D919C911597FC01EE0FFF1FE80F9C
:10C4F000F91FEE0FFF1FEE0FFF1FEE0FFF1FEE5E87
:10C50000F94EC591D491488159816A817B811996F0
:10C510004D935D936D937C931C97FC01EE0FFF1F71
:10C52000E80FF91FEE0FFF1FEE0FFF1FEE0FFF1FAB
:10C53000E55FF94E8591949118968C93189784E055
:10C5400017968C9380E0DF91CF91089583E0089552
:10C550000F931F93CF93DF93EC018C819D81FC019E
:10C56000EE0FFF1FE80FF91FEE0FFF1FEE0FFF1F6B
:10C57000EE0FFF1FEE5EF94E0591149169857A85E5
:10C580008B859C850E941DD8F801608382E08F8393
:10C5900080E0DF91CF911F910F910895CF92DF92AC
:10C5A000EF92FF920F931F93CF93DF93EC01C98417
:10C5B000DA84EB84FC8420E030E040E85FE3C701EC
:10C5C000B6010E94ACD91816DCF08C819D81FC016B
:10C5D000EE0FFF1FE80FF91FEE0FFF1FEE0FFF1FFB
:10C5E000EE0FFF1FEE5EF94E05911491C701B601E3
:10C5F0000E941DD8F801608382E08F8380E001C033
:10C600008BE6DF91CF911F910F91FF90EF90DF901C
:10C61000CF900895CF92DF92EF92FF920F931F93E6
:10C62000CF93DF93EC01C984DA84EB84FC8420E0AF
:10C6300030E040E050E4C701B6010E94ACD91816C2
:10C64000DCF08C819D81FC01EE0FFF1FE80FF91FCC
:10C65000EE0FFF1FEE0FFF1FEE0FFF1FEE5EF94EF6
:10C6600005911491C701B6010E941DD8F80160839D
:10C6700082E08F8380E001C08BE6DF91CF911F9134
:10C680000F91FF90EF90DF90CF900895CF92DF92BF
:10C69000EF92FF920F931F93CF93DF93EC01C98426
:10C6A000DA84EB84FC8420E030E040E450E4C7010D
:10C6B000B6010E94ACD91816DCF08C819D81FC017A
:10C6C000EE0FFF1FE80FF91FEE0FFF1FEE0FFF1F0A
:10C6D000EE0FFF1FEE5EF94E05911491C701B601F2
:10C6E0000E941DD8F801608382E08F8380E001C042
:10C6F0008BE6DF91CF911F910F91FF90EF90DF902C
:10C70000CF9008950F931F93CF93DF93EC018C810B
:10C710009D81FC01EE0FFF1FE80FF91FEE0FFF1FB9
:10C72000EE0FFF1FEE0FFF1FEE5EF94E0591149105
:10C7300069857A858B859C850E941DD8F801608368
:10C7400071838283938382E08F8380E0DF91CF9136
:10C750001F910F910895CF93DF93DC0114968D9173
:10C760009C911597FC01EE0FFF1FE80FF91FEE0FCC
:10C77000FF1FEE0FFF1FEE0FFF1FEE5EF94EC5917C
:10C78000D49119964D915D916D917C911C97488340
:10C7900059836A837B8383E017968C9380E0DF91D3
:10C7A000CF910895CF93DF93DC0114968D919C91E6
:10C7B0001597FC01EE0FFF1FE80FF91FEE0FFF1F8B
:10C7C000EE0FFF1FEE0FFF1FEE5EF94EC591D491E5
:10C7D00019964D915D916D917C911C974883598379
:10C7E0006A837B83FC01EE0FFF1FE80FF91FEE0F3A
:10C7F000FF1FEE0FFF1FEE0FFF1FE55FF94E859144
:10C80000949118968C93189784E017968C9380E0F7
:10C81000DF91CF9108951F93CF93DF93EC01809127
:10C82000DE338823D1F01DE10A80DB81C02D209703
:10C8300011F480E013C08F818F3FD9F3811104C0C0
:10C84000CE010E94C86006C0CE010E949E60CE014B
:10C850000E941B61115041F7ECCF84E6DF91CF912C
:10C860001F910895CF93DF93EC01BC0180E091E22A
:10C870000E94DBE3892B41F0BE0183E091E20E943C
:10C88000DBE321E0892B09F420E0822FDF91CF91B7
:10C8900008950F931F93CF93DF93CDB7DEB72997FA
:10C8A000CDBFDEBF8B0144E050E0BC01CE0101965C
:10C8B0000E94FBE346E050E0B801CE0101960E94E1
:10C8C000EBE30E946E69009709F43FC07981AA8169
:10C8D000BB811C810D8124E036E140E050E0F9018C
:10C8E0006491671327C03196E491E11103C0A1114F
:10C8F00021C029C0EA131EC0F9013296E491E1116A
:10C9000003C0B11117C01FC0EB1314C0F901339657
:10C91000E491E11103C011110DC015C0E1130AC06B
:10C92000F9013496E491E11103C0011103C00BC079
:10C93000E01749F04F5F5F4F285E3F4F4817590798
:10C9400009F0CDCF02C0CA0102C08FEF9FEF299638
:10C95000CDBFDEBFDF91CF911F910F910895CF938F
:10C96000DF93FC012189222371F1EC016196BE0164
:10C9700087E091E20E94DBE3892B39F1BE0180E080
:10C9800091E20E94DBE3892B11F1BE018AE091E282
:10C990000E94DBE3892BD9F0BE018EEE90E20E946B
:10C9A000DBE3892BB1F0BE018DE091E20E94DBE375
:10C9B000892B79F0BE0189EE91E20E94DBE3892B9D
:10C9C00051F485E009C080E007C082E005C083E043
:10C9D00003C084E001C081E0DF91CF910895FC01A4
:10C9E0008FEF878314821582118612861386148630
:10C9F0001086118A1586178A108EA081B181109732
:10CA000011F416820DC017968C911797873029F470
:10CA100016968C918F5F868303C016968C918683C1
:10CA2000CF010895EF92FF920F931F93CF93DF935F
:10CA3000EC010C811D810E946E690817190708F02E
:10CA40006FC00C811D81CE010E94EF640C831D8399
:10CA50007E0181E1E80EF11CB801660F771F600FBF
:10CA6000711F660F771F660F771F660F771F6C5F4A
:10CA7000794EC7010E9483E38E01035F1F4F2C8113
:10CA80003D81B901660F771F620F731F660F771F15
:10CA9000660F771F660F771F60507A4EC8010E949D
:10CAA00083E38D85882311F18C819D81FC01EE0F3C
:10CAB000FF1FE80FF91FEE0FFF1FEE0FFF1FEE0F16
:10CAC000FF1FE65FF94EE491E2FF02C01D8610C031
:10CAD000F80101900020E9F7BF01601B710B605F56
:10CAE0007F4F6C0F7D1FC7010E94E4E38C819D8105
:10CAF000FC01EE0FFF1FE80FF91FEE0FFF1FEE0FF7
:10CB0000FF1FEE0FFF1FE25FF94E25913491CE011A
:10CB1000F901DF91CF911F910F91FF90EF90199440
:10CB2000DF91CF911F910F91FF90EF9008958F9219
:10CB30009F92AF92BF92CF92DF92EF92FF920F93AC
:10CB40001F93CF93DF9300D01F92CDB7DEB76C0158
:10CB50005C0181E1A80EB11C87E0F601878360E0EB
:10CB6000E62E66E1F62E00E010E01DC0B701CE0112
:10CB700001960E9483E3BE016F5F7F4FC5010E9453
:10CB8000DBE3892B59F44601F9E18F0E911CF60184
:10CB9000058F168FC4010E94126564010F5F1F4F3D
:10CBA000F8E1EF0EF11CC8010E9471698111DECF1E
:10CBB0002496CDBFDEBFDF91CF911F910F91FF90E3
:10CBC000EF90DF90CF90BF90AF909F908F9008959F
:10CBD000CF93DF931092D8311092D931ABE9BEE2F6
:10CBE000E4EBFEE291E08FEFA083B18379965B9650
:10CBF000ED93FC935C975D961D921C925E97EF01FE
:10CC00006397988322961882219788832A961882A0
:10CC1000599621E3E43DF20739F71092BD311092A5
:10CC2000BE311092B42E1092B52E1092BA2E87E01B
:10CC30008093BB2E82E790E08093C52E9093C62E02
:10CC40008DEC9EE2DF91CF9108950F931F93CF93C8
:10CC5000DF930E94E865EC018FEE92E18093DC3374
:10CC60009093DD3380932434909325348093B22EB7
:10CC70009093B32E8093D4319093D5318093D63155
:10CC80009093D7318093DA339093DB3381E00E9425
:10CC900034531C821D82CE010E94348520912D3494
:10CCA00030912E3440912F345091303469857A85FB
:10CCB0008B859C850E94A9D7882339F0CE01DF910E
:10CCC000CF911F910F910C9441610E944BAC1C823B
:10CCD0001D8280E090E08E010F5E1F4F2FC06C819F
:10CCE0007D819B01220F331FF901E60FF71FEE0F25
:10CCF000FF1FEE0FFF1FEE0FFF1FE65FF94EE491DF
:10CD0000E0FF17C0620F731F660F771F660F771F54
:10CD1000660F771F6C5F794E45E050E0C8010E94B6
:10CD2000A2E3CE010E943485CE010E949E606C81F8
:10CD30007D816F5F7F4F6C837D83CB010E94716922
:10CD40008111CDCFDF91CF911F910F910C948EACBB
:10CD5000EF92FF920F931F93CF93DF938C0120915B
:10CD6000D8313091D931EB0109900020E9F72197B2
:10CD7000C61BD70BAE01420F531F41305240D8F4AF
:10CD8000F901E652FE4C7F01AE014F5F5F4FCF01CC
:10CD90000E94BCE34091D8315091D9314F5F5F4F31
:10CDA0004C0F5D1F4093D8315093D931F801E78A79
:10CDB000F08E80E001C08DE0DF91CF911F910F9147
:10CDC000FF90EF900895CF93DF932EE1CDECDEE25C
:10CDD0003F813F3F59F00A80DB81C02D209719F435
:10CDE00080E090E010C0215099F7FACFBC0182E5B5
:10CDF00093E20E9449648C839D83019689F3CE015E
:10CE00000E941265CE01DF91CF910895EF92FF92BB
:10CE10000F931F93CF93DF938B012EE1CDECDEE2D6
:10CE20003F813F3F59F00A80DB81C02D209719F4E4
:10CE300080E090E01DC0215099F7FACF7E0121E1FA
:10CE4000E20EF11C45E050E0BC01C7010E94FBE38B
:10CE5000B801CE010E94A8668111EACFB70182E530
:10CE600093E20E9449648C839D8385E08F83CE0189
:10CE7000DF91CF911F910F91FF90EF900895209136
:10CE8000DE33213021F42091FC37213029F4BC011C
:10CE90008EEE90E20C94066780E090E00895909109
:10CEA000DE33913019F4642F0C94B0830C9423C5B5
:10CEB0000F931F93CF93DF93CDB7DEB7C058D1093F
:10CEC000CDBFDEBFFC0161857285838594850E949C
:10CED0001DD88FEF860F863030F081E491E20E94FA
:10CEE0003F678BE62AC06093E23381E08093E333AF
:10CEF000E62FF0E0EE0FFF1FE553FA4E65917491B7
:10CF00004FE450E080E098E30E94A2E39F938F9368
:10CF100082EA94E19F938F938E010F5F1F4F1F93BF
:10CF20000F930E945DE5C8010E943F670F900F902C
:10CF30000F900F900F900F9080E0C058DF4FCDBF43
:10CF4000DEBFDF91CF911F910F910895CF93DF93B3
:10CF5000EC010E9479D4682F70E080E090E00E949C
:10CF600049D869877A878B879C8782E08F8380E0A6
:10CF7000DF91CF9108950F931F93CF93DF93EC012F
:10CF800089E19CE20E94094F882329F009851A85CE
:10CF90008B859C8511C023E333E34BEC51E4698519
:10CFA0007A858B859C850E944EDA8B01AB01BC0192
:10CFB00049875A876B877C872C813D81F901EE0F69
:10CFC000FF1FE20FF31FEE0FFF1FEE0FFF1FEE0F0D
:10CFD000FF1FEE5EF94EA591B491A801BC014D93DF
:10CFE0005D936D937C931397F901EE0FFF1FE20F92
:10CFF000F31FEE0FFF1FEE0FFF1FEE0FFF1FE55F8A
:10D00000F94E85919491888784E08F8380E0DF9149
:10D01000CF911F910F9108956CE975E10C94B9C5FA
:10D0200068E775E10C94B9C56BE375E10C94B9C57B
:10D030006EEE74E10C94B9C56BEC74E10C94B9C557
:10D040001F93CF93DF93EC0110E08881882301F1D7
:10D050000E94E86545E050E0BE018EED9EE20E9430
:10D06000FBE36EED7EE282E593E20E9449648093E9
:10D07000D12E9093D22E8DEC9EE20E94126542E05A
:10D0800063E080E00E944F671F5F26961D31E9F63E
:10D0900084E0DF91CF911F910895CF93DF93CDB7B7
:10D0A000DEB7EC97CDBFDEBF8CE3E8E1F0E2DE0156
:10D0B000119601900D928A95E1F7CE0101960E949A
:10D0C0002068EC96CDBFDEBFDF91CF910895CF935E
:10D0D000DF93CDB7DEB7AA97CDBFDEBF8AE2E4E526
:10D0E000F0E2DE01119601900D928A95E1F7CE01F2
:10D0F00001960E942068AA96CDBFDEBFDF91CF9136
:10D100000895CF93DF93CDB7DEB76E97CDBFDEBF67
:10D110008EE1EEE7F0E2DE01119601900D928A9524
:10D12000E1F7CE0101960E9420686E96CDBFDEBF6A
:10D13000DF91CF910895CF93DF93EC0143E759E757
:10D1400063E770E0498B5A8B6B8B7C8B0E949765F1
:10D1500042E063E080E00E944F67CE010E94816858
:10D16000CE010E94676820E731E340E0298B3A8BCB
:10D170004B8BCE010E94976542E063E080E00E9405
:10D180004F67CE01DF91CF910C944D68CF92DF9223
:10D19000EF92FF92FC01C184D284E384F48420E006
:10D1A00030E040E85FE3C701B6010E94ACD9181631
:10D1B000FCF0C701B6010E941DD86093DF33C701A0
:10D1C000B6019F772CEA35EC47E257E30E94ACD9D1
:10D1D00018163CF460E470E080E00E9446CB80E0EA
:10D1E00008C060E870E080E00E9446CB80E001C0AB
:10D1F0008BE6FF90EF90DF90CF900895CF92DF9273
:10D20000EF92FF92FC01C184D284E384F48420E095
:10D2100030E040E050E4C701B6010E94ACD91816D6
:10D22000FCF0C701B6010E941DD86093E133C7012D
:10D23000B6019F772CEA35EC47E257E30E94ACD960
:10D2400018163CF464E070E080E00E9446CB80E079
:10D2500008C068E070E080E00E9446CB80E001C03A
:10D260008BE6FF90EF90DF90CF900895CF92DF9202
:10D27000EF92FF92FC01C184D284E384F48420E025
:10D2800030E040E85FE3C701B6010E94ACD9181650
:10D29000FCF0C701B6010E941DD86093E033C701BE
:10D2A000B6019F772CEA35EC47E257E30E94ACD9F0
:10D2B00018163CF460E170E080E00E9446CB80E00C
:10D2C00008C060E270E080E00E9446CB80E001C0D0
:10D2D0008BE6FF90EF90DF90CF9008958CE891E07F
:10D2E000089521E08334914008F020E0822F0895D2
:10D2F0009C012F55314081E02932310508F080E052
:10D30000089521E08036914008F020E0822F0895B2
:10D31000CF92DF92EF92FF92CF93DF93EC01C9841B
:10D32000DA84EB84FC84A7019601C701B6010E9450
:10D330006FDB81113CC0E894F7F82FEF3FEF4FE728
:10D340005FE7C701B6010E946FDB81110AC02FEFB2
:10D350003FEF4FE75FE7C701B6010E94A9D7181654
:10D3600034F18C819D81FC01EE0FFF1FE80FF91F46
:10D37000EE0FFF1FEE0FFF1FEE0FFF1FE65FF94ED0
:10D38000E491E3FF14C089E19CE20E94094F8111FE
:10D390000EC025E832E441E25DE369857A858B853C
:10D3A0009C850E944EDA69877A878B879C87DF91FC
:10D3B000CF91FF90EF90DF90CF9008958091E3336D
:10D3C000882349F01092E3336091E23380E00E94B9
:10D3D0004ECB80E0089583E00895FF920F931F9352
:10D3E000CF93DF931F921F92CDB7DEB7F82EE6E200
:10D3F000F4E322EA33E0DF01C9011D920197E9F766
:10D400002FEE32E1208331832093C6373093C73724
:10D4100005E81BE02CED33E400932D3410932E34FB
:10D4200020932F34309330340CEE11E528E73FE39E
:10D4300000933134109332342093333430933434A6
:10D4400000E010E020E83FE30093353410933634D9
:10D45000209337343093383483E0809328348F2DF1
:10D460004A8369830E945ECB6981862F0E9469CBC3
:10D470004A81842F0E9474CBF0923F34F0923D3465
:10D480000F900F90DF91CF911F910F91FF90089512
:10D49000C3E6D4E310E60E94D07C8230E1F30E9420
:10D4A000D77C8230C1F30E94E84E863009F052C129
:10D4B0000E9423CAC0904A34D0904B34E0904C3440
:10D4C000F0904D34C616D706E806F90620F70E94FC
:10D4D00023CA6C597F4F8F4F9F4F60934A3470938C
:10D4E0004B3480934C3490934D340E94467CD3CF80
:10D4F0000E944EC0882329F08CEC0E942053823079
:10D5000051F20E940D5A823031F20E94D3A1823032
:10D5100011F20E94C9618093503881112EC0809110
:10D520002634909127348F3E924109F019C18091A1
:10D53000C6379091C7378F3E924109F011C116C18D
:10D540000E94098680935038811117C00E94D8B676
:10D5500080935038811111C00E94AE74809350386E
:10D5600081110BC00E9464CA80935038811105C09C
:10D570000E9497B7823031F48ECF0E9420538230C0
:10D58000B9F789CF0E9440AE823009F484CF0E945F
:10D59000ACAF823009F47FCF0E9473B0823009F4BF
:10D5A0007ACF0E945390823009F475CF0E94E36FC6
:10D5B000823009F470CF0E94A272823009F46BCFDE
:10D5C0000E948974823009F466CF0E94B75082307D
:10D5D00009F461CF0E94BE86843008F0D1C05BCFD1
:10D5E0004FEF50E063E674E380913D340E94FCCA43
:10D5F000811139C0C0936134D0936234FE0101902F
:10D600000020E9F7E356F443E0934134F0934234C9
:10D6100043E650E063E674E382E697E30E94FBE3AF
:10D620008091633490E00E947BE385329105F1F1B3
:10D6300054F481329105B9F18432910509F447C05F
:10D64000892BD1F157C08834910509F440C01CF4EE
:10D65000CF97E9F14FC08B37910509F443C08E375E
:10D66000910539F147C0883009F015CF8091DE333C
:10D67000811111C080E29BE39F938F938091D154DD
:10D680008F938091D0548F930E9469E40F900F90F4
:10D690000F900F9003C088E00E94D8AB80913F3478
:10D6A00080933D34F8CE0E94B459F5CE0E94B8590B
:10D6B000F2CE0E94BC59EFCE8091DE33813009F466
:10D6C000EACE62E677E380E00E94BBC2E4CE10922D
:10D6D000DE3383E694E30E947BC162E677E30E9437
:10D6E000BBC2D9CE81E08093DE3383E694E30E940F
:10D6F000687ED1CE8091DE33813019F547EF50E05E
:10D7000063E674E382E695E30E94FBE382E695E339
:10D710009F938F9381E791E29F938F9383E694E3A6
:10D720009F938F930E9434E580916134909162348D
:10D730000E94687E0F900F900F900F900F900F90A7
:10D74000AACE83E694E30E94E37462E677E30E9444
:10D75000BBC2A1CE0E94E84E823009F4D2CEC8CE20
:10D760001093503880E60E94205309CF1092503811
:10D770000E94E55280935038882309F4E1CEFDCE13
:10D780008091C7289091C8280E94EDD2682F70E040
:10D7900080E090E00E944BD823E333E34BE451E474
:10D7A0000E94ACD987FF77CE0E94DE69823009F0F3
:10D7B00017CF71CE80933D34089580933E34089501
:10D7C000CF93C82F80919523882379F040E050E0D3
:10D7D000BA018C2F0E943154EC2FFF27E7FDF09502
:10D7E000E251F44D81E080830AC06C2F87E291E51D
:10D7F0000E942E50AB01BC018C2F0E9431544091ED
:10D80000BC235091BD236091BE237091BF238C2F08
:10D810000E947A5D89EA9DE68093962390939723F0
:10D8200082E0CF910895CF92DF92EF92FF920F9313
:10D830001F93CF93DF93CDB7DEB7E097CDBFDEBFA9
:10D8400098E17E01A9E1EA0EF11CF701A92F1192DE
:10D85000AA95E9F7FE0131966F0111929A95E9F7C1
:10D86000F60194E08902E00DF11D1124408F518FE3
:10D87000628F738F80E090E0A0E8BFE380839183A4
:10D88000A283B3830093562C1093572C2093582CCB
:10D890003093592C0E9441870E94BC59B601C701A0
:10D8A0000E94865780935038811101C082E0E09633
:10D8B000CDBFDEBFDF91CF911F910F91FF90EF9011
:10D8C000DF90CF9008950F931F93E0918F23FF2750
:10D8D000E7FDF095ED53F64D9381913099F4009169
:10D8E000A0231091A1232091A2233091A323409142
:10D8F000A8235091A9236091AA237091AB230E9481
:10D90000136C1DC0E0919023FF27E7FDF095ED53C8
:10D91000F64D9381913099F40091A0231091A123A9
:10D920002091A2233091A3234091A8235091A923B1
:10D930006091AA237091AB2370580E94136C89EAFE
:10D940009CE6809396239093972382E01F910F91FA
:10D9500008950F931F93CF93C82F85E3C802F0015A
:10D960001124E154F54D40815181628173818C2FE6
:10D970000E947A5D0091A0231091A1232091A223FF
:10D980003091A32340919C2350919D2360919E232D
:10D9900070919F238C2F0E94136C88E39DE68093E7
:10D9A00096239093972382E0CF911F910F91089532
:10D9B0000F931F930091A0231091A1232091A223E4
:10D9C0003091A3234091AC235091AD236091AE23BD
:10D9D0007091AF230E94136C80EE9BE68093962398
:10D9E0009093972382E01F910F9108950E944187A1
:10D9F0008091B5230E949A538091B4230E9434539E
:10DA00008091B6230E9438538091B7230E947257A9
:10DA10008091B8239091B923A091BA23B091BB23F0
:10DA20008093562C9093572CA093582CB093592C3C
:10DA300064E089E19CE20E94264F0E94695A10929C
:10DA4000EA2B80E00895CF93C82F4091BC235091DA
:10DA5000BD236091BE237091BF230E947A5D8C2FFD
:10DA60000E94F66C80E00E940EAE80EFCF91089588
:10DA70000F931F93E0918F23FF27E7FDF095ED5360
:10DA8000F64D9381913039F083E29DE680939623A1
:10DA90009093972318C00091A4231091A52320915F
:10DAA000A6233091A7234091A8235091A9236091E8
:10DAB000AA237091AB230E94136C88ED9CE680939F
:10DAC00096239093972382E01F910F910895FF92E0
:10DAD0000F931F93CF93DF93CDB7DEB7C058D10913
:10DAE000CDBFDEBFF82E0E94E8658EEFF81205C0AC
:10DAF0008EE791E20E943F6719C08F2D0E94FE5A67
:10DB00001F928F9325E33BE33F932F938E010F5F8B
:10DB10001F4F1F930F930E945DE5C8010E943F674E
:10DB20000F900F900F900F900F900F9042E062E0D7
:10DB300080EF0E944F678F2D0E94F66C80EFC058D7
:10DB4000DF4FCDBFDEBFDF91CF911F910F91FF90CF
:10DB500008954F925F926F927F929F92AF92BF9281
:10DB6000CF92DF92EF92FF920F931F93CF93DF93A9
:10DB70008F3F09F045C02CEA35EC47E257E360914E
:10DB80004F2D7091502D8091512D9091522D0E94CA
:10DB9000ACD918160CF469C12CEA35EC47E257E30E
:10DBA0006091472D7091482D8091492D90914A2D7B
:10DBB0000E94ACD918160CF45DC12CEA35EC47E292
:10DBC00057E360914B2D70914C2D80914D2D90918C
:10DBD0004E2D0E94ACD918160CF455C12CEA35EC28
:10DBE00047E257E36091532D7091542D8091552D4C
:10DBF0009091562D0E94ACD918160CF43FC171C1FA
:10DC00008230A1F52CEA35EC47E257E36091472DCD
:10DC10007091482D8091492D90914A2D0E94ACD948
:10DC200018160CF427C12CEA35EC47E257E3609153
:10DC30004B2D70914C2D80914D2D90914E2D0E9429
:10DC4000ACD918160CF41FC12CEA35EC47E257E3A7
:10DC50006091532D7091542D8091552D9091562D9A
:10DC60000E94ACD918160CF409C131C18823D9F22D
:10DC7000813051F32CC17E018DEEE80EF11CF701CD
:10DC800080819181A281B381BC01CD019F772CEA73
:10DC900035EC47E257E30E94A9D787FD46C06E01E5
:10DCA000F1EFCF0ED11CF60140805180628073806D
:10DCB00020E030E0A901C301B2010E94A9D787FD8D
:10DCC00034C0FE01EF52FF4F2081318142815381E8
:10DCD000349760817181828193810E943AD69B0141
:10DCE000AC015F77C301B2010E943BD62B013C011E
:10DCF0009F772CEA35EC47E257E30E94A9D787FDCE
:10DD000014C0AB2CAA0C8A2D0E9448C080938D238E
:10DD1000992493949A0C892D0E9448C080938E2355
:10DD200020918D23822780FD02C08B2DDBC0B09215
:10DD30008C23F80180819181A281B381BF77809388
:10DD4000A0239093A123A093A223B093A323F70130
:10DD500040815181628173817F774093A4235093E6
:10DD6000A5236093A6237093A72320FF2DC0A09224
:10DD70008F239092902377FA709477F87094409262
:10DD80009C2350929D2360929E2370929F23F601C4
:10DD900080819181A281B3818093A8239093A9234C
:10DDA000A093AA23B093AB23CB50DF4F88819981F6
:10DDB000AA81BB818093AC239093AD23A093AE2323
:10DDC000B093AF238A2D2AC090928F23A0929023E4
:10DDD00040929C2350929D2360929E2370929F2399
:10DDE000F60180819181A281B381B0588093A823EC
:10DDF0009093A923A093AA23B093AB23CB50DF4FDA
:10DE000088819981AA81BB81B0588093AC2390937B
:10DE1000AD23A093AE23B093AF23892D0E9448C0B9
:10DE20008D7F813039F089EA9DE680939623909327
:10DE3000972369C0809190230E9448C0811103C03C
:10DE40008FEF809390238B2D0E946F5D6093BC2396
:10DE50007093BD238093BE239093BF2383E69CE6FB
:10DE600080939623909397234EC082E090E032E017
:10DE7000B32E0DC080E090E0B12C09C083E090E0AB
:10DE800023E0B22E04C081E090E0BB24B394FC01F7
:10DE9000E251F44D108225E3289FE001299FD00D27
:10DEA0001124CA51D64D8E0107511F4FF8018081B0
:10DEB0009181A281B381BC01CD019F772CEA35EC21
:10DEC00047E257E30E94A9D787FFD5CE2ECF81E046
:10DED0008093ED2B86EF9CE6809396239093972377
:10DEE00012C08EEFDF91CF911F910F91FF90EF90B5
:10DEF000DF90CF90BF90AF909F907F906F905F909A
:10DF00004F900C94676D82E0DF91CF911F910F913C
:10DF1000FF90EF90DF90CF90BF90AF909F907F9059
:10DF20006F905F904F900895CF93DF93C7E1DCE24D
:10DF3000888199810E94094F8093B42388819981B7
:10DF40000E94044F8093B523888199810E94134FCA
:10DF50008093B623888199810E94184F8093B723BC
:10DF6000888199810E941F4F6093B8237093B923D1
:10DF70008093BA239093BB2381E00E94345381E0C5
:10DF80000E94385380E00E949A5381E00E947257A9
:10DF900081E0809395238FEF80938C2389EA9DE61F
:10DFA000809396239093972383E08093EA2B10929B
:10DFB000ED2B80E0DF91CF9108950E94946F109235
:10DFC000952380E008958091EA2B833059F40E94D4
:10DFD0001D4F813049F0E0919623F0919723809175
:10DFE0008C23199483E0089582E008958EEF9FE6D4
:10DFF0008093D1239093D22382E008952F923F9271
:10E000004F925F926F927F928F929F92AF92BF9248
:10E01000CF92DF92EF92FF920F931F93CF93DF93F4
:10E02000CDB7DEB7CA54D109CDBFDEBF98E19E019E
:10E03000275E3F4F29AB3AABD901E92F1D92EA95F4
:10E04000E9F7285131091901D9011D929A95E9F78B
:10E0500024E08202F00111242B96EEAFFFAF2B9744
:10E06000E20DF31D80E090E0A0E8BFE380839183A0
:10E07000A283B383C090C923D090CA23E090CB235E
:10E08000F090CC234090C5235090C6236090C723C6
:10E090007090C8238090C1239090C223A090C32386
:10E0A000B090C423A5019401C301B2010E94A9D775
:10E0B00018165CF080E090E0A0E8BFE329968CAFF2
:10E0C0009DAFAEAFBFAF29970AC080E090E0A0E857
:10E0D000BFEB29968CAF9DAFAEAFBFAF2997A30121
:10E0E0009201C501B4010E943AD60E9418D89B0142
:10E0F00077FF04C022273327261B370BB901882757
:10E1000077FD8095982F0E944BD825966CAF7DAFF8
:10E110008EAF9FAF2597C092562CD092572CE0928D
:10E12000582CF092592C0E9441870E94BC5920E043
:10E1300030E040E050E425966CAD7DAD8EAD9FADF6
:10E1400025970E94ACD918166CF08091CD23909140
:10E15000CE23A091CF23B091D0238BAF9CAFADAF96
:10E16000BEAFDBC02AE037ED43E25CE325966CAD41
:10E170007DAD8EAD9FAD25970E94ACD918162CF7BA
:10E1800009E110E08AE0882E87ED982E83E2A82E20
:10E190008CE3B82E412C512C32012B96AEADBFAD85
:10E1A0002B97A20DB31D58962196AEAFBFAF219706
:10E1B0004BAA5CAA6DAA7EAA8FAA98AEA9AEBAAEE7
:10E1C00029962CAD3DAD4EAD5FAD29976FA978ADC9
:10E1D00089AD9AAD0E944EDA9B01AC016091C523D6
:10E1E0007091C6238091C7239091C8230E943BD68B
:10E1F0002196EEADFFAD2197608371838283938377
:10E20000C092562CD092572CE092582CF092592C58
:10E21000B101CE0149960E948657809350388111F2
:10E22000AAC020E030E040E85FE36BA97CA98DA99B
:10E230009EA90E943BD66BAB7CAB8DAB9EAB20E026
:10E2400030E048EC51E40E94B0D79B01AC0160E0A3
:10E2500070E080E291E40E94B1DA2B013C018091F0
:10E26000CD239091CE23A091CF23B091D0238BAF1B
:10E270009CAFADAFBEAFC090C923D090CA23E09091
:10E28000CB23F090CC23A7019601BC01CD010E94C5
:10E290003AD64B015C0120E030E040E251E4C3019A
:10E2A000B2010E94B0D79B01AC01C501B4010E942C
:10E2B0004EDA9B01AC01C701B6010E943BD66B014F
:10E2C0007C012BA93CA94DA95EA9CA01B9010E94F4
:10E2D0003BD620E030E048EC51E40E94B0D79B01EF
:10E2E000AC016FA978AD89AD9AAD0E943BD66FABFA
:10E2F00078AF89AF9AAF9B01AC0125966CAD7DAD2F
:10E300008EAD9FAD25970E94ACD9181634F40150FC
:10E3100011090115110509F053CF8BAD9CADADADC1
:10E32000BEAD8093562C9093572CA093582CB0934D
:10E33000592C2B96EEADFFAD2B97E20DF31D80917E
:10E34000C1239091C223A091C323B091C423808F95
:10E35000918FA28FB38FB101CE0149960E9486574B
:10E3600080935038811107C082ED91E78093D123CB
:10E370009093D22382E0C65BDF4FCDBFDEBFDF913B
:10E38000CF911F910F91FF90EF90DF90CF90BF90B2
:10E39000AF909F908F907F906F905F904F903F9045
:10E3A0002F900895CF93DF931F92CDB7DEB7898367
:10E3B0000E9441874091DB235091DC236091DD2353
:10E3C0007091DE2389810E947A5D8091D8230E941A
:10E3D0009A538091D7230E9434538091D9230E946D
:10E3E00038538091DA230E9472578091D323909101
:10E3F000D423A091D523B091D6238093562C90930B
:10E40000572CA093582CB093592C64E089E19CE2DE
:10E410000E94264F0E94695A1092EA2B8AEA91E2E2
:10E420000E9407E580E00F90DF91CF9108950F9350
:10E430001F93CF93C82F07E11CE2F80180819181DF
:10E440000E94094F8093D723F801808191810E9417
:10E45000044F8093D823F801808191810E94134F4B
:10E460008093D923F801808191810E94184F809375
:10E47000DA23F801808191810E941F4F6093D3239A
:10E480007093D4238093D5239093D6238C2F0E940E
:10E490006F5D6093DB237093DC238093DD23909387
:10E4A000DE2381E00E94345380E00E94385380E0F4
:10E4B0000E949A5381E00E94725740E050E060E26F
:10E4C00071E44093C9235093CA236093CB23709384
:10E4D000CC2385E3C89FF0011124E155F54D40811F
:10E4E0005181628173814093CD235093CE236093F9
:10E4F000CF237093D0236C2F87E291E50E941B50AD
:10E500006093C5237093C6238093C7239093C82339
:10E510000E94475E6093C1237093C2238093C323FC
:10E520009093C423C093C02386EF9FE68093D123AA
:10E530009093D22384E08093EA2B80E0CF911F91C7
:10E540000F9108958091EA2B843059F40E941D4F59
:10E55000813049F0E091D123F091D2238091C02302
:10E56000199483E0089582E00895E091E123F0E0BA
:10E57000ED53F64D8381882341F080ED92E780933F
:10E58000DF239093E02382E008956EE274E286E157
:10E5900094E20E94865780935038882371F308953F
:10E5A0001F93CF93DF93E091E123F0E0ED53F64D1D
:10E5B00081E09381913009F080E08093F42BC5EFE6
:10E5C000DBE210E0612F87E291E50E942E50AB0163
:10E5D000BC01812F0E943154612F8091172C9091A2
:10E5E000182C0E941B5069937993899399931F5F0C
:10E5F000163041F784EB91E20E94687E8EE393E748
:10E600008093DF239093E02382E0DF91CF911F91ED
:10E6100008951F93CF93DF930E9441878091E22357
:10E620008093C329E091E123F0E08091E323ED534F
:10E63000F64D83870E9465C0C6EED3E210E0499193
:10E64000599169917991812F0E947A5D1F5F1630EF
:10E65000B1F78091E5230E949A538091E4230E94B0
:10E66000385364E089E19CE20E94264F0E94695A77
:10E670001092EA2BDF91CF911F9108950E940973A8
:10E6800080E008950F931F93CF93DF93CDB7DEB74C
:10E69000C058D109CDBFDEBF182F0E94E8651E3FCC
:10E6A00029F481EC91E20E943F6719C0812F0E94FA
:10E6B000FE5A1F928F9383E69BE39F938F938E0165
:10E6C0000F5F1F4F1F930F930E945DE5C8010E94CB
:10E6D0003F670F900F900F900F900F900F9042E0B8
:10E6E00062E08AEF0E944F670E9409738AEFC05868
:10E6F000DF4FCDBFDEBFDF91CF911F910F91089506
:10E70000FF920F931F93CF93DF931092F42B82E02D
:10E710008093EA2B06EE13E2CFEBDAE2F12C8F2D99
:10E720000E946F5DF80161937193819391938F01C2
:10E73000488159816A817B818F2D0E947A5D6F2D7E
:10E740008091172C9091182C0E941B50F801648B1B
:10E75000758B868B978BF394E596F6E0FF12DFCFEF
:10E7600066E174E28EEF93E20E94CEC62AE43CE0BA
:10E7700042E85EE30E94A9D787FF03C08EEF0E94A4
:10E780004273CAE0D4E213E0699179918991999139
:10E790002C893D894E895F890E943AD69F772CEA61
:10E7A00035EC47E257E30E94ACD918161CF4812FD0
:10E7B0000E9442731F5F163039F784E08093E12393
:10E7C0008091D2298093E32381E08093D2298091A4
:10E7D000C3298093E2231092C3290E9465C08091CF
:10E7E000172C9091182C0E94044F8093E523809160
:10E7F000172C9091182C0E94134F8093E42380E0F3
:10E800000E94385380E00E949A5380E00E9454B2E4
:10E8100085EB92E78093DF239093E02382E0DF9102
:10E82000CF911F910F91FF9008950F931F93CF9356
:10E83000DF938C01EB018091622C882399F0809109
:10E84000562C9091572CA091582CB091592CBC016A
:10E85000CD019F772CEA35EC47E257E30E94A9D718
:10E8600087FD4FC088819981AA81BB81BC01CD0100
:10E870009F772CEA35EC47E257E30E94ACD9181693
:10E88000F4F48C819D81AE81BF81BC01CD019F7765
:10E890002CEA35EC47E257E30E94ACD918167CF419
:10E8A00088859985AA85BB85BC01CD019F772CEA17
:10E8B00035EC47E257E30E94ACD9181624F188E101
:10E8C000F801A6E1B4E201900D928A95E1F788E1A2
:10E8D000FE01AEE2B4E201900D928A95E1F788E183
:10E8E000E5EFFBE2DF011D928A95E9F782E0809374
:10E8F000F42B80E893E78093DF239093E02380E07C
:10E9000003C08EE801C086E8DF91CF911F910F917F
:10E9100008958091EA2B823021F08091F42B82308F
:10E9200049F40E941D4F813039F0E091DF23F091CE
:10E93000E023199483E0089582E00895E8ECF7E37A
:10E9400080E2DF011D928A95E9F78FEE92E18093D4
:10E95000E6379093E7378083918308958091E63777
:10E960009091E7378F3E924111F08CE508958091A8
:10E97000C8379091C9378F3E9241B9F780E008952A
:10E98000CF93DF93C82FCB01BA010E94FDDA27E0B5
:10E99000C29FE0011124C853D84C0E9418D86D833F
:10E9A0007E838F839887DF91CF91089597E0899F29
:10E9B000F0011124E853F84C6581768187819085B8
:10E9C0000E944BD808952F923F924F925F926F9280
:10E9D0007F928F929F92AF92BF92CF92DF92EF92EF
:10E9E000FF920F931F93CF93DF93CDB7DEB7279797
:10E9F000CDBFDEBF8C011B828091E92B823009F4F0
:10EA0000A6C6D801BC90B110CFC680E06E01B3E0BD
:10EA1000CB0ED11C3DC0F6018081811108C0B72CFE
:10EA2000D7011C926E01B3E0CB0ED11CBAC688325E
:10EA300039F4B72CF7011082FFEFCF1ADF0AB1C605
:10EA40008B33B9F3A82EB12CC5010E9457E3892B53
:10EA500039F4B5018BEE91E20E94D0E3892B51F09D
:10EA600047018FEF881A980AC5010E947BE3D701FE
:10EA70008C937401BFEFCB1ADB0AF70180818111FF
:10EA8000CACFB72CD8018C916E01B3E0CB0ED11C4C
:10EA9000F8011CC08E32E1F090E0C0970A9790F028
:10EAA0008181803391F4828190E0C0970A9760F46D
:10EAB000DF01119611968C9111978D938111FACFE8
:10EAC000808104C0818101C080E331968111E2CF51
:10EAD000F601A080A11007C036C0D6011196AC90F7
:10EAE000BFEFCB1ADB0A76018A2C912CC4010E945D
:10EAF0006BE3892B91F7C4010E9473E38D36910576
:10EB0000A1F4F601818190E00E9473E383379105BF
:10EB100061F4D60112968C9190E00E9473E38736DF
:10EB2000910519F4F601339602C0FE013396AA202E
:10EB300061F08A2DD701893209F41C9211968C91CB
:10EB40008111F9CF02C0FE013396BFE2BB1609F472
:10EB500000C68081882319F0CF010E94AF5980E15F
:10EB6000E8EEF7E3DF011D928A95E9F78AE5E0E434
:10EB7000FDE2DF01982F1D929A95E9F7E6EEFCE29F
:10EB8000DF011D928A95E9F789E19CE20E94014F1D
:10EB90008093E72C812C912C80E8A82E8FE3B82E4F
:10EBA0005524539492E0492E24E0322EBDC3C70170
:10EBB000B6010E941DD8862F90E08F35910508F090
:10EBC000CCC5FC01EC50FF4F0C94F4DF1092E72C05
:10EBD0005092412D8091E9378F5F8093E937A4C32C
:10EBE0005092E72C5092412D8091E9378F5F8093AE
:10EBF000E9379AC34092E72C5092412D8091E93732
:10EC00008F5F8093E93790C383E08093E72C509225
:10EC1000412D8091E9378F5F8093E93785C38DE07F
:10EC20008093E62C5092402D7FC388E0B2C01092B2
:10EC3000162D5092702D8091EA378F5F8093EA37BE
:10EC400073C35092162D5092702D8091EA378F5FCA
:10EC50008093EA3769C34092162D5092702D8091AF
:10EC6000EA378F5F8093EA375FC31092172D509277
:10EC7000712D8091ED378F5F8093ED3755C35092A2
:10EC8000172D5092712D8091ED378F5F8093ED3766
:10EC90004BC3C701B6010E9468DB6C837D838E8302
:10ECA0009F8320E030E040E251E4C701B6010E94BA
:10ECB0004EDA6B017C0120E030E040E251E46C81EF
:10ECC0007D818E819F810E944EDA9B01AC01C7013C
:10ECD000B6010E943AD60E941DD8623001F128F494
:10ECE000662341F0613089F038C56330E9F0643063
:10ECF00001F133C5B5E0B093E62C5092402D8091E0
:10ED0000E8378F5F8093E8370FC33092E62C60932B
:10ED1000402D8091E8378F5F8093E83705C350928C
:10ED2000E62C5092402D00C34092E62C5092402D8C
:10ED3000FBC283E08093E62C5092402DF5C2C701C0
:10ED4000B6010E9468DB6C837D838E839F8320E005
:10ED500030E040E251E4C701B6010E944EDA6B0197
:10ED60007C0120E030E040E251E46C817D818E81C5
:10ED70009F810E944EDA9B01AC01C701B6010E943F
:10ED80003AD60E941DD8662319F0613061F0E5C4BF
:10ED900087E08093E62C5092402D8091E8378F5F7A
:10EDA0008093E837C1C2E6E0E093E62C6093402D03
:10EDB0008091E8378F5F8093E837B6C2C701B6010C
:10EDC0000E9468DB6C837D838E839F8320E030E02C
:10EDD00040E251E4C701B6010E944EDA6B017C01AA
:10EDE00020E030E040E251E46C817D818E819F81A2
:10EDF0000E944EDA9B01AC01C701B6010E943AD6CF
:10EE00000E941DD8623009F0A8C48EE08093E62CE1
:10EE10005092402D89C25092192D5092732D84C268
:10EE20005092182D5092722D8091F1378F5F809300
:10EE3000F1377AC24092182D5092722D8091F1379D
:10EE40008F5F8093F13770C283E016C03092182D27
:10EE50005092722D8091F1378F5F8093F13764C2A9
:10EE6000F5E0F093182D5092722D8091F1378F5F5D
:10EE70008093F13759C286E08093182D5092722DFD
:10EE80008091F1378F5F8093F1374EC2C701B60191
:10EE90000E9468DB6C837D838E839F8320E030E05B
:10EEA00040E251E4C701B6010E944EDA6B017C01D9
:10EEB00020E030E040E251E46C817D818E819F81D1
:10EEC0000E944EDA9B01AC01C701B6010E943AD6FE
:10EED0000E941DD8662319F0613059F03EC410928B
:10EEE0001B2D5092752D8091F2378F5F8093F237F2
:10EEF0001BC260931B2D6093752D8091F2378F5F3D
:10EF00008093F23711C240921B2D5092752D809143
:10EF1000F2378F5F8093F23707C23092E72C50921E
:10EF2000412D8091E9378F5F8093E937FDC11092C1
:10EF30001C2D5092762D8091EB378F5F8093EB37AD
:10EF4000F3C150921C2D5092762D8091EB378F5F3C
:10EF50008093EB37E9C1C701B6010E9468DB6C837F
:10EF60007D838E839F8320E030E040E251E4C7013F
:10EF7000B6010E944EDA6B017C0120E030E040E2F5
:10EF800051E46C817D818E819F810E944EDA9B01CC
:10EF9000AC01C701B6010E943AD60E941DD861306B
:10EFA00089F028F06230A1F06330C1F0D6C399E057
:10EFB0009093E62C5092402D8091E8378F5F80939C
:10EFC000E837B2C1AAE0A093E62C6093402DACC113
:10EFD000BBE0B093E62C5092402DA6C1ECE0E0934C
:10EFE000E62C5092402DA0C11092112D50926B2D05
:10EFF0008091EC378F5F8093EC3796C15092112D42
:10F0000050926B2D8091EC378F5F8093EC378CC1E1
:10F01000C701B6010E941DD8862F90E08D3391055F
:10F0200008F099C3FC01ED5AFE4F0C94F4DF1092E6
:10F03000E82C5092422D8091F3378F5F8093F33705
:10F0400073C15092E82C5092422D8091F3378F5F1C
:10F050008093F33769C15092222D50927C2D80917C
:10F06000F5378F5F8093F5375FC14092222D509224
:10F070007C2D8091F5378F5F8093F53755C11092C5
:10F08000222D50927C2D8091F5378F5F8093F5373C
:10F090004BC150921F2D5092792D46C15092202D78
:10F0A00050927A2D8091F6378F5F8093F6373CC16E
:10F0B0005092212D50927B2D8091F6378F5F809357
:10F0C000F63732C11092212D50927B2D8091F63768
:10F0D0008F5F8093F63728C15092142D50926E2D79
:10F0E0008091F7378F5F8093F7371EC11092142DF0
:10F0F00050926E2D8091F7378F5F8093F73714C150
:10F100005092122D50926C2D8091F7378F5F809323
:10F11000F7370AC150922B2D5092852D8091F737E9
:10F120008F5F8093F73700C1C701B6010E9468DB8B
:10F130000E941DD860931E2D5092782DF5C0C0926C
:10F14000052DD092062DE092072DF092082D809289
:10F150005F2D9092602DA092612DB092622DE4C03F
:10F16000C0922C2DD0922D2DE0922E2DF0922F2D8D
:10F170008092862D9092872DA092882DB092892D15
:10F18000D3C0C092232DD092242DE092252DF09251
:10F19000262D80927D2D90927E2DA0927F2DB09273
:10F1A000802DC2C0C092ED2CD092EE2CE092EF2CBC
:10F1B000F092F02C8092472D9092482DA092492DEC
:10F1C000B0924A2DB1C0C092F12CD092F22CE092B4
:10F1D000F32CF092F42C80924B2D90924C2DA09217
:10F1E0004D2DB0924E2DA0C0C092F52CD092F62C91
:10F1F000E092F72CF092F82C80924F2D9092502DA7
:10F20000A092512DB092522D8FC0C092F92CD09265
:10F21000FA2CE092FB2CF092FC2C8092532D9092D1
:10F22000542DA092552DB092562D7EC0C092FD2C2B
:10F23000D092FE2CE092FF2CF092002D8092572D60
:10F240009092582DA092592DB0925A2D6DC0C09217
:10F25000012DD092022DE092032DF092042D809288
:10F260005B2D90925C2DA0925D2DB0925E2D5CC0C6
:10F27000C092342DD092352DE092362DF092372D5C
:10F2800080928E2D90928F2DA092902DB092912DE4
:10F290004BC0C092382DD092392DE0923A2DF09289
:10F2A0003B2D8092922D9092932DA092942DB0920E
:10F2B000952D3AC0C0923C2DD0923D2DE0923E2D2E
:10F2C000F0923F2D8092962D9092972DA092982D9E
:10F2D000B092992D29C0C092302DD092312DE0925C
:10F2E000322DF092332D80928A2D90928B2DA09208
:10F2F0008C2DB0928D2D18C0C701B6010E941DD86B
:10F300006093E92C7093EA2C8093EB2C9093EC2C77
:10F3100081E090E0A0E0B0E08093432D9093442DF5
:10F32000A093452DB093462DD8012C90222009F4AE
:10F3300016C2822D90E00E9462E3892B09F421C25B
:10F340003801BFEF6B1A7B0AF8018181803349F4E1
:10F350008281883531F40E5F1F4FC12CD12C76018C
:10F3600014C2BE016F5F7F4FC3010E94FADF6B01C1
:10F370007C0109811A816016710609F006C203C278
:10F380008091112D0E947257182F01C010E06091DA
:10F390005F2D7091602D8091612D9091622D0E9462
:10F3A0001DD8662359F06091052D7091062D80912E
:10F3B000072D9091082D0E944157182F6091632DC1
:10F3C0007091642D8091652D9091662D0E941DD8BD
:10F3D000662371F06091092D70910A2D80910B2D9B
:10F3E00090910C2D0E941DD8862F0E941D59182F18
:10F3F0006091672D7091682D8091692D90916A2D93
:10F400000E941DD8662371F060910D2D70910E2D14
:10F4100080910F2D9091102D0E941DD8862F0E9453
:10F420005C59182F60917D2D70917E2D80917F2DDC
:10F430009091802D0E941DD8662359F06091232D54
:10F440007091242D8091252D9091262D0E9488B2B7
:10F45000182F6091812D7091822D8091832D909134
:10F46000842D0E941DD8662371F06091272D709124
:10F47000282D8091292D90912A2D0E941DD8862F0C
:10F480000E949B59182F8091782D882329F0809114
:10F490001E2D0E94DA57182F8091792D882329F08C
:10F4A00080911F2D0E940E58182F80917C2D88234B
:10F4B00029F08091222D0E9454B2182F80917A2D2C
:10F4C000882329F08091202D0E944358182F809185
:10F4D0007B2D882329F08091212D0E947758182FA9
:10F4E00080916C2D882329F08091122D0E94F25872
:10F4F000182F80916D2D882329F08091132D0E9463
:10F500003159182F8091852D882329F080912B2D3A
:10F510000E947059182F80916E2D882329F08091B8
:10F52000142D0E94EA58182F8091E62C8D3029F076
:10F530008091702D8823A9F00FC060912C2D7091BF
:10F540002D2D80912E2D90912F2D0E947A578093F2
:10F550005038882369F32DC18091162D0E943053B5
:10F56000182F8091712D882329F08091172D0E94EA
:10F570003453182F8091722D882329F08091182DF3
:10F580000E949A53182F8091752D882329F080911D
:10F590001B2D0E947657182F8091762D882329F0F5
:10F5A00080911C2D0E943853182F4091E62C50E07A
:10F5B0004F30510508F0B4C0FA01E057FE4F0C94EB
:10F5C000F4DF0E94C356182FABC067E47DE28DEED6
:10F5D0009CE20E94CE56182FA3C00E940257182FFB
:10F5E0009FC067E47DE28DEE9CE20E940D57182FCC
:10F5F00097C00E94946F182F93C067E47DE28DEE50
:10F600009CE20E946054182F8BC00E94DD6F182F5F
:10F6100087C067E47DE28DEE9CE20E941574182F8E
:10F620007FC060912C2D70912D2D80912E2D909169
:10F630002F2D0E941DD8862F47E45DE26DEE7CE2FF
:10F640000E943C53182F6CC067E47DE28DEE9CE273
:10F650000E940A55182F64C00E94BD55182F60C023
:10F660000E942456182F5CC00E945B56182F58C069
:10F670006091192D89E19CE20E949C4F8091E72CBA
:10F68000843038F48230D8F4882349F0813079F01E
:10F6900047C0843009F044C080931D2C41C067E40A
:10F6A0007DE28DEE9CE20E949356182F39C067E4EC
:10F6B0007DE28DEE9CE20E948657182F31C0A0900B
:10F6C0003C2DB0903D2DC0903E2DD0903F2DE09030
:10F6D000382DF090392D00913A2D10913B2D20912D
:10F6E000342D3091352D4091362D5091372D8F93FB
:10F6F0008091332D8F938091322D8F938091312D76
:10F700008F938091302D8F9367E47DE28DEE9CE2A4
:10F710000E94D188182F0F900F900F900F900F908C
:10F7200060E089E19CE20E949C4F8091422D8130F3
:10F7300061F48091E82C811104C00E949C5A812FB1
:10F7400038C00E94CD5A812F34C0812F32C08BEC3B
:10F7500030C083E02EC084E82CC083E82AC0109219
:10F7600050386091E92C7091EA2C8091EB2C9091AB
:10F77000EC2C0E94364F80916B2D882309F406CE25
:10F78000FFCD85E616C086E614C0822D90E0FC0110
:10F79000E154F109EA31F10500F7E156FE4F0C940E
:10F7A000F4DFD8018C9174C968018B2D78017B2C12
:10F7B0003EC92796CDBFDEBFDF91CF911F910F913C
:10F7C000FF90EF90DF90CF90BF90AF909F908F9081
:10F7D0007F906F905F904F903F902F900895CF93C0
:10F7E000DF93EC0162E677E30E94A86680935038CD
:10F7F000811102C095E09F83DF91CF910895FC01B4
:10F800008789908D0C94E37483FF06C0E091BB2937
:10F81000F091BC2990E2958382FF06C0E091BD295A
:10F82000F091BE2990E2958381FF06C0E091BF2947
:10F83000F091C02990E2958380FF06C0E091C12934
:10F84000F091C22980E28583089583FF06C0E0918C
:10F85000BB29F091BC2990E2968382FF06C0E0911B
:10F86000BD29F091BE2990E2968381FF06C0E09108
:10F87000BF29F091C02990E2968380FF06C0E091F5
:10F88000C129F091C22980E2868308958091453490
:10F89000811107C084E00E94047C81E0809345349C
:10F8A000089584E00E94257C109245340895CF92FB
:10F8B000DF92EF92FF920F931F93CF93DF93C12CB0
:10F8C00026E0D22EC092AB29D092AC2930EAE32EAA
:10F8D00036E0F32EE092AD29F092AE2900E816E072
:10F8E0000093AF291093B029C0E6D6E0C093B129A8
:10F8F000D093B229C092B329D092B429C093B5292C
:10F90000D093B6290093B7291093B829E092B9296A
:10F91000F092BA292DEC3CEC4CED50E40E94ACD9AD
:10F92000C092BB29D092BC29E092BD29F092BE2999
:10F9300018164CF4C093BF29D093C0290093C12955
:10F940001093C22908C00093BF291093C029C09307
:10F95000C129D093C229DF91CF911F910F91FF90C0
:10F96000EF90DF90CF9008950E948DD560E070E019
:10F9700080E091E40E94577C0C94ACD581E08093A8
:10F980004E34089520E093E088ED08B618BE84BF99
:10F99000909380002091820021FDFCCF08BEFFCF14
:10F9A00080914E3481110E94C27C83E00895809141
:10F9B0004F34882341F0F89461E089E790E00E9499
:10F9C0008FD582E0089583E00895CF93DF93CDB77C
:10F9D000DEB7AD97CDBFDEBF21E2EEEEF1E2DE0194
:10F9E000119601900D922A95E1F722E02093CA0129
:10F9F000DE019296E8E0F0E024912D933196EE300E
:10FA0000F105D1F72DE228A7E0E1F0E0E491EF71F4
:10FA100021E030E02C0F3D1F2E0F311DF901208118
:10FA200029A7E2E1F0E0E491EF719E012E0F311D74
:10FA3000F90121812AA7E4E1F0E0E491EF719E0150
:10FA40002E0F311DF90121812BA71CA61092CA018E
:10FA500025E0FC012783BE016E5D7F4F0E94A866F2
:10FA600080935038AD96CDBFDEBFDF91CF91089522
:10FA700081E080934F3480E00895CF93DF93EC01D1
:10FA800020E030E040E051E469857A858B859C85F3
:10FA90000E94ACD918166CF0CE010E94D263698521
:10FAA0007A858B859C850E94577C0E9465C080E08A
:10FAB00001C08BE6DF91CF91089565E07CE30C9463
:10FAC000F8C567EE7BE30C94F8C568EC7BE30C9417
:10FAD000F8C56AEA7BE30C94F8C566E97BE30C940D
:10FAE000A3C5CF93DF938BE497E49F938F93C0EDEF
:10FAF000D4E589818F9388818F930E9469E485E1A1
:10FB000095E49F938F9389818F9388818F930E942F
:10FB100069E48DE894E49F938F9389818F93888122
:10FB20008F930E9469E483EC93E49F938F93898180
:10FB30008F9388818F930E9469E40E9450AC8DB7A7
:10FB40009EB740968DBF9EBF80E0DF91CF91089514
:10FB5000CF93DF938EE993E49F938F93C0EDD4E529
:10FB600089818F9388818F930E9469E480E392E476
:10FB70009F938F9389818F9388818F930E9469E4EB
:10FB800085EA90E49F938F9389818F9388818F93E7
:10FB90000E9469E48DE894E49F938F9389818F9309
:10FBA00088818F930E9469E483EC93E49F938F9301
:10FBB00089818F9388818F930E9469E48DB79EB766
:10FBC00044968DBF9EBF80E0DF91CF910895CF9383
:10FBD000DF9384E890E49F938F93C0EDD4E589810F
:10FBE0008F9388818F930E9469E486E09DE39F93C1
:10FBF0008F9389818F9388818F930E9469E483EC2E
:10FC000093E49F938F9389818F9388818F930E9430
:10FC100069E48DB79EB70C968DBF9EBF80E0DF91E3
:10FC2000CF910895CF93DF938EED9CE39F938F93B5
:10FC3000C0EDD4E589818F9388818F930E9469E418
:10FC40008DE69CE39F938F9389818F9388818F9317
:10FC50000E9469E483EC93E49F938F9389818F934F
:10FC600088818F930E9469E48DB79EB70C968DBFF3
:10FC70009EBF80E0DF91CF910895CF93DF938AE418
:10FC80009CE39F938F93C0EDD4E589818F93888106
:10FC90008F930E9469E481E29CE39F938F93898113
:10FCA0008F9388818F930E9469E483EC93E49F9300
:10FCB0008F9389818F9388818F930E9469E48DB798
:10FCC0009EB70C968DBF9EBF80E0DF91CF910895C7
:10FCD0002F923F924F925F926F927F928F929F925C
:10FCE000AF92BF92CF92DF92EF92FF920F931F934A
:10FCF000CF93DF93CDB7DEB76A97CDBFDEBF5C0190
:10FD00000E94E8652C011F86188A198A1A8AF50153
:10FD100001900020E9F73197EA19FB09E130F24040
:10FD200008F002C2D5018C91882359F17501BFEF0B
:10FD3000EB1AFB0A850120E0211115C0883229F059
:10FD40008132C8F08F37B9F001C021E06801EFEFD0
:10FD5000CE1ADE0A90E02A8F0E9473E3D8018C93BA
:10FD600086012A8D08C021E0893209F420E0F801DB
:10FD700080830F5F1F4FD7018D917D018111DCCFF3
:10FD800001C08501F801108210925038FDE19F2ECC
:10FD9000AAE36A2EA2E27A2E812CB6E02B2E03C0B3
:10FDA0009A9409F49CC18BE79CE2A2E2B0E08B87B5
:10FDB0009C87AD87BE876B8A7C8A8D8A8DE79CE2A3
:10FDC000A2E2B0E08F839887A987BA87EFE0F2E2DA
:10FDD000DE011196822D01900D928A95E1F7C20104
:10FDE0000E94EF648501075F1F4F75019FEFA91AFD
:10FDF000B90AD7016C9170E0CE010B960E94D0E356
:10FE0000892B21F487010E5D1F4F04C0A016B10697
:10FE100061F793C16501BFEFAB1ABB0AF6016081C0
:10FE200070E0CE0143960E94D0E3892B91F0D60179
:10FE30001D928D0192012F5E3F4F288F398F46E032
:10FE400050E0B701C9010E94FBE33AE0C30ED11CA8
:10FE500004C0A016B106F1F670C15801D8013D905A
:10FE60008D01E32CF12CC7010E9457E3892B59F433
:10FE7000B701CE0101960E94D0E3892B21F40C1525
:10FE80001D0559F75AC18501BEE63B1641F0E2E275
:10FE90003E120CC0D50111968C918232A9F5F20167
:10FEA00017821186128613861486A3C0B0E3EB1A5C
:10FEB000F108EAE0EE16F10418F0FDE23F1217C077
:10FEC000BE016A5E7F4FC5010E94FADFD20119961A
:10FED0006D937D938D939C931C978E899F898A1532
:10FEE0009B0509F42DC1E4E01796EC9382C0FBE773
:10FEF0003F124FC0E7E0D2011796EC93FFEFAF1A25
:10FF0000BF0AE2E0FE2E95C02FEFA21AB20AE5E08A
:10FF1000D2011796EC9362E270E0C5010E94D0E333
:10FF20008E8B9F8B009709F408C1DC011C92F501B0
:10FF300001900020E9F73197EA19FB093397C8F0DF
:10FF4000F80181818033A9F48281883791F440E0FF
:10FF500050E060E070E0C5010E946BE1D2011996AB
:10FF60006D937D938D939C931C9783E017968C9350
:10FF700008C0B501C2010E94A86680935038811163
:10FF800053C0AE88BF88BFEFAB1ABB0AAE8ABF8A28
:10FF900030C0E4E73E120EC0E1E0D2011796EC93C8
:10FFA00080E090E0A0E8BFE3F20181879287A38719
:10FFB000B4871FC0F6E63F120CC0E1E0D2011796ED
:10FFC000EC93179719961D921D921D921C921C97E7
:10FFD00010C0BBE53B12B1C0F2012782B501C201DE
:10FFE0000E94A8668093503881111EC07BE6F72ED0
:10FFF0007DC0BE01695F7F4FC5010E9415E45C01B1
:020000021000EC
:10000000009709F49AC0DC018C918D3729F4119680
:100010008C91F50131965F018C3209F48BC0FFEFB2
:10002000AF1ABF0AF12C05C0F82E22E0281708F4F9
:100030005DC08F858201035F1F4F882341F043E03D
:1000400050E0BE01615F7F4FC8010E94FBE3688DF5
:10005000798DC8010E944964D20114968D939C93B6
:1000600015978F3FBFEF9B07B9F10E9478698823EE
:1000700071F0888D998D0E943264882341F043E0AD
:1000800050E0688D798DCE010F960E94FBE3F2015E
:10009000428053804114510411F1F11081CE8091BE
:1000A000D42E811108C08DEC9EE20E94C86080931E
:1000B0005038F82E1BC08091E92B823099F08DECDE
:1000C0009EE20E949E608093503881110EC08DEC9C
:1000D0009EE20E941B610AC064E6F62E07C05DE640
:1000E000F52E04C04BECF42E01C0F82E42E060E087
:1000F0008F2D0E944F6781E00E940EAE6A96CDBFA1
:10010000DEBFDF91CF911F910F91FF90EF90DF90B5
:10011000CF90BF90AF909F908F907F906F905F90A7
:100120004F903F902F90089587E68093503837E6A0
:10013000F32EDCCF22E0F22E7CCF9CE6F92ED6CF38
:1001400086E6F82ED3CF2F923F924F925F926F9216
:100150007F928F929F92AF92BF92CF92DF92EF9257
:10016000FF920F931F93CF93DF9300D000D0CDB7B2
:10017000DEB78C0169837A834B835C835A0128E064
:10018000A21AB108A60EB71EDC0116967C907B0160
:10019000BFEFEB1AFB0A8BE7FB01808380E0912C19
:1001A00095E0692E29E1422E22E2522E35E1232EDE
:1001B00032E2332E4DE7842EED82FE82D80117966F
:1001C0009C919F3F09F429C1882339F02CE2ED81ED
:1001D000FE8120833196ED83FE838091FA37811171
:1001E00019C0C80141969F938F933F922F923E81F1
:1001F0003F938D818F930E9434E5AD81BE81A80F1E
:10020000B91FAD83BE830F900F900F900F900F908A
:100210000F9018C0C80141969F938F935F924F92A1
:10022000BE81BF93ED81EF930E9434E52D813E8125
:10023000280F391F2D833E830F900F900F900F9042
:100240000F900F90D80117968C911797843059F51D
:100250001996CD90DD90ED90FC901C97A70196012A
:10026000C701B6010E946FDB811117C0E894F7F84F
:100270002FEF3FEF4FE75FE7C701B6010E946FDB4B
:10028000811121C12FEF3FEF4FE75FE7C701B601B3
:100290000E94A9D718160CF016C1F8011186128613
:1002A0001386148610C1811113C0EFE1F2E2AD8113
:1002B000BE81862D01900D928A95E1F72D813E81B8
:1002C0002C5F3F4F2D833E83D80117968C9199C0A8
:1002D000823061F4F80184858F9383858F938285C2
:1002E0008F9381858F93A4E2B2E214C0833029F505
:1002F000D8011C968C911C978F931B968C911B9701
:100300008F931A968C911A978F9319968C918F933D
:10031000AAE2B2E2BF93AF93FE81FF932D812F93A8
:100320000E9434E5AD81BE81A80FB11DAD83BE83AF
:10033000F8018781CDBFDEBF64C0853059F4D80194
:1003400058968C9158978F9357968C918F93A2E3E0
:10035000B2E20CC0863009F5D80158968C915897B6
:100360008F9357968C918F93A7E3B2E2BF93AF938D
:10037000FE81FF932D812F930E9434E5AD81BE81D4
:10038000A80FB11DAD83BE83F80187810F900F9038
:100390000F900F900F900F9034C0813091F52CEAA0
:1003A00035EC47E257E3D80119966D917D918D9117
:1003B0009C911C970E94A9D787FF12C0ECE3F2E240
:1003C000AD81BE8186E001900D928A95E1F7ED81C5
:1003D000FE813596ED83FE83D80117968C9111C06E
:1003E000E2E4F2E2AD81BE81862D01900D928A9504
:1003F000E1F7ED81FE813496ED83FE83D8011796F7
:100400008C91873049F42BE7ED81FE812083319672
:10041000ED83FE8380E001C081E0AD81BE81AA153D
:10042000BB0518F08FEF9FEF65C0F80102811381C3
:100430000115110549F0D80116969C912FEF290D51
:1004400099153CF0992EBACEED80FE807914B4F067
:1004500020C0ED81FE81D801CF01019680821696E1
:100460009C9016973FEF320F92161CF4232FFC013D
:10047000F3CF8D839E838D0181E0A0CEF7012DE720
:10048000CF01019620839A94791414F4FC01F8CFDB
:100490007C018DE79AE0A0E0F70180839183A2833D
:1004A000F2E0EF0EF11C89819A812B813C81820F51
:1004B000931F8E159F0508F4B5CFC701A981BA8196
:1004C0008A1B9B0B17C0C8010E948869F8014185EF
:1004D00052856385748520858D819E810E94C2C866
:1004E0002D813E81280F311D2D833E83D801179623
:1004F0008C9187CF2696CDBFDEBFDF91CF911F9124
:100500000F91FF90EF90DF90CF90BF90AF909F90B2
:100510008F907F906F905F904F903F902F900895B5
:1005200040E052E062E675E30E94A3806091D054FF
:100530007091D15482E695E30C94B8E4CF92DF92A7
:10054000EF92FF920F931F93CF93DF93CDB7DEB758
:100550006B97CDBFDEBFF82E9091F837992309F441
:10056000F3C02CE6821310C00E94E86562E677E3D0
:1005700083E694E30E94A2C8BC018DE091E20E9450
:1005800006670DEC1EE24AC08091E92B0DEC1EE2DD
:10059000882309F443C0EE24EA94C8010E94AF64A2
:1005A0008823E1F1823029F48091FF37811120C046
:1005B0001DC0843029F48091FC37811119C016C008
:1005C0008530B1F48091FE37882381F0F801818570
:1005D0009285A385B485BC01CD019F772CEA35ECCB
:1005E00047E257E30E94A9D787FF02C0F801E782DC
:1005F000F801028113810115110579F60FC0F80188
:10060000028113810115110549F440E052E062E6D0
:1006100075E384EB9EE20E94A38096C0F801978167
:100620009F3F69F7809142348F93809141348F933B
:100630001F92FF921F9281E08F9387E492E29F9333
:100640008F939E012F5F3F4F7901FF922F930E945E
:1006500034E51092413410924234B701C8010E942F
:10066000A8668091F937F801868386E0878386E65D
:1006700090E0818B928B1282138240E052E062E61E
:1006800075E384EB9EE20E94A380CDBFDEBF893F6D
:1006900031E0930708F058C08C01FC01EE59FA4C88
:1006A0002081203309F441C06C0184ECC81A8EEF1C
:1006B000D80AD601AA5DBB4CB801615071098E9170
:1006C0008033D9F76D597A4C7E0193E1E90EF11C24
:1006D000C7012B8F0E94E4E32B8D2C3241F0F601F1
:1006E000EA5DFB4C0150110982918C32D9F7B801B7
:1006F00082E695E30E94CBC9FF92EF929F938F937E
:1007000082E592E29F938F930D591A4C1F930F939A
:100710000E9434E56091D0547091D15482E695E303
:100720000E94B8E4CDBFDEBF0FC07E01F3E1EF0E43
:10073000F11CBC016D597A4CC7010E94E4E3980199
:10074000245C3E4F6901CBCF6B96CDBFDEBFDF91FE
:10075000CF911F910F91FF90EF90DF90CF90089570
:10076000613019F0623029F008958DEC9EE20C940E
:1007700090820C949E82CF92DF92EF92FF92FC01C6
:10078000C184D284E384F48420E030E040EA50E481
:10079000C701B6010E94ACD918160CF453C0C701AA
:1007A000B6010E941DD86093F8371092FB37109263
:1007B000FC371092FD371092FE371092FF3720E081
:1007C00030E040E85FE3C701B6010E94ACD987FD85
:1007D00003C081E08093FB3720E030E040E050E44C
:1007E000C701B6010E94ACD987FD03C081E08093A8
:1007F000FC3720E030E040E450E4C701B6010E943D
:10080000ACD987FD03C081E08093FD3720E030E064
:1008100040E850E4C701B6010E94ACD987FD03C08F
:1008200081E08093FE3720E030E040EA50E4C701E9
:10083000B6010E94ACD987FD07C081E08093FF37E5
:1008400080E003C08BE601C080E0FF90EF90DF9076
:10085000CF9008956DEE77E40C94B9C566E977E41E
:100860000C94B9C562E677E40C94B9C5BF92CF92F7
:10087000DF92EF92FF920F931F93CF93DF93CDB749
:10088000DEB76897CDBFDEBF6B0128E1FC01DE015A
:10089000119601900D922A95E1F78AEAE82E8AE2F4
:1008A000F82E8E010F5F1F4FB12CF701808182302F
:1008B00029F4F801108211821282138280915C5314
:1008C0008B1114C020916C5330916D5340916E5335
:1008D00050916F53F80160817181828193810E94F0
:1008E0004EDAF6016083718382839383809178531B
:1008F0008B1114C0209188533091895340918A53B1
:1009000050918B53F80160817181828193810E94A3
:100910004EDAF601648375838683978380919453BE
:100920008B1114C02091A4533091A5534091A6532C
:100930005091A753F80160817181828193810E9457
:100940004EDAF60160877187828793878091B05372
:100950008B1114C02091C0533091C1534091C253A8
:100960005091C353F80160817181828193810E940B
:100970004EDAF6016487758786879787B394F5E327
:10098000EF0EF11C0C5F1F4F86E0B8128ECF6896F9
:10099000CDBFDEBFDF91CF911F910F91FF90EF9000
:1009A000DF90CF90BF900895F8940E94B47C0E948D
:1009B0002B850E94ACD50E942CCA0E941DB70E94B4
:1009C0009E740E9465C00E94D7A940E060E080E06C
:1009D0000E94ED690E9425660E9419850E941D876C
:1009E0000E94D0530E94A4D58091A200846080937D
:1009F000A2008091A20082608093A2008091A20058
:100A000081608093A20078940E9450AC0E947AC1C9
:100A10000E94486AFDCFE82FF0E0EE0FFF1FE75E6F
:100A2000F74B659174914FE450E080E098E30C94AB
:100A3000A2E380914034823041F440E060E081E004
:100A40000E94ED6980E00E94DD6B0C9473CC682FEE
:100A500081E00C9408CB10925138109252381092C9
:100A60005338109254380895CF93DF93EC018C8162
:100A70009D81880F991F880F991F209153383091BD
:100A80005438820F931F809355389093563844E022
:100A900050E06BE578E30E94A4D440915B3850911C
:100AA0005C3860915D3870915E3849875A876B87F2
:100AB0007C8780E0DF91CF9108958F929F92AF92D3
:100AC000BF92CF92DF92EF92FF92CF93DF93EC0130
:100AD0008091EA2B882369F089E0DF91CF91FF9024
:100AE000EF90DF90CF90BF90AF909F908F900C943D
:100AF000D8AB89859A85AB85BC8580935738909310
:100B00005838A0935938B0935A38CE010E94348592
:100B10008093503881116EC0C984DA84EB84FC84E0
:100B2000A7019601C701B6010E946FDB81112FC09A
:100B300046015701E894B7F82FEF3FEF4FE75FE723
:100B4000C501B4010E946FDB81110AC02FEF3FEF96
:100B50004FE75FE7C501B4010E94A9D71816BCF0A2
:100B60008090573890905838A0905938B0905A38A3
:100B7000A5019401C701B6010E943AD69F772CEADD
:100B800035EC47E257E30E94ACD9181674F5809112
:100B9000573890915838A0915938B0915A3880936D
:100BA0005B3890935C38A0935D38B0935E388C814D
:100BB0009D81880F991F880F991F2091533830917C
:100BC0005438820F931F809355389093563844E0E1
:100BD00050E06BE578E30E9435D5809057389090CF
:100BE0005838A0905938B0905A3889869A86AB8682
:100BF000BC8680E0DF91CF91FF90EF90DF90CF90A7
:100C0000BF90AF909F908F9008950E9458BC80E055
:100C1000089580915F38909160388F3E924111F035
:100C20008EE5089580917D3890917E388F3E924177
:100C3000B9F780917F38909180388F3E924181F74B
:100C40008091E84F9091E94F8F3E924149F7809112
:100C5000EA4F9091EB4F8F3E924111F780917C517A
:100C600090917D518F3E9241D9F680E0089594E0B5
:100C7000899FF0011124E15AF74C42835383648326
:100C80007583089594E0899FF0011124E651F04B9B
:100C900045AB56AB67AB70AF08955F926F927F9292
:100CA0008F929F92AF92BF92CF92DF92EF92FF927C
:100CB0000F931F93CF93DF93CDB7DEB76097CDBF70
:100CC000DEBFBE016F5F7F4F8FE190E50E943684EB
:100CD000CE0101964C0187E9A82E80E5B82E97EA4F
:100CE000C92E90E5D92E27EBE22E20E5F22E07ED56
:100CF00010E537EE632E33E5732E512CF40141914C
:100D00005191619171914F01F5014193519361931B
:100D100071935F01F60141935193619371936F0158
:100D2000F70141935193619371937F01852D0E9447
:100D3000C074F80111921192119211928F01F30176
:100D400010821182128213825394F8E16F0E711C8B
:100D500084E05812D3CF6096CDBFDEBFDF91CF9134
:100D60001F910F91FF90EF90DF90CF90BF90AF90C9
:100D70009F908F907F906F905F90089580918138C1
:100D800008951F93CF93DF938BE697E1EFE7F8E3A6
:100D9000DF019C011D9221503040E1F78FEE92E17E
:100DA00080937F38909380388093E84F9093E94FF9
:100DB000C8E8D8E3C0938238D0938338C09384388E
:100DC000D0938538C0938638D093873881E090E0FF
:100DD0006DE27FE420E030E01BEB129FA001139F47
:100DE000500D1124FA01E158F74CD90111961A9FC0
:100DF00090011B9F300D11242857374C23873487CF
:100E000061877287BA016857774C9C0101968032DE
:100E1000910519F78BEB829FF001839FF00D112450
:100E2000E158F74CC387D4876187728780E280934B
:100E30008138DF91CF911F910895CF93DF93EAEE30
:100E4000FFE484E991E0DF01EC011D922197E9F7CD
:100E5000AFE5B8E380E2ED0119928A95E9F78FEEEC
:100E600092E18D939C9380937D3890937E3880831C
:100E7000918380937C5190937D51DF91CF910C941D
:100E8000C1860E941F910E94C18680E00C94EB4EA7
:100E9000E0918238F0918338848581111BC02281D2
:100EA0003381808191814BEBDF011D924A95E9F7F7
:100EB000228333838083918381E08487809181388A
:100EC000815080938138828193818093823890937E
:100ED000833805C08CE10E94D8ABE0E0F0E0CF01A0
:100EE0000895A4E8B8E3ED91FC911197858781E01E
:100EF000878782E08487828193818D939C9381E0B0
:100F00000E945FAF0C949EB9EF92FF920F931F93D4
:100F1000CF93DF9300D01F92CDB7DEB78C014B8308
:100F20005C8369837A830E944887FC014B815C81E2
:100F300069817A81009761F48EE02496CDBFDEBF8F
:100F4000DF91CF911F910F91FF90EF900C94205360
:100F500083E0858785E096E88483958306831783FD
:100F60008B017A0126E0D8014D915D916D917D91C3
:100F70008D01CF0185599F4FDC014D935D936D939A
:100F80007C931397D7014D915D916D917D917D017A
:100F9000418B528B638B748B215034962111E3CF9C
:100FA00083E02496CDBFDEBFDF91CF911F910F91DB
:100FB000FF90EF900C947187CF92DF92EF92FF92A7
:100FC0006B017C010E944887009739F48EE0FF9006
:100FD000EF90DF90CF900C9420532FE538E8FC0180
:100FE00024833583E556FF4FC082D182E282F382AB
:100FF00021E0FC01278782E00E94718780E0FF905A
:10100000EF90DF90CF900895809186389091873847
:10101000FC0124853EEF320F323018F424E024879F
:101020000895243011F080E090E00895E091863832
:10103000F091873822813381808191814BEBDF01F0
:101040001D924A95E9F72283338380839183E0914F
:101050008638F09187380280F381E02DE09386385E
:10106000F09387388485823011F483E084878091FF
:1010700081388F5F809381388FEF0E945FAF81E06E
:10108000409182385091833820918638309187384A
:101090004217530709F080E00895BC016F5E7F4F4F
:1010A000DC011696ED91FC91179785599F4F199584
:1010B0000E94168881110E94695A80E00895855621
:1010C0009F4F20E034E244E759E4FC0160817181E4
:1010D000828193810E944EDA0E941DD80E9449D8D5
:1010E0000E9462BC0E94168881110E94695A80E0A9
:1010F00008958091863890918738FC0124853EEFD1
:10110000320F323018F424E024870895243011F08F
:1011100080E090E00895CF93DF93C0918638D0911E
:1011200087388C859EEF980F923018F484E08C8776
:1011300005C0843019F080E090E010C02097D9F30A
:10114000DE011296ED91FC9113978785882329F093
:10115000EC17FD0711F0DF01F4CFCD01DF91CF9146
:101160000895CF93DF93EC012A813B818881998197
:101170004BEBFB01DE0101900D924A95E1F72A83CA
:101180003B8388839983DF91CF9108958FEE92E11D
:1011900080937E5190937F51809336529093375233
:1011A00008952F923F924F925F926F927F928F920B
:1011B0009F92AF92BF92CF92DF92EF92FF920F93E6
:1011C0001F93CF93DF93CDB7DEB76D97CDBFDEBF53
:1011D0004C011B0129013A01ED86FE860F87188B11
:1011E0001A2D0B2DEBA8BCA8ADA82EA929838091A0
:1011F000622C882399F08091562C9091572CA091C5
:10120000582CB091592CBC01CD019F772CEA35ECBC
:1012100047E257E30E94A9D787FDF6C680918A2D41
:1012200090918B2DA0918C2DB0918D2DBC01CD0175
:101230009F7731E039872CEA35EC47E257E30E948B
:10124000ACD9181614F0198610C02DEC3CEC4CECFF
:101250005DE36091302D7091312D8091322D909110
:10126000332D0E94A9D787FDD1C6F10180819181DC
:10127000A281B381BC01CD019F77F1E0FD832CEA0F
:1012800035EC47E257E30E94ACD918160CF01D82EA
:10129000F10184819581A681B781BC01CD019F7741
:1012A000F1E0F98B2CEA35EC47E257E30E94ACD928
:1012B00018160CF0198AF10180859185A285B385F5
:1012C00020918E2D30918F2D4091902D5091912D08
:1012D000298F3A8F4B8F5C8F2091922D3091932DD7
:1012E0004091942D5091952D2D8B3E8B4F8B588F87
:1012F0004091962D5091972D6091982D7091992D38
:10130000F090632CF11021C01092C65181E08093BF
:10131000C75182E08093C8513985332341F04D8114
:10132000411178C65989511175C68CE9A6C6CB0101
:10133000BA019F772CEA35EC47E257E30E94ACD91B
:1013400018160CF06CC68BE998C6BC01CD019F77CE
:10135000A1E0AD8F2CEA35EC47E257E30E94ACD90F
:1013600018160CF01D8EB1E0FB1216C01092C6517B
:1013700082E08093C751F092C851E985EE2339F09D
:10138000FD81F11147C62D8D222379F243C66D8967
:101390007E898F89988DCDCF32E0F31217C081E01E
:1013A0008093C651F092C7511092C8514985442389
:1013B00041F0598951112EC68D8D882309F4B5CF7E
:1013C00029C6698D7A8D8B8D9C8DB3CFB101C401F7
:1013D0000E943A519985992309F451C020911E2CFD
:1013E00030911F2C4091202C5091212C6091722C17
:1013F0007091732C8091742C9091752C0E943AD628
:101400009F772CEA35EC47E257E30E94A9D787FF84
:1014100036C02091222C3091232C4091242C5091C5
:10142000252C6091762C7091772C8091782C90915E
:10143000792C0E943AD69F772CEA35EC47E257E3A5
:101440000E94A9D787FF1BC02091262C3091272C02
:101450004091282C5091292C60917A2C70917B2CF2
:1014600080917C2C90917D2C0E943AD69F772CEA1B
:1014700035EC47E257E30E94A9D787FDC9C58FA97C
:1014800080931D2C89E19CE20E94424F85E5E9E1B1
:10149000FCE2A1EEB1E501900D928A95E1F788E1B9
:1014A000E2E7FCE2A1E8B1E501900D928A95E1F74F
:1014B0008091642C8111B8C523E333E34BEC51E4F4
:1014C0006E2D7B2D8A2D99810E944EDA4B015C0195
:1014D0006093B5517093B6518093B7519093B851C2
:1014E00023E333E34BEC51E4C301B2010E944EDA33
:1014F0006093995170939A5180939B5190939C5112
:1015000023E333E34BEC51E46D857E858F85988929
:101510000E944EDA60939D5170939E5180939F512B
:101520009093A05123E333E34BEC51E4612F702FF0
:10153000C6010E944EDA162F072F412F502FBC01F3
:101540004093A1515093A2516093A3517093A45121
:1015500080912C2D90912D2DA0912E2DB0912F2D7D
:10156000BC01CD019F770E9486D80E941DD82B0117
:101570003C016093C2517093C3518093C4519093C6
:10158000C5511091C6518091C751A82FB0E0AD87C9
:10159000BE877D01EE0CFF1CEE0CFF1CF101EE0D71
:1015A000FF1D80819181A281B381BC01CD019F7714
:1015B0002CEA35EC47E257E30E94A9D7881F882719
:1015C000881F8983E12FF0E0E987FA878F01000FF8
:1015D000111F000F111FF101E00FF11F8081918198
:1015E000A281B381BC01CD019F772CEA35EC47E2A3
:1015F00057E30E94A9D7881F8827881FF981F823FD
:10160000F983F093C1512CEA35EC47E257E3C50169
:10161000B4019F770E94ACD9181624F00D831E8365
:10162000870105C1E985FA85EE0FFF1FEE0FFF1F49
:10163000E25EF34DA985BA85AA0FBB1FAA0FBB1F97
:10164000AE58B34D2D913D914D915C91608171816A
:10165000828193810E943AD6698B7A8B8B8B9C8B8B
:10166000ED85FE85EE0FFF1FEE0FFF1FE25EF34DCF
:10167000AD85BE85AA0FBB1FAA0FBB1FAE58B34DC9
:101680002D913D914D915C91608171818281938119
:101690000E943AD66D8B7E8B8F8B988FA50194011B
:1016A000C501B4010E944EDA20E030E040E850E489
:1016B0000E944EDA6D837E838F83988729893A89C9
:1016C0004B895C89CA01B9010E944EDA6B017C0129
:1016D0002D893E894F89588DCA01B9010E944EDA81
:1016E0009B01AC01C701B6010E943BD69B01AC0136
:1016F0006D817E818F8198850E943AD66B017C0135
:1017000020E030E0A9010E94ACD91816D4F4C7013A
:10171000B6010E9427DB6B017C012D893E894F8930
:10172000588D69897A898B899C890E94B9D99B01D6
:10173000AC01C701B60190580E94B0D76B017C0183
:1017400003C0C12CD12C760180911D2C833021F453
:10175000F7FAF094F7F8F09420E030E0A901C50121
:10176000B4010E94A9D787FF04C0F7FAF094F7F8F4
:10177000F09429853A85220F331F220F331F2D83C2
:101780003E83890102581E4AA70196016D897E8910
:101790008F89988D0E944EDA9B01AC0169897A8904
:1017A0008B899C890E943AD620E030E040E05FE3DC
:1017B0000E944EDAD8015B966D937D938D939C9336
:1017C0005E970D851E85000F111F000F111FF80178
:1017D000E258FE4A5F01A701960169897A898B89DF
:1017E0009C890E944EDA9B01AC016D897E898F89AC
:1017F000988D0E943BD620E030E040E05FE30E94FD
:101800004EDAD5015B966D937D938D939C935E9795
:10181000E091C851F0E0EE0FFF1FEE0FFF1FE258FE
:10182000FE4A138E148E158E168E10925038F801C3
:10183000E258FE4AC38CD48CE58CF68CF7FAF0940F
:10184000F7F8F094ED81FE81E258FE4A838D948D85
:10185000A58DB68DBC01CD019058A70196015F778B
:101860000E94B0D70E949FD64B015C0120E030E07F
:10187000A901C701B6010E94ACD91816C4F020E036
:1018800030E0A901B401C5010E94ACD99401A501C1
:1018900018162CF46BED7FE089E490E404C06BED46
:1018A0007FE089E490EC0E943AD64B015C01C401D0
:1018B000D5018093AD519093AE51A093AF51B093A9
:1018C000B0519401A501B401C5010E946FDB8111E3
:1018D000CFC3B981BB23B1F1C301B2010E9449D882
:1018E0006B017C012CEA35EC47E257E30E94A9D753
:1018F00087FD11C0B0901D2C2BED3FE049EC50E46A
:10190000C701B6010E944EDA9B01AC01C12CD12C5B
:10191000E12CF12CEFC081E090E0A0E0B0E08093FA
:10192000C2519093C351A093C451B093C551B0908C
:101930001D2C2BED3FE049EC50E4C12CD12CE12CC7
:10194000F12CD8C0ED85FE85EE0FFF1FEE0FFF1FB7
:10195000EA51FE4A980122583E4A7901D9015B9624
:101960002D913D914D915C915E9760817181828155
:1019700093810E943AD6F7012381348145815681B3
:101980000E943AD66B017C01E985FA85EE0FFF1FB4
:10199000EE0FFF1FEA51FE4A2D813E8122583E4A3A
:1019A0001901D9015B962D913D914D915C915E9706
:1019B00060817181828193810E943AD6F1012381F5
:1019C0003481458156810E943AD6A70196015F77FE
:1019D0000E94B0D70E949FD61B018983998B20E07B
:1019E00030E0A901C701B6010E94ACD91816E4F095
:1019F00020E030E0A901B101898199890E94ACD928
:101A000091014981598918162CF46BED7FE089E426
:101A100090E404C06BED7FE089E490EC0E943AD63C
:101A20001B01F82EE92E02C0F980E988C101AF2D13
:101A3000BE2D8093B1519093B251A093B351B09306
:101A4000B45191014F2D5E2DB1018F2D9E2D0E941D
:101A50006FDB81110DC391014F2D5E2DB401C501C6
:101A60000E94ACD91816B4F42BED3FE049EC50E4D9
:101A7000B1018F2D9E2D0E943BD61B01AB01BC01F5
:101A80004093B1515093B2516093B3517093B4519C
:101A9000F82EE92E9401A501B1018F2D9E2D0E94F3
:101AA0003AD66B017C01B0901D2CF3E0BF1669F0B3
:101AB000C301B2010E9449D82BED3FE049EC50E44C
:101AC0000E944EDA9B01AC0115C02BED3FE049ECC2
:101AD00050E40E943AD66B017C01C301B2010E941E
:101AE00049D82BED3FE049EC50E40E944EDA9B01CF
:101AF000AC0108C082E0B81205C0B601C7010E945F
:101B00003BD604C0B601C7010E943AD69B01AB0187
:101B1000BC014093B9515093BA516093BB5170933B
:101B2000BC5169017C018091632C813061F4F7FA2A
:101B3000F094F7F8F094C092B951D092BA51E09273
:101B4000BB51F092BC51F801E258FE4A238D348D0E
:101B5000458D568DED81FE81E258FE4A638D748D70
:101B6000858D968D0E94B9D969837A838B839C83F6
:101B70006093B5517093B6518093B7519093B8511B
:101B80002090C851312CF101EE0FFF1FEE0FFF1F07
:101B9000EA51FE4AD101AA0FBB1FAA0FBB1FA258D0
:101BA000BE4A13962D913D914D915C91169760819F
:101BB0007181828193810E943AD64B015C016093CE
:101BC000BD517093BE518093BF519093C051A701F6
:101BD000960169817A818B819C810E944EDA6B012A
:101BE0007C01A50194010E94B9D92B013C016093AD
:101BF000A5517093A6518093A7519093A85120911D
:101C0000F5293091F6294091F7295091F8292D8333
